:100000000C94BB0C0C94EC0C0C94EC0C0C94EC0CC1
:100010000C94EC0C0C94A1560C9433470C947D7406
:100020000C94EC0C0C94EC0C0C94EC0C0C94EC0C70
:100030000C94EC0C0C94EC0C0C94EC0C0C94EC0C60
:100040000C94EC0C0C948A810C9425560C94EC0CBA
:100050000C94EC0C0C94EC0C0C94EC0C0C948D7239
:100060000C94EC0C0C94DA4E0C94B14E0C94EC0CF9
:100070000C94EC0C0C94EC0C0C94EC0C0C94EC0C20
:100080000C94B47F0C94EC0C0C94EC0C0C94EC0CD5
:100090000C94884E0C945F4E0C94EC0C0C94EC0C6D
:1000A0000C94EC0C0C94EC0C0C94EC0C0C94EC0CF0
:1000B0000C94EC0C0C948B3E0C94EC0C0C94EC0C0F
:1000C0000C94EC0C0C94EC0C0C94EC0C0C94364E44
:1000D0000C940D4E0C94EC0C0C94E44D0C94BB4D14
:1000E0000C94EC0CDB12B8129412F8125013171384
:1000F000471336130514E213BE132214A614411439
:100100009D148C145E178C17C317FA17D018091991
:1001100042197B19571A571A571A571A571A571A4A
:10012000571A571A571A571A571A571A571A571A47
:10013000571A571A571A571A571A571A571A571A37
:10014000571A571A571A571A571A571A571A31184F
:1001500068189F18B419ED19261A3A1C401C461C41
:100160004C1C521C581C5E1C641C6A1C701C761CA7
:100170007C1C8E1C941C9A1CA01CA61CAC1CB21CC3
:10018000B81CBE1CC41CCA1CD01CD61CDC1CE21C27
:10019000E81CEE1CF41C001D061D0C1D121D2A1D62
:1001A000301D361D3C1D421D481D961D9C1DA21D67
:1001B000AE1DB41DBA1DC61DCC1DD21DD81DDE1D21
:1001C000E41DF61DFC1D021E081E0E1E141E2C1E14
:1001D000321E381E3E1E561E5C1E621E681E6C1E9F
:1001E000701E741E7A1E7E1E821E861E8A1E8E1E23
:1001F000921E981E9E1EA41EAA1EB01EB61EBC1ED7
:10020000C21E181D4E1D541D5A1D601D661D6C1DFD
:100210001A1E201E261E441E4A1E501EC81ECE1E1A
:10022000D41EEA1DF01D721D781D7E1D841D8A1DC1
:10023000901DA81DC01DFA1C821C881C1E1D241D9B
:10024000DA1EE01EE61EC431C431DE31C431EB31AA
:1002500004321F323A32B83EC13EC93EDD3EEF3E67
:10026000013F0C3FB44AB74AA64AAA4AB04AEE4AEE
:10027000BB4ABF4AC54AC94ACD4AD34AD74ADB4AD4
:10028000EE4AE14AE54AE94A445049504E50585036
:100290006250DB506C5074507C50865090509A5095
:1002A000A950B350DB50BD50C750D150237557757E
:1002B0008C75AC75E1751676267650779A76A476AD
:1002C000D8760D771B7781869886AF86C686DD86C1
:1002D000F4860B8722873A87598770878787A68796
:1002E000BC87212000464143544F52592052455368
:1002F00045542120003400330032004E6F6E6500FB
:1003000053746F70706564004E65757472616C2013
:100310005475726E004D6F76696E67205265766512
:10032000727365004D6F76696E6720466F727761F4
:100330007264004272616B696E670054414E4B20DB
:10034000524553544F5245440025004865616C7432
:1003500068204C6576656C3A200056454849434C08
:10036000452052455041495220434F4D504C455431
:10037000450054414E4B2044455354524F59454437
:100380000025004865616C7468204C6576656C3AA0
:100390002000290056454849434C452052455041CC
:1003A000495220535441525445442028005245504C
:1003B000414952204F5045524154494F4E204341EC
:1003C0004E43454C4C45440029004D414348494E5D
:1003D000452047554E204849542120280052455079
:1003E000414952204F5045524154494F4E204341BC
:1003F0004E43454C4C454400290043414E4E4F4E20
:100400002048495421202800547572726574207266
:100410006F746174696F6E206973206E6F74206FE2
:1004200066207479706520536572766F2E204E6F4A
:1004300020736574757020617661696C61626C65AA
:100440002E0054757272657420656C6576617469EE
:100450006F6E206973206E6F74206F6620747970E0
:100460006520536572766F2E204E6F20736574750C
:100470007020617661696C61626C652E00546F70EA
:10048000204C65667400546F702043656E7465720D
:1004900000546F70205269676874004D6964646C21
:1004A00065204C656674004D6964646C6520436525
:1004B0006E746572004D6964646C6520526967688A
:1004C0007400426F74746F6D204C65667400426FE7
:1004D00074746F6D2043656E74657200426F74743E
:1004E0006F6D205269676874004649524D574152FA
:1004F000452056455253494F4E3A20006942757384
:1005000000534275730050504D004E6F6E6520448D
:100510006574656374656400417A696D75746820FB
:1005200020202000456C65766174696F6E20200084
:100530005475726E20202020202020005468726F95
:1005400074746C6520202000537469636B20202034
:10055000202020204D696E2020202043656E746588
:10056000722020204D617820202020446561646243
:10057000616E642020526576657273656400524135
:1005800044494F20494E464F202D20004E4F5420C5
:1005900044455445435445440049474E4F52454411
:1005A00000416E616C6F67004469676974616C003B
:1005B000417578204368616E2E2020204D696E20A1
:1005C000202020204D617820202020205479706543
:1005D000004368616E6E656C73207574696C697A2E
:1005E00065643A20004368616E6E656C73206465D3
:1005F0007465637465643A20004D656368616E6973
:1006000063616C207265636F696C00416972736F1E
:100610006674004D656368616E6963616C20426158
:100620007272656C3A200020284D31290020284D37
:10063000322900202842290042617272656C2045EF
:100640006C65766174696F6E3A20200020284D3009
:10065000290020284D312900202841290054757295
:1006600072657420526F746174696F6E3A20202035
:10067000004472697665204D6F746F72733A202062
:1006800020202020004D4F544F52205459504553A4
:100690000054616E6B2028444B4C4D20747970657A
:1006A00029004361720048616C66747261636B007B
:1006B00054616E6B00554E4B4E4F574E005965734B
:1006C000004E6F002900252C20446563656C65721F
:1006D0006174696F6E20666163746F7220002028F8
:1006E0004B69636B6261636B2073706565642000A6
:1006F000547261636B205265636F696C20456E6153
:10070000626C65643A202020004E2F4120666F7293
:100710002076656869636C6520747970650054752E
:10072000726E204D6F64653A20202020202020200A
:10073000202020202020004E2F4120666F7220763E
:10074000656869636C652074797065002500202DEB
:1007500020004E65757472616C205475726E204174
:100760006C6C6F7765643A2020200020736563000D
:100770005472616E736D697373696F6E2044656C3A
:1007800061793A2020202020002073656300456EA7
:1007900067696E652050617573652054696D653AAF
:1007A00020202020202000207365630053686966A4
:1007B000742054696D653A202020202020202020BC
:1007C00020202020004175746F6D61746963004DB5
:1007D000616E75616C005472616E736D69737369DB
:1007E0006F6E20547970653A20202020202000254B
:1007F00000596573202D200052657665727365205F
:100800005370656564204C696D697465643A202095
:10081000002500596573202D2000466F72776172A4
:1008200064205370656564204C696D697465643A31
:10083000202000206D73290025207468726F747465
:100840006C6520666F7220002028004D6F746F72F7
:10085000204E7564676520456E61626C65643A2060
:100860002020200029004E6F6E65004E6F6E6500DF
:100870002C205072657365743A20002900202841AD
:10088000646A757374656420746F200020284C6559
:1008900076656C3A2000446563656C2052616D702A
:1008A00020456E61626C65643A202020202000297A
:1008B000004E6F6E65004E6F6E65002C20507265A5
:1008C0007365743A20002900202841646A757374A6
:1008D000656420746F200020284C6576656C3A2092
:1008E00000416363656C2052616D7020456E6162EA
:1008F0006C65643A2020202020004163746976658D
:100900002044726976696E672050726F66696C6503
:100910003A200056656869636C6520547970653AC1
:100920002020202020202020202020004452495632
:10093000452053455454494E475300207365630086
:100940005265636F696C2064656C61793A20202080
:100950002020202020202020202020202020202097
:10096000002500596573202D200042617272656C6C
:1009700020456C65766174696F6E2053706565649F
:10098000204C696D697465643A20002500596573CF
:10099000202D200054757272657420526F7461743A
:1009A000696F6E205370656564204C696D6974656C
:1009B000643A202000545552524554205345545413
:1009C000494E475300556E6B6E6F776E00486561F8
:1009D0007679004D656469756D004C6967687400CF
:1009E000437573746F6D00556E6B6E6F776E004F4D
:1009F00070656E2050616E7A65720054616D697920
:100A00006120537065630020736563207265636FB6
:100A1000766572792900207365632072656C6F6159
:100A2000642C2000204D4720686974732C2000201E
:100A300063616E6E6F6E20686974732C20002800ED
:100A400057656967687420436C6173733A2020208E
:100A500020200044616D6167652050726F66696C8B
:100A6000653A2020200059657320280041636365A2
:100A70007074204D472044616D6167653A200059CC
:100A8000657320280053656E64204D47204952202D
:100A9000436F64653A2020004E2F4100526570611B
:100AA000697265642062793A202020202020004E5F
:100AB0002F41004869742050726F746F636F6C200F
:100AC000323A20202000290020285465616D200042
:100AD000466972652050726F746F636F6C3A2020A4
:100AE000202000466972652050726F746F636F6CCE
:100AF0003A202020200049732052657061697220DD
:100B000054616E6B3F202020004952202620546102
:100B10006E6B20426174746C696E67204469736106
:100B2000626C656400424154544C4520494E464F26
:100B300000554E4B4E4F574E0042656E6564696ED0
:100B40006920544253204D6963726F0042656965A4
:100B5000722055534D2D52432D3200546169676503
:100B60006E20536F756E642043617264004F706530
:100B70006E2050616E7A657220536F756E642043EB
:100B80006172640042656E6564696E692054425307
:100B9000204D696E6900536F756E642063617264E5
:100BA0003A2000534F554E44204341524400486977
:100BB0006C6C205068797369637320456E61626C58
:100BC00065643A20202020202020202000426172ED
:100BD00072656C2053746162696C697A6174696FC3
:100BE0006E20456E61626C65643A200053656E73D9
:100BF0006F722064657465637465643A20202020F8
:100C000020202020202020202020596573005365BB
:100C10006E736F72206E6F742064657465637465A3
:100C2000642100494E45525449414C204D454153A1
:100C30005552454D454E5420554E495400556E6B06
:100C40006E6F776E005370656564206465637265CE
:100C5000617365732062656C6F7720005370656502
:100C60006420696E637265617365732061626F767B
:100C700065200056656869636C652044657374720D
:100C80006F7965640043616E6E6F6E204869740011
:100C90004272616B6573204170706C6965640056C7
:100CA00061726961626C650020286F6620352900D9
:100CB0003320286F66203329003220286F662033C6
:100CC00029003120286F66203329003220286F66E2
:100CD000203229003120286F6620322900506F739E
:100CE0002000417578204368616E6E656C20005667
:100CF00061726961626C65004F6E004F666600420A
:100D000000410045787465726E616C20496E7075A3
:100D1000742000070809090B0C0C0B0C0C5475729D
:100D200072657420537469636B202D200046756EC4
:100D30006374696F6E202300202D3E2000207365B0
:100D40006300547572726574206D6F76656D656EA3
:100D5000742064656C61793A2020004E6F6E6500E6
:100D60005965730054757272657420737469636B8E
:100D70002066756E6374696F6E733A200046554E37
:100D80004354494F4E2054524947474552530076E9
:100D9000206375746F666629002028004C56432036
:100DA000456E61626C65643A202020202020007628
:100DB00000566F6C746167653A2020202020202047
:100DC00020202000596573004E6F004261747465E5
:100DD00072792044657465637465643A2000424109
:100DE00054544552590053657269616C2033205444
:100DF0007820426175643A2020004175782053655F
:100E00007269616C20426175643A202020004D6F48
:100E1000746F722053657269616C20426175643A27
:100E200020005553422053657269616C2042617500
:100E3000643A2020200042415544205241544553F9
:100E400000524144494F204641494C5341464500D8
:100E5000526164696F205265616479202D200052CF
:100E6000657665727365643A2020004D6178205084
:100E7000756C73653A20004D696E2050756C736512
:100E80003A2000456E642056616C75657300456EAE
:100E900064205265636F696C20536572766F2053CE
:100EA0006574757000456E6420526F746174696F6B
:100EB0006E20536572766F20536574757000456EB1
:100EC0006420456C65766174696F6E205365727637
:100ED0006F20536574757000536572766F20756E60
:100EE0002D726576657273656400536572766F2046
:100EF00072657665727365640052657665727365B6
:100F0000643A2020004D61782050756C73653A205A
:100F1000004D696E2050756C73653A200053746102
:100F200072742056616C75657300494E56414C4988
:100F30004420534552564F2E204E4F205345545572
:100F4000502E005365747570205265636F696C2074
:100F5000536572766F0053657475702054757272A4
:100F6000657420526F746174696F6E2050616E20D9
:100F7000536572766F005365747570205475727284
:100F8000657420456C65766174696F6E2050616E82
:100F900020536572766F0000002100240027002A8C
:100FA000002D003000330001010000040107010A98
:100FB0000100002200250028002B002E0031003403
:100FC0000002010000050108010B010000200023C0
:100FD00000260029002C002F003200000100000331
:100FE00001060109010505050507050808080802AD
:100FF0000202020A0A0808040404040101010101B2
:101000000101010303030303030303040707070CA0
:101010000C0C0C0C0C0C0C02020202060606060656
:101020000606060B0B0B0B0B0B0B0B010210202003
:10103000080810204010204080020102010804022C
:1010400001010204081020408080402010080402A2
:1010500001800402018040201008040201080402FB
:101060000101020408102040800102040810204001
:101070008000000A0B02090C0D0E08070304010092
:101080000000000000000000000000000000000060
:10109000000000000000000000000000001211101D
:1010A0000000000000000000000000000000000040
:1010B00000000000000000556E6B6E6F776E0044FC
:1010C000657461636865642F4E41005265636F69A2
:1010D0006C20536572766F0050616E205365727696
:1010E0006F00536572766F2F455343004F6E626FEA
:1010F000617264204D6F746F7220447269766572FC
:10110000004F70656E2050616E7A65722053636F78
:1011100075742053657269616C20455343005361B7
:10112000626572746F6F74682053657269616C00D8
:10113000506F6C6F6C752053657269616C005365FC
:1011400072766F203100536572766F2032005365DE
:1011500072766F203300536572766F2034005365CA
:1011600072766F203500536572766F2036005365B6
:1011700072766F203700536572766F203800456EA7
:1011800067616765205472616E736D697373696F0F
:101190006E00446973656E67616765205472616EA5
:1011A000736D697373696F6E005365742054757243
:1011B0006E204D6F64653A2031005365742054757C
:1011C000726E204D6F64653A20320053657420546E
:1011D00075726E204D6F64653A203300456E616212
:1011E0006C65204E65757472616C205475726E73F7
:1011F0000044697361626C65204E65757472616C40
:10120000205475726E730042617272656C20537463
:101210006162696C697A6174696F6E3A20547572A3
:101220006E6564204F4E0042617272656C2053748B
:101230006162696C697A6174696F6E3A2054757283
:101240006E6564204F46460048696C6C2050687992
:10125000736963733A205475726E6564204F4E0053
:1012600048696C6C20506879736963733A205475CF
:10127000726E6564204F464600494F20506F72746D
:101280002041204F7574707574202D204F6E0049D9
:101290004F20506F72742041204F75747075742008
:1012A0002D204F666600494F20506F7274204220F7
:1012B0004F7574707574202D204F6E00494F20506B
:1012C0006F72742042204F7574707574202D204FFA
:1012D0006666004C56432045786974202D20566F71
:1012E0006C7461676520526573746F726564007613
:1012F00029004C5643207468726573686F6C6420D3
:1013000072656163686564212028004C69676874B0
:101310002031204F6E004C696768742031204F6681
:1013200066004C696768742032204F6E004C696714
:1013300068742032204F666600326E64204D47206C
:1013400053746F7000326E64204D47205374617285
:10135000740052756E6E696E67204C6967687473AD
:10136000204F6E0052756E6E696E67204C6967681B
:101370007473204F666600417578204F75747075E0
:1013800074204F6E00417578204F7574707574200D
:101390004F66660053746F70205265766F6C766985
:1013A0006E6720417578204C696768740053746FCC
:1013B0007020417578204F757470757420426C6987
:1013C0006E6B696E6700537461727420417578208A
:1013D0004F757470757420426C696E6B696E67002E
:1013E00036202D20537461727420526570656174CB
:1013F000696E670036202D2053746F700055736539
:10140000722046756E6374696F6E20310055736586
:10141000722046756E6374696F6E203200466F727B
:10142000776172642047656172004E657574726100
:101430006C2047656172005265766572736520475E
:101440006561720053657420416363656C2052616D
:101450006D70204C6576656C3A20005365742044AD
:101460006563656C2052616D70204C6576656C3AE1
:1014700020005365742042617272656C2053656E62
:1014800073697469766974793A20005365742048E9
:10149000696C6C2053656E73697469766974793A06
:1014A0002000416E616C6F67205573657220467530
:1014B0006E6374696F6E2031202D2000416E616C67
:1014C0006F6720557365722046756E6374696F6E21
:1014D0002032202D20002D00202D200020005452ED
:1014E00055450046414C53450025005761697469D4
:1014F0006E6720666F7220726164696F2E2E2E20D7
:1015000000466972652043616E6E6F6E00466972B7
:101510006520526570616972205369676E616C0065
:10152000416972736F6674202D204D616E75616C18
:101530002054726967676572004D656368616E6902
:1015400063616C205265636F696C202D204D616E64
:1015500075616C20547269676765720053657276B5
:101560006F205265636F696C202D204D616E75612F
:101570006C20547269676765720048696768204922
:101580006E74656E7369747920466C61736820555A
:101590006E6974202D204D616E75616C20547269E6
:1015A00067676572004D47205374617274004D4740
:1015B0002053746F7000417578204F757470757486
:1015C000205072657365742044696D004175782000
:1015D0004F757470757420466C6173686564004162
:1015E0007578204F757470757420496E76657273C6
:1015F0006520466C61736865640053746F702041A8
:101600007578204F757470757420426C696E6B69C3
:101610006E670053746F70205265766F6C76696EDA
:101620006720417578204C6967687400310031206B
:101630002D20537461727420526570656174696EF7
:10164000670031202D2053746F7000320032202D3E
:1016500020537461727420526570656174696E679D
:101660000032202D2053746F7000330033202D2062
:10167000537461727420526570656174696E67009D
:1016800033202D2053746F7000340034202D2053EC
:101690007461727420526570656174696E6700349C
:1016A000202D2053746F7000350035202D20537489
:1016B00061727420526570656174696E67003520CF
:1016C0002D2053746F70003600401F7017D007A094
:1016D0000FA00FDC05D007C40910278813983A1013
:1016E000276C023A026C023A026C023A026C02B0B7
:1016F00036384A5C121C255C125C121C255C12BC3C
:101700007FC7F2C07887A5B7C5A00F8813B80B4074
:101710001FB80BB80B7017401F2900202D20416403
:101720006A757374656420746F2000202853656E99
:10173000736974697669747920002900202D20412D
:10174000646A757374656420746F20002028536583
:101750006E73697469766974792000537461727468
:10176000205265766F6C76696E6720417578204CE3
:101770006967687400536F6E790052435441204D7D
:10178000616368696E652047756E00436C61726BBA
:10179000204D616368696E652047756E0052435441
:1017A000412052657061697200494255205265704E
:1017B00061697200436C61726B205265706169727D
:1017C000004F70656E50616E7A6572005673546199
:1017D0006E6B00464F560054616967656E00486540
:1017E0006E67204C6F6E670054616D6979612031BE
:1017F0002F33350054616D69796120322D53686F44
:10180000740054616D69796100556E6B6E6F776E0F
:10181000003A200042697420004761703A2000417C
:101820006972736F6674202D20456E61626C656409
:10183000004D656368616E6963616C205265636F1A
:10184000696C202D20456E61626C6564004169728F
:10185000736F6674202D2044697361626C65640047
:101860004D656368616E6963616C205265636F6981
:101870006C202D2044697361626C656400436F6D58
:101880006D73206368616E67656420746F205553C3
:101890004200436F6D6D73206368616E67656420FD
:1018A000746F2053657269616C20310044726976EF
:1018B000696E672050726F66696C6520736574206D
:1018C000746F2023005475726E20456E67696E65D3
:1018D000204F6E004D616E75616C207472616E7385
:1018E0006D697373696F6E202D2070757420696E39
:1018F000206E65757472616C206765617220626527
:10190000666F7265207374617274696E6720656EAC
:1019100067696E6521005475726E20456E67696E49
:1019200065204F666600456E67696E652041757477
:101930006F2053687574646F776E00536D6F6B65BD
:101940007220656E61626C656400536D6F6B6572C9
:101950002064697361626C65640053657420766FFE
:101960006C756D653A20005573657220536F756E06
:1019700064200000919E11241FBECFEFD1E2DEBF94
:10198000CDBF00E00CBF15E0A0E0B2E0EDE4F9E768
:1019900001E00BBF02C007900D92AA3AB107D9F738
:1019A00022E1AAEAB5E001C01D92A939B207E1F728
:1019B0001CE0CBEBDCE000E006C021970109802FA2
:1019C000FE010E9477A9CA3BD10780E00807A9F76A
:1019D0000E948B8E0C9437AF0C9400002F923F9294
:1019E0004F925F926F927F928F929F92AF92BF922F
:1019F000CF92DF92EF92FF920F931F93CF93DF93DB
:101A0000CDB7DEB7A9970FB6F894DEBF0FBECDBF36
:101A100085EC91E00E94C2AE6A327F448105910557
:101A200019F00E94517C08C049EC51E060E070E080
:101A300084E39EE00E94AAAE40E052EC61E070E0D8
:101A400089E898E00E94926C4091DA0F5091DB0F88
:101A50006091DC0F7091DD0F8CEE97E00E94926C2C
:101A60004091DE0F5091DF0F6091E00F7091E10F18
:101A70008FE497E00E94926C4091E20F5091E30F47
:101A80006091E40F7091E50F82EB96E00E94926CFA
:101A900083EC9CE09093AD058093AC0584E89AE0DC
:101AA0009093AB058093AA0589E898E09093EC0C9D
:101AB0008093EB0C1092ED0C1092C80C1092C50C98
:101AC0001092C70C1092C60C11E010938C0D0E945E
:101AD000CE8B8091F80F8093560610925506109287
:101AE000800082E0809381008FE286BB10926F00BD
:101AF00010928500109284009BE29093A0009AE0DF
:101B00009093A10089BB109272001092A5001092D0
:101B1000A4001092A9001092A8001092AB0010929D
:101B2000AA001092AD001092AC0099EA90932001A7
:101B3000109321018ABB109273001092250110921C
:101B40002401109229011092280110922B01109269
:101B50002A0110922D0110922C018091D10E9091AA
:101B6000D20E8093E6059093E705813071F461E031
:101B70008FE30E94E14F8091E705882319F00E94CE
:101B800040580FC00E9429580CC08091E705882357
:101B900011F062E001C060E08FE30E94E14F0E941B
:101BA000CE5A8091D30E9091D40E8093ED059093F0
:101BB000EE05813071F461E08EE30E94E14F809187
:101BC000EE05882319F00E9411580FC00E94FA57A1
:101BD0000CC08091EE05882311F062E001C060E046
:101BE0008EE30E94E14F0E949B5A60E085E40E94D0
:101BF000E14F62E08CE30E94E14F62E08BE30E94E0
:101C0000E14F62E080E40E94E14F62E081E40E94E3
:101C1000E14F62E082E40E94E14F62E081E20E94D3
:101C2000E14F62E084E40E94E14F61E089E30E94B9
:101C3000E14F61E08AE30E94E14F0E943D360E943D
:101C4000775961E085E30E94E14F61E085E00E9401
:101C5000E14F61E070E085E00E941D5061E084E0AA
:101C60000E94E14F61E087E00E94E14F61E089E27C
:101C70000E94B24F61E089E20E94E14F6A9A60E0FF
:101C800085E30E94B24F60E085E00E94B24F60E0C1
:101C900084E00E94B24F60E087E00E94B24F7298E9
:101CA00061E088E00E94E14F80E090E09C012C5CC4
:101CB000314FF901ED55FF4F40814F3629F43297EE
:101CC00020813181232B31F403968837910571F7F8
:101CD00060E001C061E088E00E94B24F61E08BE209
:101CE0000E94E14F60E08BE20E94B24F0E94775960
:101CF0000E941A788091740A813009F06CC080913A
:101D0000770A9091780AA091790AB0917A0A409165
:101D10007B0A50917C0A60917D0A70917E0A841B37
:101D2000950BA60BB70B84379E40A105B10500F3B8
:101D30000E94517C80915306909154060E94984DC8
:101D400080915306909154060E94984D0E947F60A6
:101D500065EE72E080915306909154060E943A4CD1
:101D600001E010E00E9441360E9477596EEE72E069
:101D700080E090E00E94285162EE72E0809153066C
:101D8000909154060E943A4C0E943D360E9473592D
:101D90000530110531F064EF71E080E090E00E94C1
:101DA00028510F5F1F4F06301105E1F68091530651
:101DB000909154060E94984D0E947F608091530636
:101DC000909154060E94984D80915306909154062C
:101DD0000E94984D02C081118BCF80916F0082606C
:101DE00080936F0080918400909185008056904F81
:101DF000909389008093880081E08093620D8093A6
:101E0000650D8093680D80936B0D8093770D8093A3
:101E10007A0D9091890F9150943040F08093890F02
:101E200061E070E085E591E00E94AB779091890FC9
:101E30002DEF290F80914D0F223008F0AEC18A306E
:101E400079F03CF4883009F45DC0893009F45DC153
:101E500053C18B3009F49EC08C3009F4E0C04CC1F2
:101E600083E290E00E9491AAFC0188E090E09383D5
:101E700082838824839499249A9495828482AA24C4
:101E8000AA94B12CB782A68211861086108E53E8D0
:101E9000752E718E6FE4C62E67E0D62ED38EC28E5D
:101EA00079E6E72E72E0F72EF182E0820EED1FE078
:101EB00011A300A312A2F0934506E0934406CF01BC
:101EC0000E94E55183E290E00E9491AAFC0189E022
:101ED00090E09383828395828482B782A682118662
:101EE0001086108E718ED38EC28EF182E08211A385
:101EF00000A312A2F0934306E0934206CF010E9492
:101F0000E551D0C280E290E00E9491AAFC0188E0F5
:101F100090E0938382838824839499249A94958271
:101F20008482AA24AA94B12CB782A6821186108634
:101F3000108E9AE0D92ED18E2FE4E22E27E0F22ED9
:101F4000F38EE28E01E512E011830083F0934506E3
:101F5000E0934406CF010E94E46780E290E00E9493
:101F600091AAFC0189E090E0938382839582848228
:101F7000B782A68211861086108ED18EF38EE28EE5
:101F800011830083F0934306E0934206CF010E9441
:101F9000E46788C289E190E00E9491AAFC0188E090
:101FA00090E093838283CC24C394DD24DA94D58299
:101FB000C482EE24EA94F12CF782E6821186108620
:101FC000108E05E412E011830083F0934506E09340
:101FD0004406CF010E942A671092770D8091890FE5
:101FE000843009F05FC289E190E00E9491AAFC016F
:101FF00089E090E093838283D582C482F782E6826F
:1020000011861086108E11830083F0934306E093AF
:102010004206CF010E942A6710927A0D43C289E1DD
:1020200090E00E9491AA8C0175E8872E75E0972EAA
:10203000DC0111969C928E9287E090E013969C931F
:102040008E931297AA24A394BB24BA941596BC929B
:10205000AE921497CC24CA94D12C1796DC92CE92CF
:10206000169719961C921E92189758961C92C801A2
:102070000E945982A5EEEA2EA3E0FA2EF801F18221
:10208000E0821093450600934406C8010E94C26591
:102090001092620D8091890F843009F003C289E1AA
:1020A00090E00E9491AA8C01DC0111969C928E9284
:1020B00086E090E013969C938E9312971596BC92AF
:1020C000AE9214971796DC92CE92169719961C92A0
:1020D0001E92189758961C92C8010E945982F801C6
:1020E000F182E0821093430600934206C8010E94E9
:1020F000C2651092650DD6C189E080934D0F69E0ED
:1021000070E089E191E00E94AB7780E290E00E946C
:1021100091AAFC0188E090E09383828388248394D1
:1021200099249A9495828482AA24AA94B12CB78285
:10213000A68211861086108E50E8D52ED18E6FE4BF
:10214000E62E67E0F62EF38EE28E0DE512E01183A7
:102150000083F0934506E0934406CF010E9491511D
:1021600080E290E00E9491AAFC0189E090E09383D4
:10217000828395828482B782A68211861086108E11
:10218000D18EF38EE28E11830083F0934306E093A9
:102190004206CF010E94915185C18A3079F03CF40A
:1021A000883009F455C0893009F425C11BC18B3032
:1021B00009F471C08C3009F4A8C014C183E290E026
:1021C0000E9491AAFC017090950F88E090E09383A3
:1021D00082838824839499249A9495828482AA2461
:1021E000AA94B12CB782A68211861086108E83E83D
:1021F000682E618E9FE4C92E97E0D92ED38EC28EB1
:1022000029E6E22E22E0F22EF182E0820EED1FE0BE
:1022100011A300A372A2F0934706E093460683E25F
:1022200090E00E9491AAFC0189E090E09383828370
:1022300095828482B782A68211861086108E618E66
:10224000D38EC28EF182E08211A300A372A210C1CC
:1022500080E290E00E9491AAFC0188E090E09383E4
:1022600082838824839499249A9495828482AA24D0
:10227000AA94B12CB782A68211861086108EAAE08D
:10228000DA2ED18EBFE4EB2EB7E0FB2EF38EE28E7A
:1022900001E512E0D2C089E190E00E9491AAFC0120
:1022A00088E090E093838283CC24C394DD24DA9485
:1022B000D582C482EE24EA94F12CF782E68211865C
:1022C0001086108E05E412E011830083F093470618
:1022D000E093460689E190E00E9491AAFC0189E022
:1022E00090E093838283D582C482F782E68211864E
:1022F0001086108E11830083F0934906E093480600
:102300001092770D10927A0DB7C0923049F481E0A7
:102310008093890F61E070E085E591E00E94AB77E2
:1023200089E190E00E9491AA8C0185E8882E85E0E1
:10233000982ED80111969C928E9287E090E0139689
:102340009C938E931297AA24A394BB24BA941596B7
:10235000BC92AE921497CC24CA94D12C1796DC92DE
:10236000CE92169719961C921E92189758961C9208
:10237000C8010E94598235EEE32E33E0F32EF801B6
:10238000F182E082109347060093460689E190E0CF
:102390000E9491AA8C01DC0111969C928E9286E09B
:1023A00090E013969C938E9312971596BC92AE92E2
:1023B00014971796DC92CE92169719961C921E923D
:1023C000189758961C92C8010E945982F801F18210
:1023D000E08210934906009348061092620D109215
:1023E000650D4AC089E080934D0F69E070E089E196
:1023F00091E00E94AB7780E290E00E9491AAFC01FC
:1024000088E090E0938382838824839499249A942B
:1024100095828482AA24AA94B12CB782A6821186BE
:102420001086108EA0E8DA2ED18EBFE4EB2EB7E036
:10243000FB2EF38EE28E0DE512E011830083F09304
:102440004706E093460680E290E00E9491AAFC01D4
:1024500089E090E09383828395828482B782A6820A
:1024600011861086108ED18EF38EE28E118300833A
:10247000F0934906E09348068091480690914906FA
:10248000DC01ED91FC910280F381E02D19958091A2
:10249000460690914706DC01ED91FC910280F381A4
:1024A000E02D19958091890F8250823050F589E195
:1024B00090E00E9491AA8C0185E895E0F801918353
:1024C000808386E090E09383828381E09FEF958311
:1024D00084838FEF90E09783868311861086108E19
:1024E000C8010E94598285EE93E0D8018D939C9398
:1024F0001093400600933F06C8010E94C2651092E7
:10250000650DE0914E0F8E2FEE0F990BAA0BBB0BB2
:10251000FC013897E830F10508F0B9C08827EE587B
:10252000FF4F8F4F0C9477A983E290E00E9491AA0D
:10253000FC0188E090E09383828381E09FEF9583A4
:1025400084838FEF90E09783868311861086108EA8
:1025500084E8818F8FE497E0938F828F89E692E001
:10256000918380838EED9FE091A380A312A21EC071
:1025700080E290E00E9491AAFC0188E090E09383C1
:10258000828381E09FEF958384838FEF90E0978330
:10259000868311861086108E87E8818F8FE497E0FE
:1025A000938F828F8DE592E091838083F0934E0626
:1025B000E0934D069CC080E290E00E9491AAFC014D
:1025C00088E090E09383828381E09FEF958384830A
:1025D0008FEF90E09783868311861086108E8DE0B2
:1025E000818F8FE497E0938F828F81E592E0DCCF3B
:1025F00089E190E00E9491AAFC0188E090E0938339
:10260000828381E09FEF958384838FEF90E09783AF
:10261000868311861086108E85E492E091838083F4
:10262000F0934E06E0934D061092770D60C08CE15A
:1026300090E00E9491AA8C0185E895E0F8019183D1
:10264000808385E090E09383828381E09FEF958390
:1026500084838FEF90E09783868311861086108E97
:10266000C8010E94598289E795E038C089E190E06D
:102670000E9491AAFC011382128215821482178291
:10268000168211861086108E81E292E08DCF8CE04A
:1026900080934E0F6CE070E08AE191E00E94AB778E
:1026A00089E190E00E9491AA8C0185E895E0F8010B
:1026B0009183808385E090E09383828381E09FEF24
:1026C000958384838FEF90E09783868311861086AD
:1026D000108EC8010E94598285EE93E0D8018D9337
:1026E0009C9310934E0600934D061092680D8091B6
:1026F0004D0690914E06DC01ED91FC910280F38134
:10270000E02D19958091560F843658F4853608F0DF
:1027100084E664E6681B80914D0690914E060E9407
:10272000825280914E0F8C508230A8F46091570FE6
:102730007091580F85E00E9429416091590F709166
:102740005A0F85E00E940E4180915B0FE0914D068B
:10275000F0914E06808FE0914F0F8E2FEE0F990B68
:10276000AA0BBB0BFC013897E830F10508F0E5C077
:102770008827E658FF4F8F4F0C9477A983E290E0AB
:102780000E9491AAFC0189E090E09383828381E01A
:102790009FEF958384838FEF90E0978386831186E4
:1027A0001086108E84E8818F8FE497E0938F828F5C
:1027B00089E692E0918380838EED9FE091A380A3D0
:1027C00012A21EC080E290E00E9491AAFC0189E062
:1027D00090E09383828381E09FEF958384838FEFE2
:1027E00090E09783868311861086108E87E8818F0C
:1027F0008FE497E0938F828F8DE592E091838083C1
:10280000F0935206E0935106C8C080E290E00E9427
:1028100091AAFC0189E090E09383828381E09FEF9D
:10282000958384838FEF90E097838683118610864B
:10283000108E8DE0818F8FE497E0938F828F81E5FA
:1028400092E0DCCF89E190E00E9491AAFC0189E04E
:1028500090E09383828381E09FEF958384838FEF61
:1028600090E09783868311861086108E85E492E02F
:1028700091838083F0935206E093510610927A0D73
:102880008CC08CE190E00E9491AA8C0195E8692EA1
:1028900095E0792EF8017182608224E0822E912CDD
:1028A00093828282AA24A394BB24BA94B582A48280
:1028B000CC24CA94D12CD782C68211861086108E61
:1028C000C8010E94598259E7E52E55E0F52ED8013E
:1028D000ED92FC9210935206009351068CE190E029
:1028E0000E9491AA8C01FC01718260829382828293
:1028F000B582A482D782C68211861086108E0E946D
:102900005982D801ED92FC921093D60C0093D50C0D
:10291000C8010E9484663FC089E190E00E9491AAAC
:10292000FC0113821282158214821782168211868C
:102930001086108E81E292E061CF8CE080934F0F81
:102940006CE070E08BE191E00E94AB7789E190E070
:102950000E9491AA8C0185E895E0F801918380831B
:1029600084E090E09383828381E09FEF958384836A
:102970008FEF90E09783868311861086108EC801B2
:102980000E94598285EE93E0D8018D939C93109319
:1029900052060093510610926B0D80915106909152
:1029A0005206DC01ED91FC910280F381E02D199536
:1029B0008091550F843658F4853608F084E664E635
:1029C000681B80915106909152060E94825280911C
:1029D0004F0F8C50823000F56091500F7091510F65
:1029E00084E00E9429416091520F7091530F84E05E
:1029F0000E940E418091540FE0915106F0915206D1
:102A0000808F80914F0F8D3039F48091540FE09179
:102A1000D50CF091D60C808F8EE190E00E9491AAA7
:102A20008C01D090600FA090640FB090650F8090E3
:102A3000620F9090630F85E895E0F80191838083A1
:102A400083E090E09383828381E09FEF958384838A
:102A5000EE24EA94F12CF782E68211861086108E1D
:102A6000C8010E94598289E392E0D80111969C9393
:102A70008E935A969C928E9259975C96BC92AE9287
:102A80005B975D96DC921093820D0093810D6091AF
:102A9000660F7091670F83E00E9429416091680F73
:102AA0007091690F83E00E940E418091600FE09168
:102AB000810DF091820D808F8091600F0E9476775A
:102AC0008091810D9091820DDC01ED91FC9102804D
:102AD000F381E02D199580916A0F8823D1F083E26C
:102AE00090E00E9491AAFC0180916D0F90916E0F71
:102AF00020916B0F30916C0F40916F0F5091700FC0
:102B000068E070E073836283158214825783468382
:102B100015C083E290E00E9491AAFC0180916D0FA4
:102B200090916E0F20916B0F30916C0F48E050E048
:102B30005383428315821482F782E68211861086BF
:102B4000108E4DE252E051834083328F218F948F5B
:102B5000838FF093DD05E093DC058091DC05909197
:102B6000DD050E9408678091770D8823F9F089E1DF
:102B700090E00E9491AAFC0188E090E09383828318
:102B8000158214828FEF93E0978386838FEF91E015
:102B900091878087108E85E492E091838083F09303
:102BA000760DE093750DCF010E942A6780917A0D12
:102BB0008823F9F089E190E00E9491AAFC0189E064
:102BC00090E093838283158214828FEF93E0978342
:102BD00086838FEF91E091878087108E85E492E065
:102BE00091838083F093790DE093780DCF010E945B
:102BF0002A6785E89AE090930E1280930D12109147
:102C0000980F2091970F8091860F9091880F3091A7
:102C1000890F3093AE059093B1058093B20530E0F3
:102C2000AFEFB0E00E9428AF24E630E040E050E093
:102C30000E94DAAE20936F12612F70E080E090E086
:102C40000E9495AD23EC34E64AEA5AE30E94F6ADC1
:102C50002AE939E949E55FE30E948CA9609369128A
:102C600070936A1280936B1290936C12109295007D
:102C700010929400109290008CE08093910084EF69
:102C800090E0909399008093980011E018BB82E047
:102C900080937100809100020E94698B809153069D
:102CA00090915406209156064091820F5091830FC7
:102CB0005093E5114093E411209385129093841270
:102CC000809383121092B3051093E61180919F0FA9
:102CD000853040F010929F0F60E070E08BE691E04D
:102CE0000E94AB7710919F0F123009F441C0F0F4AD
:102CF000112309F463C0113009F058C08BE090E053
:102D00000E9491AA2DE233E0FC01318320832FE45D
:102D100037E0328721879093500680934F061093B7
:102D20006E0D1093710D1093740D67C0133009F47C
:102D30005EC01430D9F585E090E00E9491AA8C0124
:102D400029E833E0FC0121933193CF0141E065E8AC
:102D50007AE00E94203E85E792E0D8018D939C9313
:102D60001093500600934F0681E080936E0D41C092
:102D700086E090E00E9491AA21ED32E0DC012D93E3
:102D80003C939093500680934F068FB7F8942CEDA8
:102D900035E03093201120931F11109225118FBF21
:102DA00081E080936E0D8093710D25C010929F0F6E
:102DB00060E070E08BE691E00E94AB7785E090E008
:102DC0000E9491AA8C0129E833E0FC012193319300
:102DD000CF0140E065E87AE00E94203E85E792E07E
:102DE000D8018D939C931093500600934F06109238
:102DF0006E0D1092710D1092740D80914F0690918E
:102E00005006DC01ED91FC910190F081E02D1995C7
:102E10008091620D81111FC08091650D81111BC0D1
:102E20008091680D811117C080916B0D811113C0C5
:102E300080916E0D81110FC08091710D81110BC0B9
:102E40008091740D811107C081E00E94CA8B882394
:102E500009F43DC335C3A12CB12C312C812C412C5C
:102E6000512C612C912C712C05E815E0EE24EA948C
:102E7000A3E0FA2ECC24CA94DD24D394C5018C5C43
:102E8000914FFC01ED55FF4FE081EE2309F40FC394
:102E9000DC01AF55BF4F8D919C91892B09F407C37D
:102EA0008E2F90E0FC01F797EB32F10508F0FFC29E
:102EB0008827EE57FF4F8F4F0C9477A98091620DB2
:102EC000882309F4F4C27110F2C289E190E00E94F3
:102ED00091AA9C01FC011183008387E090E0938319
:102EE000828315821482F782E682D186C086108E94
:102EF000C90128A739A70E94598228A539A5E5EE5E
:102F0000F3E0D901ED93FC933093530D2093520DD0
:102F1000C9010E94C2657AC18091650D882309F4B8
:102F2000C6C29110C4C289E190E00E9491AA9C019E
:102F3000DC0111961C930E93E6E0F0E01396FC93EF
:102F4000EE93129715961C921E9214971796FC9268
:102F5000EE9216971996DC92CE92189758961C927C
:102F600028A739A70E94598228A539A5E5EEF3E0E4
:102F7000D901ED93FC933093550D2093540DC90165
:102F80000E94C2657CC18091680D882309F48FC2BC
:102F900061108DC289E190E00E9491AA9C01DC0140
:102FA00011961C930E93E5E0F0E01396FC93EE93DC
:102FB000129715961C921E9214971796FC92EE92F9
:102FC00016971996DC92CE92189758961C9228A7BD
:102FD00039A70E94598228A539A5E5EEF3E0D90169
:102FE000ED93FC933093570D2093560DC9010E9429
:102FF000C2657EC180916B0D882309F458C25110BF
:1030000056C289E190E00E9491AA9C01DC011196D0
:103010001C930E93E4E0F0E01396FC93EE9312976A
:1030200015961C921E9214971796FC92EE92169784
:103030001996DC92CE92189758961C9228A739A719
:103040000E94598228A539A5E5EEF3E0D901ED9358
:10305000FC933093590D2093580DC9010E94C2650D
:1030600080C180916E0D882309F421C241101FC2D6
:1030700089E190E00E9491AA9C01DC0111961C93C9
:103080000E93E2E0F0E01396FC93EE931297159600
:103090001C921E9214971796FC92EE921697199610
:1030A000DC92CE92189758961C9228A739A70E94B6
:1030B000598228A539A5E5EEF3E0D901ED93FC93FB
:1030C00030935B0D20935A0DC9010E94C26582C1E5
:1030D0008091710D882309F4EAC18110E8C189E16A
:1030E00090E00E9491AA9C01DC0111961C930E9322
:1030F000E1E0F0E01396FC93EE93129715961C9284
:103100001E9214971796FC92EE9216971996DC92DF
:10311000CE92189758961C9228A739A70E945982D8
:1031200028A539A5E5EEF3E0D901ED93FC933093A2
:103130005D0D20935C0DC9010E94C26584C1809120
:10314000740D882309F4B3C13110B1C189E190E055
:103150000E9491AA1C01DC0111961C930E931396F8
:103160001C921E92129715961C921E9214971796F7
:10317000FC92EE9216971996DC92CE92189758967A
:103180001C920E94598225EE33E0F10131832083A5
:1031900030925F0D20925E0DC1010E94C26585C113
:1031A0008091620D882309F482C1711080C18CE185
:1031B00090E00E9491AA9C01DC0111961C930E9351
:1031C000E7E0F0E01396FC93EE93129715961C92AD
:1031D0001E9214971796FC92EE9216971996DC920F
:1031E000CE92189758961C9228A739A70E94598208
:1031F00028A539A5E9E7F5E0D901ED93FC933093D3
:10320000610D2093600DC9010E9484667724739438
:103210004EC18091650D882309F449C1911047C1C1
:103220008CE190E00E9491AA9C01DC0111961C9314
:103230000E93E6E0F0E01396FC93EE93129715964A
:103240001C921E9214971796FC92EE92169719965E
:10325000DC92CE92189758961C9228A739A70E9404
:10326000598228A539A5E9E7F5E0D901ED93FC934A
:103270003093640D2093630DC9010E9484669924E4
:10328000939415C18091680D882309F410C16110D1
:103290000EC18CE190E00E9491AA9C01DC01119684
:1032A0001C930E93E5E0F0E01396FC93EE931297D7
:1032B00015961C921E9214971796FC92EE921697F2
:1032C0001996DC92CE92189758961C9228A739A787
:1032D0000E94598228A539A5E9E7F5E0D901ED93C7
:1032E000FC933093670D2093660DC9010E9484669C
:1032F00066246394DCC080916B0D882309F4D7C0E9
:103300005110D5C08CE190E00E9491AA9C01DC0193
:1033100011961C930E93E4E0F0E01396FC93EE9369
:10332000129715961C921E9214971796FC92EE9285
:1033300016971996DC92CE92189758961C9228A749
:1033400039A70E94598228A539A5E9E7F5E0D901F6
:10335000ED93FC9330936A0D2093690DC9010E948F
:10336000846655245394A3C080916E0D882309F47C
:103370009EC041109CC08CE190E00E9491AA9C01EB
:10338000DC0111961C930E93E2E0F0E01396FC939F
:10339000EE93129715961C921E9214971796FC9214
:1033A000EE9216971996DC92CE92189758961C9228
:1033B00028A739A70E94598228A539A5E9E7F5E091
:1033C000D901ED93FC9330936D0D20936C0DC901E1
:1033D0000E948466442443946AC08091710D8823BE
:1033E00009F465C0811063C08CE190E00E9491AA4D
:1033F0009C01DC0111961C930E93E1E0F0E0139622
:10340000FC93EE93129715961C921E9214971796A2
:10341000FC92EE9216971996DC92CE9218975896D7
:103420001C9228A739A70E94598228A539A5E9E747
:10343000F5E0D901ED93FC933093700D20936F0D5F
:10344000C9010E9484668824839431C08091740DE0
:10345000882369F131102BC08CE190E00E9491AA81
:103460001C01DC0111961C930E9313961C921E9264
:10347000129715961C921E9214971796FC92EE9234
:1034800016971996DC92CE92189758961C920E9425
:10349000598229E735E0F101318320833092730DA1
:1034A0002092720DC1010E9484663324339433E06C
:1034B000A30EB11C88E7A816B10409F0DFCCC4CC78
:1034C00082E00E94CA8B882311F01DA216C081E001
:1034D0000E94CA8B882329F082E00E94AE8B811162
:1034E00080C68CE30E948A4F892B09F06BC68CE35F
:1034F0000E948A4F892B09F06BC686E0ECECFFE056
:10350000DE01549601900D928A95E1F78091C50FE6
:103510009090D50FA090C60FB090C70F9091C80F94
:103520007091C90F6091CA0F5091CB0F4091D20F8B
:103530002091D30F3091D40FE0914F06F0915006B7
:10354000FFA3EEA30091810D1091820D5090F30F17
:10355000E090EC0FF090ED0F7090F60F6090F50F8B
:10356000C0905E0FD0905F0F4090610F30905C0F65
:1035700020905D0FFDA1FB8B8A8F9B8EAC8EBD8E44
:103580009E8F7F8F68A359A34AA33CA32BA3F2E18C
:103590008F2EFE017396DE01119601900D928A9492
:1035A000E1F7E5E8FAE0F093BC05E093BB05ADA1D7
:1035B000A98388879986AA86BB869C877D876E8724
:1035C0005F87488B3A8B298B22E1FE013196A8EC6C
:1035D000B5E001900D922A95E1F72092190E3092F4
:1035E0001A0E4092180ED092110EC092100E5092E8
:1035F000830D6092150E7092140EF092130EE092ED
:10360000120E1093170E0093160E2EA13FA13093A9
:10361000BE052093BD05911107C01092D4058111FC
:1036200003C010925B0AA3C081E080935B0A009103
:10363000560A1091570A8091E70960E00E94E14F15
:10364000D801ED91FC910190F081E02DC801199510
:103650008091C805882359F1813071F08330C1F41D
:1036600088E293E29093CA058093C90589E080932C
:10367000CD0580E197E217C088EB9BE09093CA05E7
:103680008093C90583E08093CD0588E99AE30BC058
:1036900088E893E19093CA058093C90586E08093FA
:1036A000CD0580EE9EE29093CC058093CB05809172
:1036B000CF058823E9F18091D3056091CD0570E0B5
:1036C0008823C9F08091D5058823A9F080E090E097
:1036D0000E9495AD9B01AC0160E070E088EC92E443
:1036E0000E94F0A96093BF057093C0058093C10547
:1036F0009093C20525C080E090E00E9495AD9B01AB
:10370000AC0160E070E088EC92E40E94F0A9609364
:10371000BF057093C0058093C1059093C2051092B8
:10372000B6051092B7051092B8051092B9051FC0E2
:103730001092BF051092C0051092C1051092C205EB
:103740006091CE0570E080E090E00E9495AD9B0115
:10375000AC0160E070E088EC92E40E94F0A9609314
:10376000B6057093B7058093B8059093B90510928C
:10377000DB051092C7051092BA051092C30510928E
:10378000C4051092C5051092C6050E94C36F6E98BD
:10379000769AEE9880916A008F7C80936A0080917F
:1037A0001A0E882321F080916A00806203C0809104
:1037B0006A00806380936A00EE980E94637280E0E2
:1037C00090E040E09C012C5C314FF901ED55FF4F3A
:1037D0005081552331F0329720813181232B09F01C
:1037E0004F5F03968837910569F74093E005AFEE88
:1037F000B5E020E030E08AE5282E8FE5382E97ED01
:10380000492E9DE5592E4DEF642E4DE5742E5DEB4E
:10381000852E5DE5952E6AECA62E6DE5B62E40EE62
:103820005FE501E61FE573E6E72E7FE5F72EE3E1AE
:10383000CE2EE0E6DE2EC9018C5C914FFC01ED55E9
:10384000FF4F6081662309F4C6C28F559F4FFC016C
:1038500080819181892B09F4BEC270E0FB01319710
:10386000E637F10508F0B7C28827E355FF4F8F4FC1
:103870000C9477A982EC9CE811969C938E93ABC232
:1038800081EC9CE811969C938E93A5C280EC9CE8F9
:1038900011969C938E939FC289EB9CE811969C9302
:1038A0008E9399C281EC94E611969C938E9393C269
:1038B00083E694E611969C938E938DC284E694E6FB
:1038C00011969C938E9387C286E494E611969C93FE
:1038D0008E9381C282E394E611969C938E937BC271
:1038E00083E294E611969C938E9375C287EC93E6DF
:1038F00011969C938E936FC283E692E611969C93E9
:103900008E9369C28AEB93E611969C938E9363C261
:103910008CE793E611969C938E935DC28FEA93E6B3
:1039200011969C938E9357C288EB93E611969C93C5
:103930008E9351C281EB93E611969C938E934BC26A
:103940008FE993E611969C938E9345C28DE993E699
:1039500011969C938E933FC28BE993E611969C93AC
:103960008E9339C28BE893E611969C938E9333C263
:1039700089E893E611969C938E932DC28AE793E68D
:1039800011969C938E9327C28AE693E611969C9398
:103990008E9321C288E693E611969C938E931BC268
:1039A00086E693E611969C938E9315C280EA90E684
:1039B00011969C938E930FC28EE990E611969C937C
:1039C0008E9309C28DE990E611969C938E9303C263
:1039D00087E897E511969C938E93FDC183E593E666
:1039E00011969C938E93F7C184E393E611969C9372
:1039F0008E93F1C185E193E611969C938E93EBC172
:103A000083E193E611969C938E93E5C184EE92E652
:103A100011969C938E93DFC18DED92E611969C9347
:103A20008E93D9C18CEA92E611969C938E93D3C162
:103A300089EC9CE811969C938E93CDC181E692E629
:103A400011969C938E93C7C18FE592E611969C9335
:103A50008E93C1C184E492E611969C938E93BBC170
:103A600089E292E611969C938E93B5C18EE092E620
:103A700011969C938E93AFC183EF91E611969C9320
:103A80008E93A9C188ED91E611969C938E93A3C164
:103A90008DEB91E611969C938E939DC182EA91E6FF
:103AA00011969C938E9397C187E891E611969C930B
:103AB0008E9391C18CE691E611969C938E938BC167
:103AC00081E591E611969C938E9385C186E391E6FC
:103AD00011969C938E937FC18BE191E611969C93F6
:103AE0008E9379C180E091E611969C938E9373C179
:103AF00085EE90E611969C938E936DC18AEC90E6CC
:103B000011969C938E9367C18FEA90E611969C93D1
:103B10008E9361C18FEA9FE511969C938E935BC152
:103B200084E99FE511969C938E9355C18EE99DE59E
:103B300011969C938E934FC18DE99DE511969C93B0
:103B40008E9349C18CE99DE511969C938E9343C158
:103B500081E89FE511969C938E933DC18EE89DE58B
:103B600011969C938E9337C18DE89DE511969C9399
:103B70008E9331C18CE89DE511969C938E932BC159
:103B80008EE69FE511969C938E9325C182EC9EE56F
:103B900011969C938E931FC187E79EE511969C9387
:103BA0008E9319C185EB98E511969C938E9313C162
:103BB00081EA98E511969C938E930DC18DE898E566
:103BC00011969C938E9307C181E99CE811969C9372
:103BD0008E9301C18AE79DE511969C938E93FBC05D
:103BE00088E69DE511969C938E93F5C081EB9CE54C
:103BF00011969C938E93EFC08FE99CE511969C9350
:103C00008E93E9C08BE69EE511969C938E93E3C05C
:103C10008FE59EE511969C938E93DDC083E59EE52E
:103C200011969C938E93D7C087E49EE511969C9342
:103C30008E93D1C08BE39EE511969C938E93CBC05F
:103C40008FE29EE511969C938E93C5C083E29EE51C
:103C500011969C938E93BFC08FE29DE511969C9325
:103C60008E93B9C08DE19DE511969C938E93B3C060
:103C70008BE09DE511969C938E93ADC089EF9CE5FA
:103C800011969C938E93A7C087EE9CE511969C930A
:103C90008E93A1C085ED9CE511969C938E939BC05D
:103CA00083EC9CE511969C938E9395C08CE69FE5E2
:103CB00011969C938E938FC08AE69FE511969C93F4
:103CC0008E9389C085E69FE511969C938E9383C061
:103CD0001196DC92CE927FC01196FC92EE927BC040
:103CE00011961C930E9377C08CE59FE511969C93DB
:103CF0008E9371C011965C934E936DC01196BC92D9
:103D0000AE9269C011969C928E9265C011967C927B
:103D10006E9261C011965C924E925DC011963C927B
:103D20002E9259C0EBE6F8E51196FC93EE9353C042
:103D300088E598E511969C938E934DC0E3E8F8E5ED
:103D40001196FC93EE9347C087E59FE511969C93EF
:103D50008E9341C0E4E5FFE51196FC93EE933BC0E2
:103D60008BE49FE511969C938E9335C0E0E4FFE5CC
:103D70001196FC93EE932FC089E49FE511969C93D6
:103D80008E9329C0E2E4FFE51196FC93EE9323C0E5
:103D90008BE59DE511969C938E931DC0EEE4FDE5A9
:103DA0001196FC93EE9317C081E49DE511969C93C8
:103DB0008E9311C0EFE2FFE51196FC93EE930BC0DA
:103DC0008EE19FE511969C938E9305C0EDE0FFE593
:103DD0001196FC93EE932D5F3F4F129628373105D5
:103DE00009F029CD1092E1058091E605811114C0FA
:103DF00080E090E0FC01EB52F14F208131812456AC
:103E000031092436310528F003968837910591F75A
:103E100003C081E08093E1051092E8058091ED05F3
:103E2000811114C080E090E0FC01EB52F14F208141
:103E30003181285C31092436310528F00396883712
:103E4000910591F703C081E08093E80580914F06CA
:103E500090915006DC01ED91FC91EC5BFF4F2091BD
:103E6000A20F3091A30F4091A00F5091A10F01908C
:103E7000F081E02D61E0199580914F0690915006F8
:103E8000DC01ED91FC91EC5BFF4F2091A60F30918E
:103E9000A70F4091A40F5091A50F0190F081E02D44
:103EA00062E0199580914F0690915006DC01ED91EA
:103EB000FC91EC5BFF4F2091AA0F3091AB0F40912A
:103EC000A80F5091A90F0190F081E02D63E01995A2
:103ED00080914F0690915006DC01ED91FC91EC5BD6
:103EE000FF4F2091B50F3091B60F4091B30F509115
:103EF000B40F0190F081E02D64E0199580914F0698
:103F000090915006DC01ED91FC91EC5BFF4F20910C
:103F1000B90F3091BA0F4091B70F5091B80F01907F
:103F2000F081E02D65E0199580914F069091500643
:103F3000DC01ED91FC91EC5BFF4F2091BD0F3091C6
:103F4000BE0F4091BB0F5091BC0F0190F081E02D4E
:103F500066E0199580914F0690915006DC01ED9135
:103F6000FC91EA5BFF4F0190F081E02D4091AC0F96
:103F700061E0199580914F0690915006DC01ED911A
:103F8000FC91EA5BFF4F0190F081E02D4091AD0F75
:103F900062E0199580914F0690915006DC01ED91F9
:103FA000FC91EA5BFF4F0190F081E02D4091AE0F54
:103FB00063E0199580914F0690915006DC01ED91D8
:103FC000FC91EA5BFF4F0190F081E02D4091BF0F23
:103FD00064E0199580914F0690915006DC01ED91B7
:103FE000FC91EA5BFF4F0190F081E02D4091C00F02
:103FF00065E0199580914F0690915006DC01ED9196
:10400000FC91EA5BFF4F0190F081E02D4091C10FE0
:1040100066E0199580914F0690915006DC01ED9174
:10402000FC9106A8F7A9E02D6091B00F1995809139
:104030004F0690915006DC01ED91FC9104A4F5A58A
:10404000E02D6091B10F199580914F069091500627
:10405000DC01ED91FC9102A8F3A9E02D6091B20F73
:10406000199580E090E09C012C5C314FF901ED55F1
:10407000FF4F4081423731F4329720813181232B29
:1040800009F0B5C003968837910569F70E94558DF0
:1040900080914F0690915006DC01ED91FC91EA5A17
:1040A000FF4F0190F081E02D40E06091C20F199523
:1040B00080914F0690915006DC01ED91FC91EA5AF7
:1040C000FF4F0190F081E02D41E06091C40F199500
:1040D00080914F0690915006DC01ED91FC91EA5AD7
:1040E000FF4F0190F081E02D42E06091C30F1995E0
:1040F0008091990F882331F080914F0F8D3011F00E
:104100001092990F1092B1061092440D80919A0F5F
:104110008093B00580919C0F8093AF052091EA0FAA
:1041200030E0AFEFB0E00E9428AF24E630E040E09E
:1041300050E00E94DAAE2093450D8091E90F811185
:104140000E9492590E9426360E9460516B017C01A8
:1041500010E011110FC080915606882359F02CEA07
:104160003DE540ED57E060E070E085E89AE00E94B0
:10417000234011E00E94A169882351F00E948235FA
:104180000E94BA5B0E9477590E942E690E94ED3509
:104190000E949B84029711F00E9407420E94248E85
:1041A0000E949B840297A9F60E946051DC01CB011A
:1041B0008C199D09AE09BF098C3B9240A105B10540
:1041C00040F218C082E00E94CA8B81110DC08FC9D5
:1041D00082E00E94AE8B882309F48FC9B3E0BDA3AF
:1041E0008CC991E09DA389C9A2E0ADA386C90E94B4
:1041F000498D4ECF0E949E350E94775980916F0A5B
:10420000811102C00E9428790E94708486E30E9476
:10421000E450BC01990F880B990B6115710581055C
:10422000910511F00E941CAD2AE93CE548EE53E0EF
:1042300060E070E085E89AE0A9960FB6F894DEBFDA
:104240000FBECDBFDF91CF911F910F91FF90EF90E7
:10425000DF90CF90BF90AF909F908F907F906F90A6
:104260005F904F903F902F900C9423402F923F925D
:104270004F925F926F927F928F929F92AF92BF9276
:10428000CF92DF92EF92FF920F931F93CF93DF9322
:10429000CDB7DEB7E7970FB6F894DEBF0FBECDBF40
:1042A00080915306909154060E94984D0E947F6021
:1042B00069EE74E080915306909154060E943A4C46
:1042C0006DE875E0CE0101960E94FB4B009153060C
:1042D00010915406D801ED91FC914D815E81698168
:1042E0007A810280F381E02DC8011995C8010E94EE
:1042F000984DCE0101960E94CB4B0E94248E809156
:10430000530690915406DC01ED91FC910284F385F3
:10431000E02D199580915306909154060E94984D76
:104320000E947F606EE775E080915306909154067D
:104330000E943A4CE091700AE4300CF0E0E08AE030
:1043400095E09A83898386E095E09C838B8381E066
:1043500095E09E838D838CEF94E098878F83EE0F9A
:10436000FF0B81E090E08C0F9D1FE80FF91F60812B
:10437000718180915306909154060E94AB4D0E942A
:104380007F6068E475E080915306909154060E9426
:10439000AB4D0E947F606CE375E080915306909175
:1043A00054060E943A4CE091FE10F091FF1081817A
:1043B0009281883E934014F40E946F60E091FE1059
:1043C000F091FF10618172818091530690915406A3
:1043D0000E94A37884E00E940C80E091FE10F0918E
:1043E000FF106581768180915306909154060E945A
:1043F000A37885E00E940C80E091FE10F091FF1000
:104400006381748180915306909154060E94A37831
:1044100084E00E940C80E091FE10F091FF10678113
:1044200080915306909154060E94897888E00E94FA
:104430000C80E091FE10F091FF1080850E945B607F
:1044400060E375E080915306909154060E943A4CC7
:10445000E0910811F091091181819281883E934089
:1044600014F40E946F60E0910811F09109116181CC
:10447000728180915306909154060E94A37884E043
:104480000E940C80E0910811F091091165817681FC
:1044900080915306909154060E94A37885E00E9473
:1044A0000C80E0910811F091091163817481809171
:1044B0005306909154060E94A37884E00E940C80D9
:1044C000E0910811F0910911678180915306909154
:1044D00054060E94897888E00E940C80E0910811BF
:1044E000F091091180850E945B6064E275E0809123
:1044F0005306909154060E943A4CE0911211F091AB
:10450000131181819281883E934014F40E946F6060
:10451000E0911211F0911311618172818091530623
:10452000909154060E94A37884E00E940C80E09150
:104530001211F0911311658176818091530690914B
:1045400054060E94A37885E00E940C80E09112112D
:10455000F0911311638174818091530690915406F8
:104560000E94A37884E00E940C80E0911211F091E7
:104570001311678180915306909154060E948978A7
:1045800088E00E940C80E0911211F0911311808557
:104590000E945B6068E175E080915306909154063B
:1045A0000E943A4CE0911C11F0911D118181928181
:1045B000883E934014F40E946F60E0911C11F091CA
:1045C0001D116181728180915306909154060E9461
:1045D000A37884E00E940C80E0911C11F0911D11E1
:1045E0006581768180915306909154060E94A3784C
:1045F00085E00E940C80E0911C11F0911D116381F7
:10460000748180915306909154060E94A37884E0AF
:104610000E940C80E0911C11F0911D116781809126
:104620005306909154060E94897888E00E940C807D
:10463000E0911C11F0911D1180850E945B608091BA
:104640005306909154060E94984D0E947084C82E83
:1046500060EB75E080915306909154060E94AB4D3B
:104660000E947F600DE910E1E12CF12CD12C570163
:104670002FEFA21AB20AB501809153069091540609
:104680000E94A37849E0E416F10410F48BE001C025
:104690008AE00E940C80D8012C9180915306909161
:1046A00054062223C9F11596ED91FC91169761816C
:1046B00072810E94A378D8011596ED91FC9116970E
:1046C00081819281883E934014F40E946F6084E05F
:1046D0000E940C80D8011596ED91FC91169763818C
:1046E000748180915306909154060E94A37884E0CF
:1046F0000E940C80D8011596ED91FC9116972781A8
:104700008091530690915406222319F068EA75E0CF
:104710000BC061EA75E008C0EC14FD041CF469E903
:1047200075E002C06CE875E00E94AB4D095F1F4F59
:104730007501BCE0AB16B10409F099CF0E947F600F
:1047400065EE75E080915306909154060E943A4CB4
:104750000E947084682F80915306909154060E94A5
:104760005F7761ED75E080915306909154060E9449
:104770003A4C60916D0A70916E0A80915306909147
:1047800054060E94D9780E94248E809153069091FD
:104790005406DC01ED91FC910284F385E02D19951E
:1047A00080915306909154060E94984D0E947F601C
:1047B00065E876E080915306909154060E94AB4DD7
:1047C0000E947F6061E776E08091530690915406E5
:1047D0000E943A4C80914D0F0E94AE52BC018091D4
:1047E0005306909154060E94AB4D6DE576E08091A2
:1047F0005306909154060E943A4C80914E0F0E94AD
:10480000AE52BC0180915306909154060E943A4CDE
:1048100020914E0F80915306909154062B303CF41A
:10482000293054F4283069F46CE476E007C02B306A
:1048300041F468E576E002C062E576E00E94AB4DA7
:1048400002C00E94984D68E376E0809153069091F3
:1048500054060E943A4C80914F0F0E94AE52BC0108
:1048600080915306909154060E943A4C20914F0F2C
:1048700080915306909154062B303CF4293054F427
:10488000283069F467E276E007C02B3041F463E337
:1048900076E002C06DE276E00E94AB4D02C00E945D
:1048A000984D63E176E080915306909154060E9402
:1048B0003A4C20915C0F809153069091540622232C
:1048C00019F06BE076E002C069EF75E00E943A4CA7
:1048D00080915306909154060E94984D0E94248E18
:1048E0008091530690915406DC01ED91FC91028475
:1048F000F385E02D199580910002823011F40C941B
:10490000F82CF090730F0091760F11E08091530610
:10491000909154060E94984D0E947F606CE279E06D
:1049200080915306909154060E94AB4D0E947F6087
:1049300063E179E080915306909154060E943A4CCD
:10494000E091890FE5300CF0E0E085EB96E09A838A
:10495000898380EB96E09C838B8386EA96E09E8336
:104960008D8382EA96E098878F8381E996E09A8723
:104970008987EE0FFF0B81E090E08C0F9D1FE80F01
:10498000F91F6081718180915306909154060E94B5
:10499000AB4D6AEF78E080915306909154060E94E7
:1049A0003A4C6091000280915306909154060E9407
:1049B0005F7761EE78E080915306909154060E94F3
:1049C0003A4C8F2D0E944660FF2009F44AC067EDE3
:1049D00078E080915306909154060E943A4C809161
:1049E000530690915406112339F06091740F0E9480
:1049F00089789091740F06C060917A0F0E9489782F
:104A000090917A0F809166129813F9C76BEB78E05A
:104A100080915306909154060E943A4C809153061F
:104A200090915406112339F06091750F61110CC0FB
:104A300066EB78E006C060917B0F611105C061EB09
:104A400078E00E943A4C05C0062E000C770B0E94BD
:104A5000A3786FEA78E080915306909154060E9403
:104A60003A4C80915306909154060E94984D66E905
:104A700078E080915306909154060E943A4C802F22
:104A80000E944660002309F44AC06CE878E08091F7
:104A90005306909154060E943A4C8091530690918F
:104AA0005406112339F06091770F0E948978909114
:104AB000770F06C060917D0F0E94897890917D0FDD
:104AC000809168129813B5C760E778E0809153062B
:104AD000909154060E943A4C80915306909154064E
:104AE000112339F06091780F61110CC06BE678E00A
:104AF00006C060917E0F611105C066E678E00E94F5
:104B00003A4C05C0062E000C770B0E94A37864E691
:104B100078E080915306909154060E943A4C80911F
:104B20005306909154060E94984D6BE478E0809172
:104B30005306909154060E943A4C8091920F811135
:104B400003C00E94546035C06DEB76E0809153063F
:104B5000909154060E943A4C68E478E080915306A4
:104B6000909154060E943A4C6091920F80915306A6
:104B7000909154060E94897868E378E0809153060A
:104B8000909154060E943A4C4091930F5091940F8B
:104B900060E070E02AE080915306909154060E94F4
:104BA000734C63E378E080915306909154060E9421
:104BB000AB4D6AE178E080915306909154060E94D3
:104BC0003A4C80918A0F8436C8F463E178E0809192
:104BD0005306909154060E943A4C60918A0F80913E
:104BE0005306909154060E94897861E178E08091A3
:104BF0005306909154060E94AB4D03C080E00E9482
:104C0000546068EF77E080915306909154060E94BB
:104C10003A4C80918B0F8436C8F461EF77E0809135
:104C20005306909154060E943A4C60918B0F8091EC
:104C30005306909154060E9489786FEE77E0809138
:104C40005306909154060E94AB4D03C080E00E9431
:104C5000546066ED77E080915306909154060E946F
:104C60003A4C20914C068091530690915406222391
:104C700019F06FEC77E002C065EC77E00E94AB4D75
:104C80006CEA77E080915306909154060E943A4C6A
:104C90006091800F7091810F072E000C880B990B8B
:104CA0000E9497AD20E030E04AE754E40E94F0A96A
:104CB000AB01BC0121E080915306909154060E9403
:104CC000BB4C67EA77E080915306909154060E94AE
:104CD000AB4D6EE877E080915306909154060E94A8
:104CE0003A4C6091820F7091830F072E000C880B55
:104CF000990B0E9497AD20E030E04AE754E40E940F
:104D0000F0A9AB01BC0121E08091530690915406BB
:104D10000E94BB4C69E877E080915306909154065D
:104D20000E94AB4D60E777E0809153069091540666
:104D30000E943A4C6091840F7091850F072E000CF1
:104D4000880B990B0E9497AD20E030E04AE754E4CD
:104D50000E94F0A9AB01BC0121E080915306909123
:104D600054060E94BB4C6BE677E08091530690910D
:104D700054060E94AB4D62E577E080915306909116
:104D800054060E943A4C8091890F813011F0843092
:104D9000D9F48091860F0E9446608091860F882307
:104DA000D9F06EE477E080915306909154060E940A
:104DB0003A4C6091870F80915306909154060E945F
:104DC00089786CE477E002C067E377E0809153066E
:104DD000909154060E943A4C80915306909154064B
:104DE0000E94984D6EE177E08091530690915406B1
:104DF0000E943A4C9091890F2FEF290F8091530612
:104E000090915406223028F46091B1050E945F779A
:104E100004C069E077E00E94AB4D60EF76E08091DE
:104E20005306909154060E943A4C8091960F0E942E
:104E300046608091960F882341F16EED76E0809177
:104E40005306909154060E943A4C6091970F8091BE
:104E50005306909154060E94897866EC76E0809122
:104E60005306909154060E943A4C6091980F80919D
:104E70005306909154060E94897864EC76E0809104
:104E80005306909154060E943A4C8091530690919B
:104E900054060E94984D0E94248E80915306909152
:104EA0005406DC01ED91FC910284F385E02D199507
:104EB00080915306909154060E94984D0E947F6005
:104EC00065EB79E080915306909154060E94AB4DBA
:104ED0000E947F6064E979E08091530690915406C6
:104EE0000E943A4C8091560F8436C8F46DE879E000
:104EF00080915306909154060E943A4C6091560F4F
:104F000080915306909154060E9489786BE879E06D
:104F100080915306909154060E94AB4D03C080E0EF
:104F20000E9454606AE679E080915306909154069D
:104F30000E943A4C8091550F8436C8F463E679E0BC
:104F400080915306909154060E943A4C6091550FFF
:104F500080915306909154060E94897861E679E029
:104F600080915306909154060E94AB4D03C080E09F
:104F70000E94546060E479E0809153069091540659
:104F80000E943A4C60915E0F70915F0F16161706E3
:104F900014F50091530610915406072E000C880B4F
:104FA000990B0E9497AD20E030E04AE754E40E945C
:104FB000F0A9AB01BC0122E0C8010E94BB4CC801B2
:104FC0000E94984D6BE379E08091530690915406CE
:104FD0000E94AB4D03C080E00E9454600E94248E6A
:104FE0008091530690915406DC01ED91FC9102846E
:104FF000F385E02D199580915306909154060E94F7
:10500000984D0E947F6065E27BE08091530690910D
:1050100054060E94AB4D0E947F602091CF05809185
:10502000530690915406222309F4BFC166EF7AE03B
:105030000E943A4C0E94C36C0E9454600E94C36C50
:105040002091530630915406882389F063EE7AE06C
:10505000C9010E943A4C8091D2050E94187BBC0184
:1050600080915306909154060E94AB4D4FC060ED65
:105070007AE0C9010E943A4C8091CF050E94187BCA
:10508000BC0180915306909154060E943A4C809145
:10509000D0058823A9F168EC7AE0809153069091BD
:1050A00054060E943A4CE091D005E4300CF0E0E068
:1050B0008BEF92E09A83898389EF92E09C838B83C4
:1050C00087EF92E09E838D8385EF92E098878F83B0
:1050D000EE0FFF0B81E090E08C0F9D1FE80FF91F92
:1050E0006081718180915306909154060E943A4CE0
:1050F00066EC7AE080915306909154060E943A4CF7
:1051000080915306909154060E94984D63EB7AE08B
:1051100080915306909154060E943A4C8091D1059B
:105120000091530610915406882321F00E94187BA9
:10513000BC0102C06FEA7AE0C8010E94AB4D6CE985
:105140007AE080915306909154060E943A4C8091E7
:10515000D2050091530610915406882321F00E9435
:10516000187BBC0102C068E97AE0C8010E94AB4D1F
:1051700065E87AE080915306909154060E943A4C7B
:105180008091D4058823E1F06FE77AE0809153069F
:10519000909154060E943A4C8091D3050E94187B4E
:1051A000BC0180915306909154060E943A4C65E9E7
:1051B00075E080915306909154060E949B4D03C068
:1051C00080E00E9454606CE67AE0809153069091F2
:1051D00054060E943A4C8091D5058823E1F066E69A
:1051E0007AE080915306909154060E943A4C809147
:1051F000D3050E94187BBC01809153069091540600
:105200000E943A4C65E975E08091530690915406EE
:105210000E949B4D03C080E00E94546063E57AE0E9
:1052200080915306909154060E943A4CE091D60525
:10523000E2300CF0E2E08BEF99E09A8389838FEE05
:1052400099E09C838B8387EE99E09E838D83EE0F9C
:10525000FF0BA1E0B0E0AC0FBD1FEA0FFB1F6081A8
:10526000718180915306909154060E94AB4D60E489
:105270007AE080915306909154060E943A4CE09156
:10528000C805E4300CF0E4E080EE99E09A8389836D
:105290008AED99E09C838B8383ED99E09E838D83D7
:1052A0008DEC99E098878F8385EC99E09A878987C0
:1052B000EE0FFF0B81E090E08C0F9D1FE80FF91FB0
:1052C0006081718180915306909154060E94AB4D8C
:1052D0006EE37AE080915306909154060E943A4C16
:1052E0006091CD0580915306909154060E94897873
:1052F0006FE27AE080915306909154060E943A4CF6
:105300008091C805811110C06091CE05809153062F
:10531000909154060E94897864E27AE08091530665
:10532000909154060E943A4C6091C9057091CA054B
:10533000072E000C880B990B0E9497AD20E030E0FF
:105340004AE754E40E94F0A9AB01BC0121E080913E
:105350005306909154060E94BB4C66E17AE080911E
:105360005306909154060E943A4C6091CB0570917F
:10537000CC05072E000C880B990B0E9497AD20E0FE
:1053800030E04AE754E40E94F0A9AB01BC0121E0FF
:1053900080915306909154060E94BB4C67E07AE0DE
:1053A000809153069091540602C069E07BE00E9410
:1053B000AB4D0E94248E8091530690915406DC01DF
:1053C000ED91FC910284F385E02D199580915306AF
:1053D000909154060E94984D0E947F6063EA7BE0A2
:1053E00080915306909154060E94AB4D0E947F60BD
:1053F00066E97BE080915306909154060E943A4CF6
:10540000E0919F0FE5300CF0E5E084E89BE09A83A3
:1054100089838DE69BE09C838B838BE59BE09E8359
:105420008D838CE49BE098878F8389E39BE09A8748
:10543000898781E39BE09C878B87EE0FFF0B81E0E0
:1054400090E08C0F9D1FE80FF91F608171818091A2
:105450005306909154060E94AB4D0E94248E809179
:10546000530690915406DC01ED91FC910284F38582
:10547000E02D199580915306909154060E94984D05
:105480000E947F6063E27CE0809153069091540615
:105490000E94AB4D0E947F602091B106809153061F
:1054A000909154062223C9F16CEE7BE00E943A4CA5
:1054B00080915306909154060E94984D6DEC7BE0CC
:1054C00080915306909154060E943A4C8091990F16
:1054D0000E9446608091990F81110E948E80809178
:1054E0005306909154060E94984D6EEA7BE080919D
:1054F0005306909154060E943A4C80919B0F0E9453
:10550000466080919B0F81110E94628080915306BA
:10551000909154060E94984D04C06EE07CE00E9479
:10552000AB4D0E94248E8091530690915406DC016D
:10553000ED91FC910284F385E02D199585EE9EE5B1
:10554000A1E0BB278BAB9CABADABBEAB8091530650
:10555000909154060E94984D0E947F606DE77DE017
:1055600080915306909154060E94AB4D0E947F603B
:1055700064E67DE080915306909154060E943A4C77
:1055800020916B0A8091530690915406222319F0C2
:1055900060E67DE002C06BE57DE00E94AB4D80914E
:1055A0006B0A882349F162E47DE080915306909173
:1055B00054060E943A4C60919D0F70919E0F072EE9
:1055C000000C880B990B0E9497AD20E030E04AE771
:1055D00054E40E94F0A9AB01BC0122E08091530683
:1055E000909154060E94BB4C6DE37DE08091530680
:1055F000909154060E94AB4D97EDE92E9EE0F92E56
:1056000028E1422E2CEF522E3AE0A32EB12C44E694
:10561000C42ED12C5EE0252ED7012C91222309F433
:10562000A5C1F7013297008111810115110509F417
:105630009DC18EE69EE5A1E0BB27820F911DA11DB5
:10564000B11DABBFFC01879133243394811101C09C
:10565000312C2091530630915406C801019784974C
:1056600090F56DE17DE0C9010E943A4C09500C3182
:1056700048F4E02FF0E0EE0FFF1FE351FC4F608194
:10568000718102C06DE37CE08091530690915406D5
:105690000E943A4C0C3130F4E02FF0E0EB5DFB4F10
:1056A000808101C080E090E08D5E924F092E000C59
:1056B000AA0BBB0BABBFFC018791B22DB81B8B2F84
:1056C00009F0FBC0FCC0C80184569109843893409E
:1056D00008F03FC063E07DE0C9010E943A4CC80178
:1056E000B6010E9450A96130710531F06230710538
:1056F00059F46FEF7CE002C061E07DE080915306D9
:10570000909154060E943A4C0E9477608090530614
:10571000909054063320B1F0C8010E940C8D811185
:1057200007C06BEF7CE0C4010E943A4C87E0C5C023
:10573000813009F0C4C068EF7CE0C4010E943A4C9B
:1057400088E0BBC06FEE7CE0C4010E943A4C82E06E
:10575000B4C0C801885E93408035964408F069C0A3
:10576000C80168EE73E00E9450A94B0162EE7CE034
:10577000C9010E943A4C2AE08216910410F40E945A
:105780006F60B40180915306909154060E94A378F3
:105790000E9477606090530670905406332009F49D
:1057A00042C0C8010E940C8D282F6DED7CE0C30122
:1057B0002FAB0E943A4C849CC001859C900D949C18
:1057C000900D1124800F911FB5010E9464A9809152
:1057D0005306909154062FA9633059F06530C9F0F3
:1057E000623009F06CC0243008F03CC164ED7CE00C
:1057F0003BC1233018F462EC7CE036C1233019F44D
:1058000069EB7CE031C1243008F459C060EB7CE0E6
:105810002BC1622F0E94897868EA7CE08091530650
:105820009091540621C16FE97CE0C3010E943A4C7B
:1058300043C0C80188539A44883E934000F5093319
:105840008AE4180771F00A339AE4190789F00833DB
:105850001A44A9F560E97CE0C9010E943A4C8FE046
:105860002CC065E87CE0C9010E943A4C83E125C068
:1058700063E77CE0C9010E943A4C8CE01EC0C8017D
:1058800080529E44883E934020F400526CE57CE0B8
:1058900009C0C80188509245883E934080F4085062
:1058A00065E47CE0C9010E943A4C0A3010F40E9481
:1058B0006F60802F0E94CA5F84E00E940C8068E3C2
:1058C0007DE080915306909154060E943A4C6DE21F
:1058D0007DE080915306909154060E943A4CD70186
:1058E0006C9170E080915306909154060E94A378C9
:1058F000F70180818A3010F40E946F600E94776007
:10590000D7014C91B9E2B49FA0011124052E000CDF
:10591000660B770B8BA99CA9ADA9BEA9480F591F8F
:105920006A1F7B1FDE0111968A019B010F5F1F4FCB
:105930002F4F3F4F6BBFFA0187918D93B901A8019B
:105940008111F2CFBE016F5F7F4F8091530690911E
:1059500054060E949B4D8091530690915406DC01A1
:10596000ED91FC910284F385E02D1995B3E0EB0EE7
:10597000F11CEFE4EE16EFE0FE0609F04DCE0E94BA
:10598000248E8091530690915406DC01ED91FC9198
:105990000284F385E02D1995809153069091540669
:1059A0000E94984D0E947F606EED7DE080915306CD
:1059B000909154060E94AB4D0E947F606BEC7DE09D
:1059C00080915306909154060E943A4C0E94335A9B
:1059D00020E030E040E050E40E9491AD2091530679
:1059E0003091540687FF43C068EC7DE0C9015DC07B
:1059F000F090790F00917C0F10E00C94862468ECF5
:105A000078E080915306909154060E943A4C609140
:105A1000661280915306909154060E94897866EC34
:105A200078E080915306909154060E943A4C0C9471
:105A300006256DE778E080915306909154060E9408
:105A40003A4C6091681280915306909154060E94DE
:105A500089786BE778E080915306909154060E9414
:105A60003A4C32C86BEC7CE00E943A4C28CF64EC94
:105A70007DE0C9010E94AB4D61EB7DE08091530652
:105A8000909154060E943A4C0E94335AAB01BC01DB
:105A900022E080915306909154060E94BB4C6FEA1D
:105AA0007DE080915306909154060E94AB4D6CE9C5
:105AB0007DE080915306909154060E943A4C80916B
:105AC000E60F0E9446602091E60F80915306909168
:105AD0005406222379F069E97DE00E943A4C0E9445
:105AE0004B806FE87DE080915306909154060E94B0
:105AF000AB4D02C00E94984D0E94248E80915306A7
:105B000090915406DC01ED91FC910284F385E02D27
:105B1000199580915306909154060E94984D0E94C9
:105B20007F6066E37EE080915306909154060E9468
:105B3000AB4D0E947F6062E27EE0809153069091BF
:105B400054060E943A4C4091D60F5091D70F609165
:105B5000D80F7091D90F80915306909154060E94EE
:105B600090786EE07EE080915306909154060E94FA
:105B70003A4C4091DE0F5091DF0F6091E00F709131
:105B8000E10F80915306909154060E9490786AEF3D
:105B90007DE080915306909154060E943A4C4091CA
:105BA000DA0F5091DB0F6091DC0F7091DD0F809167
:105BB0005306909154060E94907866EE7DE08091A5
:105BC0005306909154060E943A4C4091E20F509136
:105BD000E30F6091E40F7091E50F8091530690916F
:105BE00054060E9490780E94248E809153069091D2
:105BF0005406DC01ED91FC910284F385E02D1995AA
:105C000080915306909154060E94984D0E947F60A7
:105C1000E7960FB6F894DEBF0FBECDBFDF91CF91F0
:105C20001F910F91FF90EF90DF90CF90BF90AF90BA
:105C30009F908F907F906F905F904F903F902F90AC
:105C400008952F923F924F925F926F927F928F9220
:105C50009F92AF92BF92CF92DF92EF92FF920F93FB
:105C60001F93CF93DF93CDB7DEB7C65AD1090FB6D6
:105C7000F894DEBF0FBECDBFCDB6DEB6CC55DF4F3C
:105C80001882C45AD040CD55DF4F1882C35AD04035
:105C90008091C90C8A3709F447C0C0F4873709F4EA
:105CA000D9C238F48F3109F430C5863709F4E2C11E
:105CB000F2C5883709F4DDC2893709F0ECC50E94C6
:105CC00059840E9460512B013C0129C08E3709F490
:105CD0002EC338F48B3709F4CAC18C3709F4D8C203
:105CE000DAC5813809F402C5823809F4EDC4803878
:105CF00009F0D1C565C40E946051DC01CB01841953
:105D00009509A609B70980329340A105B10508F0AD
:105D100007C50E9407420E9459840E941D480E94A4
:105D20009B84029741F7FCC40E949B84029729F050
:105D300060E084E80E94D8488BC18091700A82306C
:105D400031F0833039F482E08093F20C03C081E0BB
:105D500080933F1281E08093D30C8E010C551F4F2E
:105D60002BE0AE0144575F4F68E871E90E945A4842
:105D70000E947084893058F0015011092BE0AE0167
:105D80004F575F4F68E872E981E00E945A481092CD
:105D9000D20C772473940E948684882309F43DC131
:105DA000198222961FAE22978091D20C81110EC0CB
:105DB000BE0164577F4FCE018F5B9F4F0E94AFACF7
:105DC000CC55DF4F0881C45AD0400FC07092D20C1E
:105DD000BE016F577F4FCE018F5B9F4F0E94AFACCC
:105DE000CD55DF4F0881C35AD0401091D20CADB6CB
:105DF000BEB680916C0AEDB7FEB722E0829FE01933
:105E0000F10911240FB6F894FEBF0FBEEDBF8DB798
:105E10009EB701967C0165EA75E0CE0183569F4FDF
:105E20000E94FB4B8091700A823089F0833061F1CF
:105E3000813009F0A1C040916C0A50E0B701809117
:105E40001812909119120E94D24410E039C020918A
:105E50006C0A30E05FB7F89440E0842F90E082173E
:105E6000930774F4880F991FF701E80FF91FDC01FD
:105E7000A25EBD4E8D919C91918380834F5FEDCF4B
:105E80005FBF10923E121CC020916C0A30E05FB7D9
:105E9000F89440E0842F90E08217930774F4880F01
:105EA000991FF701E80FF91FDC01A850B34F8D913E
:105EB0009C91918380834F5FEDCF5FBF109215124D
:105EC0006DE270E0CE0183569F4F0E942A4B2091D5
:105ED0006C0A293048F0112321F0113021F418E028
:105EE00004C028E001C020E010E0121758F5F701C7
:105EF000E10FF11DE10FF11D608171814AE0CE01DA
:105F000089569F4FCB55DF4F2883C55AD0400E94FA
:105F1000D04BBE0169567F4FCE0183569F4F0E94E2
:105F2000514BCE0189569F4F0E94CB4BCE018356D9
:105F30009F4F0E9497851F5FCB55DF4F2881C55A21
:105F4000D040D3CF40E450E0BE016F5F7F4FCE0121
:105F500083569F4F0E948E85CF55DF4F1881C15ABF
:105F6000D040CE0183569F4F0E94CB4B0FB6F89482
:105F7000BEBE0FBEADBE0BC0CE0183569F4F0E946A
:105F8000CB4B0FB6F894BEBE0FBEADBE10E0BE0147
:105F90006F5F7F4FCE018F5B9F4F0E94AFAC010FB1
:105FA00010E0E1E4F0E0EC0FFD1FE00FF11F1082C4
:105FB000BE016F5B7F4F8091EB0C9091EC0C0E94C7
:105FC0005E4CB801CE018F5B9F4F0E943A48BC01E6
:105FD0008091EB0C9091EC0C0E94A3786AE0809188
:105FE000EB0C9091EC0C0E94334C8091EB0C909157
:105FF000EC0CDC01ED91FC910284F385E02D199508
:106000000E947084893048F08091D20C811103C0C5
:106010007092D20C02C01092D20C0E9459840E943D
:106020001D480E942B6881110CDE8091C80C8111E3
:106030000FC08091D30C882359F08091ED0C811111
:1060400007C08091C60C9091C70C0A970CF4A3CEA0
:106050008091700A823039F0833009F01CC481E0ED
:106060008093F20C18C481E080933F1214C4109204
:10607000D30C48C31091CC0C8FEF810F853028F0E2
:1060800060E089E80E94D84806C4133079F018F41B
:106090001230F9F004C0143079F0153099F040E670
:1060A000442E49E0542E612C712C19C0412C3BE444
:1060B000532E612C712C13C0412C26E9522E612CD9
:1060C000712C0DC0412C92EC592E66246394712CD6
:1060D00006C080E8482E85E2582E612C712C00E025
:1060E000E12EF12C5701BFE8AB0EB11C1501E8946D
:1060F00027F83324E6E9EE0EF11CE894E7F8FF24D4
:10610000023091F018F4013051F004C0033089F0EE
:106110000430A1F040E659E060E070E013C040E8D0
:1061200055E260E070E00EC040E05BE460E070E0EB
:1061300009C040E056E960E070E004C040E052EC85
:1061400061E070E08FE497E00E94926C8FE497E04A
:106150000E944F4A0E9460514B015C01F2E38F0E96
:10616000911CA11CB11C0E94DF470E946051681560
:1061700079058A059B05B8F360E870E08FE497E045
:106180000E94206A6FE070E08FE497E00E94206A2E
:10619000612F8FE497E00E94094AB1018FE497E0F4
:1061A0000E94206A0E9460514B015C012AE0820E2D
:1061B000911CA11CB11C0E94DF470E946051681510
:1061C00079058A059B05B8F367E870E08FE497E0EE
:1061D0000E94206A6FE070E08FE497E00E94206ADE
:1061E000612F8FE497E00E94094AB7018FE497E09E
:1061F0000E94206A8FE497E00E944F4A0E946051FB
:106200004B015C013EE5830E31E0931EA11CB11CE5
:106210000E94DF470E946051681579058A059B0539
:10622000B8F30F5F053009F06BCFB301A2018FE423
:1062300097E00E94926C4092DE0F5092DF0F6092C6
:10624000E00F7092E10FB301A2018AEA91E00E948F
:10625000CA8558C283E090E00E9491AA2AE0DC013E
:106260002C932FE437E012963C932E9311976AE01B
:106270000CC083E090E00E9491AA2DE0FC012083F5
:106280002FE437E0328321836DE00E942E443AC22E
:106290004091CC0C5091CD0C0091CE0C1091CF0CB4
:1062A0006091CA0C7091CB0CCE010196CB55DF4F9B
:1062B0004883C55AD040CA55DF4F5883C65AD0408C
:1062C0000E94C27ECB55DF4F4881C55AD040CA5587
:1062D000DF4F5881C65AD040892BE9F08D81873035
:1062E00050F4853080F48130B0F0642F8B819C8134
:1062F0000E940E790DC0893070F4B8018B819C81A9
:106300000E94CA8505C0BA018B819C810E94AB772F
:106310000E94878E04C061E085E80E94D848809181
:10632000C50C8111B8C281E08093C50CB4C2B09095
:10633000CA0CE090CB0CC956DF4F1882C759D04029
:1063400065EA75E0CE018F579F4F0E94FB4B6B2D86
:106350007E2DCE0184579F4F0E94C27E892B09F467
:10636000C9C0C057DF4FE881C059D0404E2F50E020
:10637000FA013197E830F10508F0BCC08827ED5DDF
:10638000FE4F8F4F0C9477A9C257DF4F88819981B8
:10639000CE58D0400E94BAAE23961FAE1EAE2397B1
:1063A00025961FAE1EAE259727961FAE1EAE2797C9
:1063B0004AE0BE016F5F7F4F90E03EC0C257DF4FA3
:1063C00088819981CE58D0400E94BAAE682F880F3C
:1063D000770B4AE00AC0C257DF4F88819981CE58B7
:1063E000D0400E94C7AE4AE0BC01CE0101960E9497
:1063F000D04BBE016F5F7F4FCE018F579F4F0E94E2
:10640000F14ACE01019663C0C257DF4F888199815E
:10641000CE58D0400E94C7AE23961FAE1EAE239723
:1064200025961FAE1EAE259727961FAE1EAE279748
:106430004AE0BE016F5F7F4F0E9468AD35C0C25712
:10644000DF4F88819981CE58D0400E94C2AE2396FA
:106450001FAE1EAE239725961FAE1EAE259727961C
:106460001FAE1EAE27972AE0AE014F5F5F4F0E941E
:1064700039AD1AC0C257DF4F88819981CE58D040BC
:106480000E94C2AE23961FAE1EAE239725961FAE66
:106490001EAE259727961FAE1EAE27972AE0AE01A7
:1064A0004F5F5F4F0E9447ADBE016F5F7F4FCE01D0
:1064B0008F5B9F4F0E94AB4BBE016F5B7F4FCE0146
:1064C0008F579F4F0E94F14ACE018F5B9F4F0E94D2
:1064D000CB4B4BE050E0BE016F5B7F4FCE018F573F
:1064E0009F4F0E948E85CB57DF4FF880C558D04014
:1064F00011E002C0F12C10E0CE018F579F4F0E9497
:10650000CB4B112309F4BCCD8E0109561F4F20E45B
:10651000AE014F5F5F4F68E87B2D8E2D0E945A4879
:10652000BE016F5B7F4FCE0101960E94AFACC95692
:10653000DF4F8881C759D040F80E81E08F0DC956D2
:10654000DF4F8883C759D040E1E0F0E0EC0FFD1F3A
:10655000EF0DF11D9CE79083E1E0F0E0EC0FFD1FF3
:10656000E80FF11D1082BE016F5F7F4F8091EB0C31
:106570009091EC0C0E945E4CC956DF4F6881C75960
:10658000D04070E0CE0101960E943A48BC01809153
:10659000EB0C9091EC0C0E94A3786AE08091EB0CDC
:1065A0009091EC0C0E94334C8091EB0C9091EC0C90
:1065B000DC01ED91FC910284F385E02D19956BC10E
:1065C0008091CA0C9091CB0C8038910509F063C181
:1065D0008E0104571F4F20E4AE014F5F5F4F68E804
:1065E00070E880E00E945A486DE875E0CE018F5750
:1065F0009F4F0E94FB4BCE018F579F4F0E94978564
:10660000C457DF4F2881CC58D040CB57DF4F88810B
:106610009981C558D040820F911DC457DF4F8883A0
:10662000CC58D04022961FAE22974BE050E0BE01DE
:106630006F5B7F4FCE018F579F4F0E94AC7ABE0198
:106640006F5B7F4FCE0101960E94AFACC457DF4F06
:106650008881CC58D040E1E0F0E0EC0FFD1FE80F5E
:10666000F11D1082BE016F5F7F4F8091EB0C909106
:10667000EC0C0E945E4CC457DF4F6881CC58D04070
:1066800070E0CE0101960E943A48BC018091EB0C6B
:106690009091EC0C0E94A3786AE08091EB0C9091B1
:1066A000EC0C0E94334C8091EB0C9091EC0CDC01D3
:1066B000ED91FC910284F385E02D1995CE018F5761
:1066C0009F4F0E94CB4BE7C08091CA0C9091CB0C9E
:1066D0008238910509F0DFC08E0104571F4F20E476
:1066E000AE014F5F5F4F68E872E87BCF8091CA0CC4
:1066F0009091CB0C8138910509F0CDC08091D30CDD
:106700008111C9C00E94878EC6C08091CA0C909129
:10671000CB0C4F9709F0BFC081E08093C80CBBC081
:106720000E949B84029719F060E084E8ABCC8091D2
:106730006F0A811102C00E9428790E947084F82E8D
:1067400065EA75E0CE0184579F4F0E94FB4BC95606
:10675000DF4F1882C759D0408E0109561F4F20E4E1
:10676000AE014F5F5F4F68E879E780E00E945A48CA
:10677000CF57DF4F19821882C158D040CD57DF4F15
:1067800019821882C358D040CB57DF4F1982188224
:10679000C558D0406F2D70E080E090E02AE0AE0157
:1067A0004F5B5F4F0E9439ADBE016F5B7F4FCE01E3
:1067B0008F579F4F0E94AB4BBE016F577F4FCE014B
:1067C00084579F4F0E94F14ACE018F579F4F0E94DE
:1067D000CB4B4BE050E0BE016F5B7F4FCE01845747
:1067E0009F4F0E94AC7AC057DF4F1881C059D040EC
:1067F000BE016F5B7F4FCE0101960E94AFACC956C0
:10680000DF4F8881C759D040810F91E0980FC9565A
:10681000DF4F9883C759D040E1E0F0E0EC0FFD1F57
:10682000E80FF11D8CE78083E1E0F0E0EC0FFD1F45
:10683000E90FF11D1082BE016F5F7F4F8091EB0C5D
:106840009091EC0C0E945E4CC956DF4F6881C7598D
:10685000D04070E0CE0101960E943A48BC01809180
:10686000EB0C9091EC0C0E94A3786AE08091EB0C09
:106870009091EC0C0E94334C8091EB0C9091EC0CBD
:10688000DC01ED91FC910284F385E02D1995CE0198
:1068900084579F4F16CF0FB6F894DEBE0FBECDBE05
:1068A000CA55DF4F0FB6F894DEBF0FBECDBFDF91E4
:1068B000CF911F910F91FF90EF90DF90CF90BF90FD
:1068C000AF909F908F907F906F905F904F903F9090
:1068D0002F9008950F931F93CF93DF938C01C1E006
:1068E000D0E00C171D07ACF00E94775964E670E009
:1068F00080E090E00E9428510E947359C017D10790
:1069000034F46AE570E080E090E00E94285121961E
:10691000E8CFDF91CF911F910F91089583E090E030
:10692000D9CF82E090E0D6CF81E090E0D3CF60E095
:1069300089E30E94B24F60E08AE30E94B24F60E0B8
:1069400085E30E94B24F60E085E00E94B24F60E0B4
:1069500084E00E94B24F60E087E00E94B24F7298DC
:106960000895CF93C0910A026C2F89E30E94B24F21
:1069700081E0C8276C2F8AE30E94B24FC0930A02BD
:10698000CF910895CF93DF93C09109026C2F89E3D3
:106990000E94B24FD1E0DC276D2F8AE30E94B24FF4
:1069A0006C2F85E30E94B24F6D2F85E00E94B24F9D
:1069B0006D2F84E00E94B24F6C2F87E00E94B24F8F
:1069C000CC2311F0729801C0729A9091090281E073
:1069D000892780930902DF91CF910895CF93DF93A8
:1069E0008091DF0C81110DC01092DE0C1092DD0C35
:1069F00081E090E09093DC0C8093DB0C8093DF0CC3
:106A000036C08091DD0C9091DE0C863191057CF1D1
:106A10008F38910534F48091DB0C9091DC0C019659
:106A200009C08D3521E0920754F48091DB0C9091E0
:106A3000DC0C02969093DC0C8093DB0C18C0863241
:106A400022E0920734F48091DB0C9091DC0C0496E8
:106A5000F1CF883E93403CF48091DB0C9091DC0CAC
:106A60008A5B9F4FE7CF1092DC0C1092DB0C8ADF21
:106A7000C091DD0CD091DE0CC93E83E0D80754F004
:106A80001092DF0C54DF26E635E348EE53E060E079
:106A900070E007C02EEE34E3AE010D2E000C660B45
:106AA000770B85E89AE00E9423409093DA0C80935C
:106AB000D90C8091DB0C9091DC0C8C0F9D1F909376
:106AC000DE0C8093DD0CDF91CF910895CF93DF939F
:106AD00080915806882319F0DF91CF917FCFC09124
:106AE000D90CD091DA0CBE0185E89AE00E94BC3F37
:106AF000882329F0BE0185E89AE00E94D43FDF9107
:106B0000CF9115CFCF93DF93C091D70CD091D80CF4
:106B1000BE0185E89AE00E94BC3F882361F0BE0177
:106B200085E89AE00E94D43F1092D80C1092D70CBE
:106B3000DF91CF91FCCEDF91CF910895CF93DF937A
:106B4000CDB7DEB728970FB6F894DEBF0FBECDBF26
:106B50008091D40C8823C1F11092D40CD3DF8091A2
:106B60005606882389F160E57EE080915306909176
:106B700054060E943A4CE091700AE4300CF0E0E0D8
:106B80008AE095E09A83898386E095E09C838B83F5
:106B900081E095E09E838D838CEF94E098878F83CE
:106BA000EE0FFF0BEC0FFD1F618172818091530688
:106BB0009091540628960FB6F894DEBF0FBECDBF55
:106BC000DF91CF910C94AB4D28960FB6F894DEBFB1
:106BD0000FBECDBFDF91CF9108956091D70C70911A
:106BE000D80C85E89AE00E94BC3F81112EC060E07D
:106BF00089E30E94B24F60E08AE30E94B24F60E0F6
:106C000085E30E94B24F60E085E00E94B24F60E0F1
:106C100084E00E94B24F60E087E00E94B24F729819
:106C20008091F40F882319F022EC34E302C021EBA9
:106C300034E342E350E060E070E085E89AE00E94CF
:106C40002B409093D80C8093D70C08958091D40C4E
:106C5000811112C00E94BA5B81E08093D40CBDDF29
:106C600080915506882341F061E47EE080915306CF
:106C7000909154060C94AB4D089560E08AE30C9417
:106C8000B24F61E08AE30C94B24F0F931F93CF93FE
:106C9000DF938C01C1E0D0E00C171D079CF0F1DF01
:106CA00064E670E080E090E00E942851E6DFC017C3
:106CB000D10734F46AE570E080E090E00E9428514A
:106CC0002196EACFDF91CF911F910F9108952F92D6
:106CD0003F924F925F926F927F928F929F92AF926C
:106CE000BF92CF92DF92EF92FF920F931F93CF93B9
:106CF000DF9300D0CDB7DEB75C010E94BA5BBDDF89
:106D00000E94775980915306909154060E94984DA5
:106D10000E947F6024E0A216B10409F448C085E017
:106D2000A816B10409F479C0A3E0AA16B10409F0C9
:106D3000B1C08CE190E00E9491AA9B838A8385E890
:106D400095E0EA81FB8191838083B382A28281E016
:106D50009FEF958384838FEF90E0978386831186DE
:106D60001086108ECF010E94598289E795E0AA8192
:106D7000BB818D939C93E091810DF091820DD08C1D
:106D8000009162111091631116950795E0906011C2
:106D9000F0906111F694E79463E47FE080915306EC
:106DA000909154060E94AB4D2224239490C08CE114
:106DB00090E00E9491AA9B838A8385E895E0EA810E
:106DC000FB8191838083B382A28281E09FEF9583D0
:106DD00084838FEF90E09783868311861086108ED0
:106DE000CF010E94598289E795E0AA81BB818D93EA
:106DF0009C93E0915106F0915206D08C009177114E
:106E00001091781116950795E0907511F090761114
:106E1000F694E79466E77FE035C08CE190E00E944D
:106E200091AA9B838A8385E895E0EA81FB8191831F
:106E30008083B382A28281E09FEF958384838FEF6A
:106E400090E09783868311861086108ECF010E9472
:106E5000598289E795E0AA81BB818D939C93E0914B
:106E60004D06F0914E06D08C00918C1110918D1131
:106E700016950795E0908A11F0908B11F694E7949F
:106E800066E57FE080915306909154060E94AB4DD9
:106E9000212C1DC06AE27FE0809153069091540638
:106EA0000F900F900F90DF91CF911F910F91FF9056
:106EB000EF90DF90CF90BF90AF909F908F907F909A
:106EC0006F905F904F903F902F900C94AB4D0E942D
:106ED0007F606DE17FE080915306909154060E949F
:106EE000AB4D61E17FE080915306909154060E9482
:106EF0003A4CB80180915306909154060E94D9787B
:106F000065E07FE080915306909154060E943A4CD0
:106F1000B70180915306909154060E94D97869EF89
:106F20007EE080915306909154060E943A4C8D2D3C
:106F30000E945B6080915306909154060E94984D88
:106F4000AA81BB81ED91FC9111970280F381E02D24
:106F5000CD011995CA2C8A2D0E9475818D3D9540D1
:106F6000A8F464E378E08A2D0E94F741EA81FB816E
:106F7000F78AE68AB70182810E9485816CED75E00F
:106F80008A2D0E947081DD20C1F01AC064E873E090
:106F90008A2D0E947081AA81BB8157961C930E9303
:106FA0005697B80112968C910E9485816CED75E020
:106FB0008A2D0E94F741DD2019F09924939401C095
:106FC000912C33243394812C21E029830E94F144B5
:106FD00080910B11882359F1AA81BB81ED91FC911D
:106FE000119760911011709111110190F081E02DB5
:106FF000CD0119958C2D0E9475818D3DB5E09B07C3
:107000005CF48438E3E09E0784F08C018D3D95406C
:1070100074F00CED15E00BC07C01853398403CF01A
:1070200064E3E62E68E0F62E02C004E813E029814E
:1070300021111FC0809101118823C9F1E09108112D
:10704000F0910911858196814091041150910511AB
:107050009C0121533109421753074CF1C196841703
:1070600095072CF10E9460516415750586059705FA
:10707000F0F0809101118823C1F0409104115091EA
:107080000511E0910811F0910911858196819C010B
:10709000285C3109421753072CF088539F4F8417FF
:1070A00095071CF481E0982605C021E029838820FB
:1070B00009F47CC0992009F445C0DD20F9F064E8AA
:1070C00073E08C2D0E947081222009F458C06091D9
:1070D000640F7091650F41E08C2D0E94B6410E94B3
:1070E000248EAA81BB8112968C910E94758108170B
:1070F0001907ACF38C2D0E94884141C064E378E00D
:107100008C2D0E94F7412220B1F06091640F7091A4
:10711000650F40E08C2D0E94B6410E94248EAA810A
:10712000BB8112968C910E9475818E159F05ACF3E0
:107130008C2D0E948841EA81FB81F78AE68AB7019B
:10714000828110C0DD20B1F064E378E08C2D0E94D4
:10715000F741AA81BB815796FC92EE925697B701F0
:1071600012968C910E9485816CED75E08C2D0E94A9
:10717000708112C064E873E08C2D0E947081EA81F6
:10718000FB81178B068BB80182810E9485816CED93
:1071900075E08C2D0E94F7410E9460512B013C014B
:1071A000F8EC4F0E511C611C711C19823320D1F177
:1071B0008091F7108823A1F14091FA105091FB10B3
:1071C000E091FE10F091FF10858196819C01285C72
:1071D0003109421753072CF088539F4F84179507A6
:1071E000FCF481E0D8268091530690915406DD206E
:1071F00039F06AEE7EE00E94AB4D82E090E006C07E
:1072000068ED7EE00E94AB4D81E090E03EDD0E94A3
:107210006051AA81BB815896DC928824839403C074
:10722000812C1EC0812C8091F710882309F4FEC1A7
:10723000E091FE10F091FF10858196814091FA1047
:107240005091FB109C0121533109421753070CF454
:10725000EDC1C19633243394841795070CF4E6C12D
:107260000E9459840E941A7885E89AE0FCD68091A1
:10727000740A882309F4AACE8091760A882309F437
:10728000A5CE0E941A780E9457868823D1F3B4E0D5
:10729000AB16B10459F0E5E0AE16B10409F463C0D1
:1072A000F3E0AF16B10409F04FC1C7C01093510FFE
:1072B0000093500FF092530FE092520FD092540F60
:1072C000B8018CE191E00E94AB77B7018EE191E0CB
:1072D0000E94AB776D2D80E291E00E940E79B8019B
:1072E00084E0B7D7B70184E099D7E0915106F091D7
:1072F0005206D08E80914F0F8D3029F4E091D50C3D
:10730000F091D60CD08E6CED75E084E00E94858102
:1073100066E970E080E090E00E94285180914F0F74
:107320008D30E1F484E00E947581A0915106B09106
:107330005206ED91FC9111970190F081E02D8D3D69
:1073400095401CF06FEF7FEF02C061E070E0CD016F
:107350001995809151069091520659C0809151061D
:107360009091520662C01093580F0093570FF092FD
:107370005A0FE092590FD0925B0FB80183E291E06F
:107380000E94AB77B70185E291E00E94AB776D2D4B
:1073900087E291E00E940E79B80185E05AD7B701E3
:1073A00085E03CD7E0914D06F0914E06D08E6CED15
:1073B00075E085E00E94858166E970E080E090E0FC
:1073C0000E94285180914E0F8D3059F585E00E9422
:1073D0007581A0914D06B0914E068D3D95404CF0C3
:1073E000ED91FC9111970190F081E02D6FEF7FEF0F
:1073F00008C0ED91FC9111970190F081E02D61E0C2
:1074000070E0CD01199580914D0690914E06DC01FA
:10741000ED91FC910190F081E02D60E070E0199514
:1074200093C080914D0690914E06DC01ED91FC9148
:107430000480F581E02D199587C01093670F0093A4
:10744000660FF092690FE092680FD092600FB8015A
:1074500082E391E00E94AB77B70184E391E00E9460
:10746000AB776D2D8CE291E00E940E79B80183E03C
:10747000F0D6B70183E0D2D68091600FE091810D04
:10748000F091820D808F8091600F0E94767783E06B
:107490000E9475812091600F222359F1B9E0BC153B
:1074A00038F020916211309163113695279502C012
:1074B0002EEE32E08217930709F446C06091640F04
:1074C0007091650F41E083E051D70E94248EEA81DC
:1074D000FB8182810E94758108171907B4F383E04C
:1074E00017D7AA81BB8157961C930E935697B80164
:1074F00027C029E02C1508F49BC020916011309121
:1075000061113695279582179307F1F06091640F0A
:107510007091650F40E083E029D70E94248EEA81B4
:10752000FB8182810E9475818E159F05B4F383E0F3
:10753000EFD6AA81BB815796FC92EE925697B7017F
:1075400012968C910E9485818091530690915406E9
:107550000E94984D0E947F60B4E0AB16B10459F0D0
:10756000E5E0AE16B10451F0F3E0AF16B10471F4EA
:107570006EE87EE005C06EEB7EE002C065EA7EE06C
:1075800080915306909154060E94AB4D0E947F60FB
:1075900063E87EE080915306909154060E94AB4DC3
:1075A00067E77EE080915306909154060E943A4C22
:1075B000B80180915306909154060E94D9786BE6E9
:1075C0007EE080915306909154060E943A4CB70198
:1075D00080915306909154060E94D9786FE57EE021
:1075E00080915306909154060E943A4C8D2D0E9432
:1075F0005B6080915306909154060E94984D0F90C5
:107600000F900F90DF91CF911F910F91FF90EF900E
:10761000DF90CF90BF90AF909F908F907F906F90B2
:107620005F904F903F902F900C947359312C18CE4F
:107630002AEC38E068CF83E090E027CB82E090E04E
:1076400024CB81E090E021CB8091E70C9091E80C75
:1076500091609093E80C8093E70C08958091E70C7B
:107660009091E80C80689093E80C8093E70C089563
:107670008091E70C9091E80C80619093E80C8093E6
:10768000E70C0895FC018281882371F083818823AF
:1076900059F013828091E70C9091E80C24E0822746
:1076A0009093E80C8093E70C0895FC018281882375
:1076B00071F0838181110BC081E083838091E70C9D
:1076C0009091E80C84609093E80C8093E70C089507
:1076D000FC018481882371F08581882359F015820B
:1076E0008091E70C9091E80C28E082279093E80CB9
:1076F0008093E70C0895FC018481882371F08581D3
:1077000081110BC081E085838091E70C9091E80C9A
:1077100088609093E80C8093E70C08958091E70CC3
:107720009091E80C20E282279093E80C8093E70C7C
:1077300008958091E70C9091E80C80629093E80C9A
:107740008093E70C0895DC01ED91FC910680F781B0
:10775000E02D60E070E0199477FF03C071956195AA
:1077600071096F3F710519F014F06FEF70E08091AF
:10777000E70C9091E80C8C7B91709093E80C8093CF
:10778000E70C8091E70C9091E80C6F30710514F4D0
:1077900080641FC06733710514F481641AC06F35AB
:1077A00071051CF48164906114C0673871051CF484
:1077B000816490630EC06F3A71051CF4816490641B
:1077C00008C0673D71051CF48164906502C0816446
:1077D00090669093E80C8093E70C089580E094E025
:1077E0009093E80C8093E70C08958091E70C9091BA
:1077F000E80C92609093E80C8093E70C8091E70C82
:107800009091E80C80649093E80C8093E70C0895C5
:107810000895089508950895089508950895089580
:107820000895089580E008950895089508950895AD
:107830000895089508950895089508950895089560
:107840000895089580E0089508950895FC016483E3
:107850000895FC0162830895FC011382148215824D
:107860001682178210860895089508950895FC01E0
:1078700083810895FC0164830895FC016783089562
:10788000FC0165830895FC0182810895FC01128248
:1078900013821482158261E086E10E94E14F61E06B
:1078A00086E10E94B24FE2E7F0E080818160808350
:1078B0001092E80C1092E70C0895FF920F931F931B
:1078C000CF93DF938C01C62FF42ED22F6AED70E098
:1078D000DC0119968D919C911A970E94206AF801FB
:1078E00081859285DC01ED91FC910190F081E02D84
:1078F0006C2F1995F80181859285DC01ED91FC9141
:107900000190F081E02D6F2D1995F8018185928508
:10791000DC01ED91FC910190F081E02D6D2F199526
:10792000EC2FF0E0BF0166527F4F6F0D711D6D0FA0
:10793000711D6F777727F80181859285DF91CF914F
:107940001F910F91FF900C94206A20E040E0B5CF8A
:1079500065E4FBCF68E4F9CFCF93DF93FC0123818B
:10796000222321F0EC0161E4F0DF1B82DF91CF9153
:107970000895CF93DF93FC012381211105C0EC0111
:1079800060E4E3DF81E08B83DF91CF910895FC0118
:107990002481222311F06CE3D8CF0895FC012781C4
:1079A000222331F02085222319F010866BE3CDCFFE
:1079B0000895FC012781222339F02085211104C07C
:1079C00021E020876AE3C1CF0895FC0125812223AD
:1079D00031F02681222319F0168269E3B6CF08958B
:1079E000FC012581222339F02681211104C021E0E8
:1079F000268368E3AACF089567E3A7CF6AE4A5CFFB
:107A000069E4A3CF66E3A1CF65E39FCF6EE49DCF8A
:107A100064E39BCF63E399CF62E397CF61E395CFB4
:107A200060E393CF6FE291CF6DE28FCF6CE28DCFA9
:107A3000242F462F6CE441CF77FF03C071956195E9
:107A4000710920E0462F6EE238CF462F20E067E430
:107A500034CF462F20E066E430CF262F64E42DCFCC
:107A6000CF92DF92FF920F931F93CF93DF938C01FE
:107A7000F62E443F81E0580738F0413187E258073D
:107A800028F040E157E202C044EF51E0243F81E09A
:107A9000380738F0E9012131374228F0C0E1D7E258
:107AA00002C0C4EFD1E0CA01845F914022E3C22E3C
:107AB000D12CB6010E9450A9462F2F2D62E4C80197
:107AC000FCDECE01845F9140B6010E9450A9462F92
:107AD0002F2D63E4C801DF91CF911F910F91FF908B
:107AE000DF90CF90EACE262F40E06FE3E6CE262F40
:107AF00040E06EE3E2CE262F40E06DE3DECE462F7F
:107B000020E06DE4DACEFC016283611104C020E064
:107B100040E06BE4D2CE089577FF03C07195619584
:107B2000710920E0462F6BE4C8CE4F925F926F92AE
:107B30007F928F929F92AF92BF92CF92DF92EF92FD
:107B4000FF920F931F93CF93DF936C01A4ECCA1A9B
:107B5000ADEFDA0AD601ED91FC917E970CF05DC095
:107B6000FC01E858FF4F812C912CA191B191AB2BD6
:107B700021F42115310549F450C0BFEF8B1A9B0A3F
:107B8000AEE18A16910489F748C0EC015401AA0CB1
:107B9000BB1CAA0CBB1CAC0EBD1EF501EC54FF4F68
:107BA00040835183628373837401EE0CFF1CEC0EDF
:107BB000FD1EF701E858FF4F31832083EC54FF4F3F
:107BC00011830083BE01680D791DFB01EC55FE4F4A
:107BD00081E080830E946051F5016083718382831C
:107BE0009383C65CDD4F88819981F701E250FE4F97
:107BF00091838083D6012D913C9111972F5F3F4F48
:107C00002D933C939C012F5F3F4F1216130614F0E7
:107C100021E030E03983288302C08FEF9FEFDF91AE
:107C2000CF911F910F91FF90EF90DF90CF90BF9079
:107C3000AF909F908F907F906F905F904F9008953E
:107C40000F931F93CF93DF93EC017093090E609312
:107C5000080E40930F0E81E090E00E9491AA8C01E3
:107C60000E9459821093EA0C0093E90C91E09093E2
:107C7000EF0D9093F00D1092EE0D1092ED0D10920D
:107C8000F30D1092F20D1092F40D1092F10D24EFFD
:107C900031E03093FB0D2093FA0D28EB3BE030935D
:107CA000FD0D2093FC0D20E233E03093020E209373
:107CB000010E2CEA3DE03093040E2093030E28E0E1
:107CC00037E030930B0E20930A0E24E931E1309314
:107CD0000D0E20930C0E1092F70D1092F60D1092CF
:107CE000F50D1092FE0D1092050E10920E0E1092D0
:107CF000F90D1092F80D1092000E1092FF0D1092D7
:107D0000070E1092060E988399839A83DF91CF9184
:107D10001F910F9108951F920F920FB60F92112489
:107D20000BB60F922F933F934F935F936F937F9375
:107D30008F939F93AF93BF93EF93FF938091E60C44
:107D40008F5F8093E60C9091E50C891708F401C1D0
:107D50001092E60C8091E40C90E08730910508F0D9
:107D6000F8C0FC018827E55DFE4F8F4F0C9477A982
:107D700060E086E10E94B24F88E08093E50C81E0EC
:107D800048C061E086E10E94B24F81E08093E50C3B
:107D900036C060E086E10E94B24F8091E20C909183
:107DA000E30C97FF05C083E08093E50C84E031C0CD
:107DB00081E08093E50C83E02CC061E086E10E94C5
:107DC000B24F83E08093E50C8091E10C8F5F80934C
:107DD000E10C803150F01092E10C85E01AC061E0B6
:107DE00086E10E94B24F81E0EDCF8091E20C90914C
:107DF000E30C880F991F9093E30C8093E20C82E0D0
:107E000008C060E086E10E94B24F81E08093E50CFB
:107E100086E08093E40C9DC061E086E10E94B24F51
:107E200088E18093E50C8091E70C9091E80C9093A9
:107E3000E30C8093E20C8091E70C9091E80C91FFA9
:107E40001DC08091E00C8823B1F08091E70C9091E7
:107E5000E80C22E092279093E80C8093E70C809145
:107E6000E70C9091E80C80649093E80C8093E70C09
:107E70001092E00C03C081E08093E00C8091E70C4D
:107E80009091E80C92FF0EC08091E00C882339F0AD
:107E90001092E80C1092E70C1092E00C03C081E005
:107EA0008093E00C8091E70C9091E80C84FF14C063
:107EB0008091E00C882369F08091E70C9091E80CA8
:107EC00020E182279093E80C8093E70C1092E00C5D
:107ED00003C081E08093E00C8091E70C9091E80C66
:107EE00087FF13C08091E00C882361F08091E70C3C
:107EF0009091E80C80589093E80C8093E70C1092D6
:107F0000E00C03C081E08093E00C8091E70C90913D
:107F1000E80C90FF14C08091E00C882369F08091F8
:107F2000E70C9091E80C21E092279093E80C809365
:107F3000E70C1092E00C03C081E08093E00C80918C
:107F4000E70C9091E80C9093E30C8093E20C109274
:107F5000E40CFF91EF91BF91AF919F918F917F9131
:107F60006F915F914F913F912F910F900BBE0F90AA
:107F70000FBE0F901F901895DC01A250BE4F20E05D
:107F800030E04D915D914617570739F4280F391F9E
:107F9000F901EC55FE4F808108952F5F3F4F2E3140
:107FA000310579F780E00895CF93DF93EC01C45C4D
:107FB000DD4FA881B981109709F442C0FC01E2505D
:107FC000FE4F20E030E0419151914617570799F557
:107FD000A901440F551F480F591FFA01E858FF4FD8
:107FE00060817181672B61F111821082FC01E20FC7
:107FF000F31FEC55FE4F1082FA01EE53FE4F118233
:108000001082235D3F4F220F331F220F331FFC01CD
:10801000E20FF31F1082118212821382FA01E859D3
:10802000FE4F11821082EA56FF4F11821082119783
:10803000B983A88305C02F5F3F4F2E31310519F654
:10804000DF91CF9108950F931F9301E010E06DDD54
:108050001F910F9108950F931F9300E010E065DDCD
:108060001F910F9108952F923F924F925F926F92BE
:108070007F928F929F92AF92BF92CF92DF92EF92B8
:10808000FF920F931F93CF93DF9300D000D0CDB713
:10809000DEB78C010E94605198012E533E4F3C8305
:1080A0002B831E830D83D801AC55BE4FBA83A983A1
:1080B0001801B2E02B1ABEEF3B0AF901AA24A394DF
:1080C000B12C32E0832E912C118210829F012A5410
:1080D0003140D9012D913C91232B09F44DC0AD8144
:1080E000BE812D913D914D915C9113977D01B4EB33
:1080F000EB0EF11CD701CD90DD90ED90FC902B01A3
:108100003C01421A530A640A750A4C145D046E0459
:108110007F0490F1C20ED31EE41EF51EAD81BE8118
:10812000CD92DD92ED92FC921397A981BA812C91A8
:10813000222311F19F0126593109D9012D913C913A
:108140002115310519F4B182A08216C07F01BAE56C
:10815000EB1AF108D7014D915C9111974217530723
:108160005CF4B182A0824F5F5F4F4D935C934217E6
:10817000530714F09182808232962D813E812C5FCC
:108180003F4F3E832D83A981BA811196BA83A9837B
:10819000E215F30509F098CFEB81FC818191919173
:1081A000FC83EB838130910599F00297C9F4EB8150
:1081B000FC81EC54F1400190F081E02D1995AB81E8
:1081C000BC81DA966D917C91DB97C801EDDE08C029
:1081D000EB81FC81EC54F1400190F081E02D199588
:1081E0002B813C8122153305B9F626960FB6F894FB
:1081F000DEBF0FBECDBFDF91CF911F910F91FF90DA
:10820000EF90DF90CF90BF90AF909F908F907F9036
:108210006F905F904F903F902F9008956E3E22E0B8
:10822000720738F06B3C98E0790728F06AEC78E048
:1082300002C06EEE72E0660F771F9FB7F89425E1DB
:10824000829FF0011124E25EFE4E748363839FBF20
:1082500008956E3E22E0720738F06B3C98E0790793
:1082600028F06AEC78E002C06EEE72E0660F771FCD
:108270009FB7F89425E1829FF0011124E25EFE4E43
:10828000768365839FBF0895660F771F282F30E0A0
:1082900095E1899FF0011124E25EFE4E8581968171
:1082A0006817790718F46581768107C08381948106
:1082B0008617970710F4638174818FB7F89495E15E
:1082C000929FF001939FF00D1124E25EFE4E7283A7
:1082D00061838FBF08956CED75E080E0D5CF982F56
:1082E0008FB7F89425E1929FF0011124E25EFE4ED3
:1082F00021E027838FBF41B121E030E0B90102C006
:10830000660F771F9A95E2F7CB01842B81B9089508
:108310008A3058F49FB7F89425E1829FF001112428
:10832000E25EFE4E118610869FBF08951F93CF9385
:10833000DF9325E1829FC0011124EC01C25EDE4E75
:108340008A8581110FC01FB7F89481E08A878989D7
:108350009A899A8389830E9460516B877C878D8775
:108360009E871FBFDF91CF911F910895CF93DF9319
:108370008A30D0F56233710538F061369DE67907B1
:1083800028F060E67DE602C062E370E0D42FC82FDB
:1083900080E090E00E9495AD20E030E04AE754E4B0
:1083A0000E94F0A920E030E04CE852E40E94F6ADD3
:1083B0009B01AC0160E070E08AEF94E40E94F0A9B8
:1083C0000E9458AA9B01DD2321F022273327261B78
:1083D000370B8FB7F89495E1C99FF0011124E25E45
:1083E000FE4E318720878FBFDF91CF9108958A306D
:1083F00008F414CF089581E08093670A089581E01E
:108400008093680A089581E08093690A0895CF9364
:108410008091360DC0910B028111FFC0C23009F46A
:108420004FC0C33009F49CC0C13009F026C180910F
:10843000690A811122C181E090E00E9491AA909383
:1084400019128093181262E083E00E94E14F1092AB
:10845000350D10921212109211121092161280E025
:1084600090E0FC01EE0FFF1FED5DF24F11821082D4
:10847000019688309105A9F71092340D1092330DB2
:1084800080916A008C6080936A00ED9A8FB7F894AF
:1084900020918400309185003093220D2093210D8E
:1084A0008FBF23E032E44AEF50E060E070E080915B
:1084B0000D1290910E12C7DD81E08093360DDDC064
:1084C0008091680A8111D9C081E090E00E9491AA50
:1084D00090931B1280931A12809104018E7F8093D7
:1084E00004018091050181608093050182EB96E093
:1084F00090934512809344122EE240EA56E861E0E0
:1085000070E00E94254F809165008B7F809365000D
:108510001092350189E0809334018EE2809332011C
:108520008CEF8093300180E98093310110924312E7
:1085300010924212109241121092401210923E126A
:10854000EEE1F2E18CED95E08193919322E1EE333F
:10855000F207D1F7C1E0C0933F122FEF31E451C0D1
:108560008091670A811189C081E090E00E9491AA00
:1085700090931D1280931C12809104018E7F809332
:1085800004018091050181608093050182EB96E0F2
:108590009093F70C8093F60C26E040E052EC61E0FB
:1085A00070E00E94254F809165008B7F809365006D
:1085B0001092350180E18093340186E0809332018E
:1085C0008EEF8093300180E9809331011092141274
:1085D000109213121092F50C1092F40C10921512C6
:1085E000E8EFFCE08CED95E0819391932DE0E43190
:1085F000F207D1F71092F30CC1E0C093F20C2BEF0D
:1086000031E44AEF50E060E070E080910D1290910B
:108610000E1219DDC093360D30C0C23069F0C33080
:10862000D1F0C13051F58091690A811126C0809145
:108630001112909112121DC08091680A81111DC003
:1086400080911A1290911B120E94518380914212C4
:10865000909143120EC08091670A81110EC08091E3
:108660001C1290911D120E94717B809113129091A7
:108670001412029711F4C093700A80910B02823099
:10868000A1F1833009F454C0813009F074C08091A5
:10869000690A882309F46FC0ED98E59A1092350DA8
:1086A00010921712109212121092111210921612AA
:1086B00080E090E0FC01EE0FFF1FED5DF24F1182B4
:1086C0001082019688309105A9F71092340D10920E
:1086D000330D80911812909119120E9426AB1092BE
:1086E000360D1092680A82E044C08091680A88239F
:1086F00009F441C080914412909145120E94034FA9
:10870000809131018F7780933101809131018F7E8B
:10871000809331011092300180911A1290911B12B6
:108720000E9426AB1092360D1092670A83E021C09A
:108730008091670A8823F9F08091F60C9091F70CEC
:108740000E94034F809131018F7780933101809196
:1087500031018F7E809331011092300180911C1283
:1087600090911D120E9426AB1092360D1092690A4C
:1087700081E080930B0280910D1290910E12CF91A7
:1087800072CCAF92BF92CF92DF92EF92FF920F9393
:108790001F93CF93DF937C016B015A01D0E0C0E0BF
:1087A0008D2F90E0F701A181B2818A159B05D0F44D
:1087B000F601E80FF91F608104EF11E721E033278C
:1087C000C6270C0F111D211D311D2BBFF801C791AC
:1087D000ED91FC9111970190F081E02DCD0119955B
:1087E000DF5FDECFED91FC9111970190F081E02DDC
:1087F0006C2FCD01DF91CF911F910F91FF90EF90E2
:10880000DF90CF90BF90AF901994CF93DF9300D0BB
:108810001F921F92CDB7DEB7FE01319625E0DF0132
:108820001D922A95E9F724E8298325E52C832AE27D
:108830002D836A834B8345E050E0BF01A2DF65E0F2
:1088400070E080E090E00E94285180E00F900F904F
:108850000F900F900F90DF91CF910895EF92FF92BC
:108860001F93CF93DF931F92CDB7DEB77C01162FF6
:10887000FC01618172810E94E97765E070E080E02F
:1088800090E00E94285142E462E4C701BEDF412F1C
:1088900060E0C701BADF811163C040E061E0C70159
:1088A000B4DF81115DC040E062E0C701AEDF81113D
:1088B00057C046E062E0C701A8DF811151C040E027
:1088C00063E0C701A2DF81114BC040E064E0C70153
:1088D0009CDF11E0811110E040E065E0C70195DF09
:1088E000811101C01F5F40E066E0C7018EDF81118A
:1088F00001C01F5F40E067E0C70187DF811101C051
:108900001F5F40E068E0C70180DF811101C01F5F89
:1089100040E069E0C70179DF811101C01F5F44E0D9
:108920006AE0C70172DF811101C01F5F44E06AE0A5
:10893000C7016BDF811101C01F5F62E370E080E05F
:1089400090E00E94285182E8898341E050E0BE0116
:108950006F5F7F4FC70115DF81E0183011F01111F3
:1089600080E00F90DF91CF911F91FF90EF900895DD
:10897000CF93DF9300D01F92CDB7DEB72AEA2983C9
:10898000FC0120812A836B834C8344E050E0BE01CC
:108990006F5F7F4FF6DE0F900F900F900F90DF917B
:1089A000CF9108953FB7F89420E0822F90E084178C
:1089B00095079CF4FC01EE0FFF1FEB5DF24FA081C9
:1089C000B181880F991FFB01E80FF91FCD01969522
:1089D0008795918380832F5FE8CF3FBF1092161257
:1089E0000895AF92BF92CF92DF92EF92FF920F93D2
:1089F0001F93CF93DF93CDB7DEB7EDB6FEB60E94DF
:108A00004F840E9444840E949B84029709F0BBC15A
:108A10000E948684882309F4B0C1A0900F12B09000
:108A20001012C0900D12D0900E12B501C601A4DA3A
:108A30008823F1F0F601E250FE4F00E010E0819152
:108A400091918A159B0571F40E946051000F111FCE
:108A5000000F111FF601E00FF11F60837183828305
:108A6000938308C00F5F1F4F0E31110541F702C0FD
:108A70000E946F8510926A0ACDB6DEB640916D0AEB
:108A800050916E0ACA01880F991F2DB73EB7281B57
:108A9000390B0FB6F8943EBF0FBE2DBF0DB71EB7F2
:108AA0000F5F1F4F8091700A823061F0833021F197
:108AB000813009F070C0B80180911812909119129C
:108AC00071DF33C03FB7F89420E0822F90E0841725
:108AD000950774F4880F991FF801E80FF91FDC015E
:108AE000A25EBD4E8D919C91918380832F5FEDCFCF
:108AF0003FBF10923E1219C03FB7F89420E0822F7A
:108B000090E08417950774F4880F991FF801E80F17
:108B1000F91FDC01A850B34F8D919C919183808304
:108B20002F5FEDCF3FBF1092151220E06AE071E099
:108B3000822F90E040916D0A50916E0A841795073C
:108B400054F5689FF001699FF00D1124E350F04F38
:108B5000A085B1858C918823E1F0A081B1813C9101
:108B6000C801830F911D830F911DDC0112978D9118
:108B70009C91A281B3814D915C9111970480F58104
:108B8000E02D4817590711F4108203C070838D93AC
:108B90009C932F5FCDCF0FB6F894DEBE0FBECDBE37
:108BA0008091F710882321F086EF90E10E94B7842E
:108BB00080910111882321F080E091E10E94B78427
:108BC00080910B11882321F08AE091E10E94B78403
:108BD00080911511882321F084E191E10E94B784EE
:108BE00080916B0A882309F465C080910B11811173
:108BF00005C080911511882309F450C080910E1191
:108C000090910F11E0911211F09113112381348191
:108C10002817390724F48085811109C00EC02181ED
:108C200032818217930734F48085811106C088E071
:108C300090E005C080E190E002C080E290E02091E9
:108C4000181130911911E0911C11F0911D114381FF
:108C500054814217530724F42085222349F00AC087
:108C600041815281241735073CF42085222311F0DD
:108C7000816003C0846001C082602091F110309156
:108C8000F2102817390719F41092F31007C09093C7
:108C9000F2108093F11081E08093F3108091F11035
:108CA0009091F210429709F472C081E080931711FD
:108CB00080930D11EDE9F0E18EE9C82E80E1D82E08
:108CC00021EA30E141E08081882309F44AC06581CE
:108CD0007681DB0117968C91882309F442C0D60176
:108CE0008C918823F1F18281938140838A33B7E0AC
:108CF0009B0794F48C0101541640093F110570F054
:108D000007531F4F093C110558F08F579440893F76
:108D1000910540F081E007C085E005C084E003C014
:108D200083E001C082E0DB0119969C91992379F0E0
:108D3000813041F0823041F0843041F0853039F4A7
:108D400081E005C085E003C084E001C082E0D90174
:108D50009C91D601981302C01C9203C04C93D90178
:108D60008C933796B7E0CB0ED11C295F3F4F50E173
:108D7000E13FF50709F0A7CF04C00E945B840E9481
:108D80006F8581E060C00E945B8480E05CC0C09021
:108D9000F410D090F5101C141D040CF04FC08091FD
:108DA0000C1100910D1210910E126091390D7091FD
:108DB0003A0D8823A1F081E080930D11C801DCD821
:108DC000811113C0A601DD0C660B770B2DE631E88F
:108DD000C80139D990933A0D8093390D06C0C80166
:108DE000CBD8811102C010920D1180911611009103
:108DF0000D1210910E126091370D7091380D88236D
:108E0000C1F081E080931711C801B6D8811152CF0B
:108E10004091F4105091F510052E000C660B770B65
:108E20002AE631E8C8010FD99093380D8093370DA9
:108E300041CFC801A1D881113DCF02C010920D11C0
:108E40001092171137CF0FB6F894FEBE0FBEEDBECD
:108E5000DF91CF911F910F91FF90EF90DF90CF9016
:108E6000BF90AF9008951F920F920FB60F921124EA
:108E70000BB60F922F933F934F938F939F93EF9344
:108E8000FF9380918400909185002091210D309175
:108E9000220D821B930B209184003091850030932A
:108EA000220D2093210D803727E1920770F19093D6
:108EB000240D8093230D809111129091121202972C
:108EC00051F49091350D8091171298133CC081E0B8
:108ED000809316123EC08091111290911212892B2C
:108EE00049F481E090E09093121280931112109255
:108EF000200D2FC08091111290911212019761F5EF
:108F00008091350D8430D8F527C02091350D28305B
:108F100008F047C09C012C5D3540293B3B4068F47C
:108F2000E091350DEF5FE093350DF0E0EE0FFF1FA0
:108F3000ED5DF24F9183808334C080911112909146
:108F40001212029771F583E090E0909312128093D1
:108F500011121092350D25C08091111290911212AC
:108F60000397B9F79091350D809117129813F1CFAF
:108F700080911712843068F382E090E0E6CF809110
:108F8000200D8F5F8093200D863018F382E090E0F3
:108F900090931212809311128091350D80931712C5
:108FA000D8CFFF91EF919F918F914F913F912F914A
:108FB0000F900BBE0F900FBE0F901F9018950F9340
:108FC0001F938091180D81110DC00E946051609314
:108FD000140D7093150D8093160D9093170D81E06D
:108FE0008093180D0E9460510091140D1091150D81
:108FF0002091160D3091170DDC01CB01801B910BD8
:10900000A20BB30B893E9340A105B10598F08AE30A
:1090100081D7892B11F060E001C061E08AE3A2D71B
:109020000E9460516093140D7093150D8093160D7E
:109030009093170D1F910F9108950F931F930E9406
:1090400060510091EE0C1091EF0C2091F00C3091DA
:10905000F10CDC01CB01801B910BA20BB30B853310
:109060009142A105B10518F081E08093ED0C1F91AC
:109070000F91A5CFFC0180E090E06150710977FD70
:1090800018C02191022E000C330B322F2227822789
:10909000932728E0AC01440F551F97FF06C0CA0173
:1090A00031E2832730E1932701C0CA01215091F7B3
:1090B000E4CF0895BF92CF92DF92EF92FF920F9389
:1090C0001F93CF93DF93CDB7DEB76E970FB6F894AB
:1090D000DEBF0FBECDBFB62EC72ED82E7A01FA0145
:1090E0001082F801108265EA75E0CE0142962E8F5B
:1090F00082D3198E188E1B8E1A8E1D8E1C8E4AE0FE
:10910000BE016F5F7F4F8B2D90E00E9468ADBE0166
:109110006F5F7F4FCE0148961ED3BE01685E7F4FC2
:10912000CE0142965ED2CE01489635D3CE0142960C
:109130000E949785198E188E1B8E1A8E1D8E1C8E7E
:109140004AE0BE016F5F7F4FC6010E9468ADBE015D
:109150006F5F7F4FCE014896FED2BE01685E7F4FA3
:10916000CE0142969ED2CE01489615D3CE014296AC
:109170000E9497858E89F80180832E8D422F50E0C2
:10918000B701CE0142960E948E85CE01429603D34E
:109190006E960FB6F894DEBF0FBECDBFDF91CF91B4
:1091A0001F910F91FF90EF90DF90CF90BF900895A7
:1091B000FF920F931F93CF93DF93CDB7DEB7C154C8
:1091C000D1090FB6F894DEBF0FBECDBFF62E8E01CB
:1091D0000F5B1F4F20E4AE014F5F5F4F682F782F6A
:1091E00080E068DF22968FAD229791E0980F22965B
:1091F0009FAF2297E1E0F0E0EC0FFD1FE80FF11DBB
:10920000FF2011F081E301C080E3808322969FADAF
:10921000229781E0890F22968FAF2297E1E0F0E05C
:10922000EC0FFD1FE90FF11D9CE79083E1E0F0E0FA
:10923000EC0FFD1FE80FF11D1082BE016F5F7F4F25
:109240008091EB0C9091EC0C39D322966FAD229764
:1092500070E0CE0101960EDFBC018091EB0C909185
:10926000EC0C0E94A3786AE08091EB0C9091EC0CDE
:10927000FAD28091EB0C9091EC0CDC01ED91FC9119
:109280000284F385E02D1995CF5BDF4F0FB6F8947C
:10929000DEBF0FBECDBFDF91CF911F910F91FF9029
:1092A00008950895CF92DF92EF92FF920F931F934C
:1092B000CF93DF936C017A018B01C0E0D0E0CE1533
:1092C000DF0589F0D8016D918D01D601ED91FC91FA
:1092D0000190F081E02DC6011995892B11F47E01D2
:1092E00002C02196ECCFC701DF91CF911F910F9162
:1092F000FF90EF90DF90CF900895FC01A089B18995
:109300008C91A689B78982FD0FC09C91818D8F5F5A
:109310008F73228D821749F0218DDF01A20FB11DBD
:109320005D969C93818F08958C910895FC01918D99
:10933000828D981761F0828DDF01A80FB11D5D96B7
:109340008C91928D9F5F9F73928F90E008958FEF25
:109350009FEF0895FC01918D828D981731F0828DD9
:10936000E80FF11D858D90E008958FEF9FEF089530
:10937000FC01918D228D892F90E0805C9F4F821B94
:1093800091098F739927089582EB96E0F1DF21E030
:10939000892B09F420E0822F08958FE497E0E8DF1D
:1093A00021E0892B09F420E0822F08958CEE97E0CC
:1093B000DFDF21E0892B09F420E0822F089589E87E
:1093C00098E0D6DF21E0892B09F420E0822F089570
:1093D000FC01848DDF01A80FB11DA35ABF4F2C9152
:1093E000848D90E001968F739927848FA689B78921
:1093F0002C93A089B1898C9180648C93938D848DFA
:10940000981306C00288F389E02D80818F7D8083C8
:109410000895EF92FF920F931F93CF93DF93EC0188
:1094200081E0888F9B8D8C8D981305C0E889F98920
:10943000808185FD23C0F62E0B8D10E00F5F1F4F3E
:109440000F731127E02E8C8DE8120BC00FB607FCAE
:10945000FACFE889F989808185FFF5CFCE01B8DFA1
:10946000F2CF8B8DFE01E80FF11DE35AFF4FF08222
:109470000B8FEA89FB898081806207C0EE89FF89B2
:109480006083E889F98980818064808381E090E04D
:10949000DF91CF911F910F91FF90EF900895CF939F
:1094A000DF93EC01888D8823C1F0EA89FB898081F4
:1094B00085FD05C0A889B9898C9186FD0EC00FB6BF
:1094C00007FCF5CF808185FFF2CFA889B9898C91FF
:1094D00085FFEDCFCE017CDFE8CFDF91CF910895FE
:1094E00080E090E0892B19F06ADF811116C080E0DE
:1094F00090E0892B19F05ADF811112C080E090E0D2
:10950000892B19F04ADF81110EC080E090E0892B91
:1095100079F03ADF81110AC008950E940000E7CF78
:109520000E940000EBCF0E940000EFCF0C940000DF
:10953000089590E0FC013197E231F10508F04EC04A
:109540008827EE5CFE4F8F4F0C9477A980918000A6
:109550008F7703C0809180008F7D80938000089575
:1095600080918000877FF9CF84B58F7702C084B562
:109570008F7D84BD08958091B0008F7703C0809166
:10958000B0008F7D8093B0000895809190008F7718
:1095900007C0809190008F7D03C080919000877FED
:1095A0008093900008958091A0008F7707C08091EC
:1095B000A0008F7D03C08091A000877F8093A000D2
:1095C0000895809120018F7707C0809120018F7DC1
:1095D00003C080912001877F8093200108950E941D
:1095E000A2AC0F931F93CF93DF938C01EB01FC018F
:1095F000808191810097B1F0688179816115710551
:1096000079F0428153812C813D814217530740F00C
:109610000E94BAAC8C819D81F8019583848313C02C
:109620000E9426AB88819981F801918380838A8189
:109630009B81938382838C819D819583848319820E
:1096400018821B821A821D821C82DF91CF911F918A
:109650000F9108950F931F93CF93DF93EC018881AF
:109660009981009729F02A813B812617370788F4D2
:109670008B016F5F7F4F0E94BEAB009761F09983B3
:1096800088831B830A832C813D81232B11F4FC01E9
:10969000108281E001C080E0DF91CF911F910F9196
:1096A0000895EF92FF920F931F93CF93DF93FB01E7
:1096B00024813581E080F180FC0104811581E11471
:1096C000F10411F480E016C02115310591F0EC0190
:1096D000020F131FB801BEDF8823A1F3288139814F
:1096E0008C819D81B701820F931F0E94BAAC1D83AC
:1096F0000C8381E0DF91CF911F910F91FF90EF904C
:109700000895EF92FF920F931F93CF93DF93EC0195
:109710007B018A01BA019EDF2881398181110DC048
:109720002115310519F0C9010E9426AB1982188252
:109730001D821C821B821A8206C01D830C83B70106
:10974000C9010E94BAACCE01DF91CF911F910F9158
:10975000FF90EF900895CF93DF93EC0161157105B1
:1097600051F0FB0101900020E9F73197AF01461B52
:10977000570BC7DF0CC088819981009711F00E94B8
:1097800026AB198218821D821C821B821A82CE018E
:10979000DF91CF910895FC01808191810C9426ABDB
:1097A0000F931F93CF93DF93CDB7DEB762970FB6BA
:1097B000F894DEBF0FBECDBF8C01CB01F801118242
:1097C0001082138212821582148250E0BE016F5FF4
:1097D0007F4F0E9425ADBE016F5F7F4FC801BBDF89
:1097E00062960FB6F894DEBF0FBECDBFDF91CF916A
:1097F0001F910F910895FC01118210821382128231
:10980000158214826115710549F0FB010190002059
:10981000E9F73197AF01461B570B73CF0895CF93EC
:10982000DF9300D01F92CDB7DEB7611571058105BA
:10983000910579F09B01AC0169833A834B835C838A
:109840000E9419AD29813A814B815C810E94DAAE78
:1098500003C060E070E0CB010F900F900F900F906D
:10986000DF91CF910895DC01ED91FC910190F081A1
:10987000E02D1994EF92FF920F931F93CF93DF93F4
:109880008C017B01C0E0D0E0F701EC0FFD1F64917B
:10989000662361F0D801ED91FC910190F081E02DFB
:1098A000C8011995892B11F02196EECFCE01DF91D9
:1098B000CF911F910F91FF90EF9008956115710561
:1098C00079F0FB0101900020E9F73197AF01461BC9
:1098D000570BDC01ED91FC910280F381E02D19948E
:1098E00080E090E008954F925F926F927F92EF92A6
:1098F000FF920F931F93CF93DF93CDB7DEB7A1975E
:109900000FB6F894DEBF0FBECDBF7C01FA01CB01CC
:1099100019A2223008F42AE08E010F5D1F4F422E5B
:10992000512C612C712CBF01A30192010E9406AF42
:10993000F901CA01015011096A3014F4605D01C0D7
:10994000695CD8016C93232B242B252B61F7B8017C
:10995000C701B4DFA1960FB6F894DEBF0FBECDBF2E
:10996000DF91CF911F910F91FF90EF907F906F90BB
:109970005F904F9008954F925F926F927F928F9277
:109980009F92AF92BF92CF92DF92EF92FF92CF93CE
:10999000DF93EC016A017B01B22E9A01AB01C70192
:1099A000B6010E948DAA882319F067E975E027C0E7
:1099B00026013701E89477F82FEF3FEF4FE75FE795
:1099C000C301B2010E948DAA81110DC02FEF3FEF9C
:1099D0004FE75FE7C301B2010E9491AD18161CF476
:1099E0006BE975E00CC02FEF3FEF4FE75FE4C70175
:1099F000B6010E9489AA181694F46FE975E0CE01A9
:109A0000DF91CF91FF90EF90DF90CF90BF90AF901C
:109A10009F908F907F906F905F904F904FCF2FEFE0
:109A20003FEF4FE75FECC701B6010E9491AD87FDA4
:109A3000E4CF20E030E0A901C701B6010E9491AD5A
:109A400087FF09C06DE2CE010EDF4C01F7FAF094FA
:109A5000F7F8F09402C0812C912CA12C60E070E00A
:109A600080E09FE3AB1441F020E030E040E251E4BD
:109A70000E94F0A9A394F6CF9B01AC01C701B601E7
:109A80000E948CA92B013C010E945DAA6B017C0104
:109A90000E9495AD9B01AC01C301B2010E948BA94C
:109AA0002B013C012AE0B701A601CE011CDF7C019D
:109AB000E80CF91CBB2029F06EE2CE01D4DEE80EE2
:109AC000F91EDB2CDD2021F120E030E040E251E402
:109AD000C301B2010E94F6AD2B013C010E945DAAB8
:109AE0004B01A12CB12C2AE0B501A401CE01FBDE73
:109AF000E80EF91EC501B4010E9495AD9B01AC01B1
:109B0000C301B2010E948BA92B013C01DA94DACF88
:109B1000C701DF91CF91FF90EF90DF90CF90BF9082
:109B2000AF909F908F907F906F905F904F9008952F
:109B300063EA75E0C3CE0F931F93CF93DF93EC01DD
:109B4000BDDE8C01CE01F4DF800F911FDF91CF913C
:109B50001F910F9108950F931F93CF93DF93EC0103
:109B600089DE8C01CE01E4DF800F911FDF91CF9160
:109B70001F910F9108951F920F920FB60F9211240B
:109B80000BB60F922F933F934F935F936F937F93F7
:109B90008F939F93AF93BF93EF93FF9382EB96E0E6
:109BA00017DCFF91EF91BF91AF919F918F917F91C2
:109BB0006F915F914F913F912F910F900BBE0F903E
:109BC0000FBE0F901F9018951F920F920FB60F9215
:109BD00011240BB60F922F933F934F935F936F9384
:109BE0007F938F939F93AF93BF93EF93FF9382EBFA
:109BF00096E083DBFF91EF91BF91AF919F918F91A1
:109C00007F916F915F914F913F912F910F900BBE7C
:109C10000F900FBE0F901F9018951F920F920FB6C6
:109C20000F9211240BB60F922F933F934F935F9394
:109C30006F937F938F939F93AF93BF93EF93FF9314
:109C40008FE497E0C5DBFF91EF91BF91AF919F91BA
:109C50008F917F916F915F914F913F912F910F90D5
:109C60000BBE0F900FBE0F901F9018951F920F9272
:109C70000FB60F9211240BB60F922F933F934F9371
:109C80005F936F937F938F939F93AF93BF93EF9364
:109C9000FF938FE497E031DBFF91EF91BF91AF919C
:109CA0009F918F917F916F915F914F913F912F91F4
:109CB0000F900BBE0F900FBE0F901F9018951F9224
:109CC0000F920FB60F9211240BB60F922F933F9362
:109CD0004F935F936F937F938F939F93AF93BF93B4
:109CE000EF93FF938CEE97E073DBFF91EF91BF91C1
:109CF000AF919F918F917F916F915F914F913F9124
:109D00002F910F900BBE0F900FBE0F901F901895C4
:109D10001F920F920FB60F9211240BB60F922F9332
:109D20003F934F935F936F937F938F939F93AF93E3
:109D3000BF93EF93FF938CEE97E0DFDAFF91EF9103
:109D4000BF91AF919F918F917F916F915F914F9153
:109D50003F912F910F900BBE0F900FBE0F901F9051
:109D600018951F920F920FB60F9211240BB60F92F7
:109D70002F933F934F935F936F937F938F939F9313
:109D8000AF93BF93EF93FF9389E898E021DBFF91B6
:109D9000EF91BF91AF919F918F917F916F915F9163
:109DA0004F913F912F910F900BBE0F900FBE0F90D0
:109DB0001F9018951F920F920FB60F9211240BB699
:109DC0000F922F933F934F935F936F937F938F9354
:109DD0009F93AF93BF93EF93FF9389E898E08DDA59
:109DE000FF91EF91BF91AF919F918F917F916F9173
:109DF0005F914F913F912F910F900BBE0F900FBE2F
:109E00000F901F901895CF93DF93EC01E881F981B3
:109E10000284F385E02D1995EA89FB8980818F7E84
:109E20008083EA89FB898081877F8083EA89FB8937
:109E300080818F778083EA89FB8980818F7D808311
:109E40008A8D898FDF91CF910895CF92DF92EF9223
:109E5000FF921F93CF93DF93EC016A017B01122FD6
:109E6000E889F98982E080834115514E61057105C9
:109E7000B1F060E079E08DE390E0A70196010E94E7
:109E800006AFDA01C9010197A109B109B695A795F5
:109E900097958795AC01411580E15807A8F0E889AE
:109EA000F989108260E874E88EE190E0A7019601DC
:109EB0000E9406AFBA01A901415051096109710917
:109EC0007695679557954795EC85FD855083EE858A
:109ED000FF854083188EEC89FD891083EA89FB8910
:109EE000808180618083EA89FB89808188608083AA
:109EF000EA89FB89808180688083EA89FB89808187
:109F00008F7D8083DF91CF911F91FF90EF90DF9045
:109F1000CF900895CF93DF93282F30E0F901EF58C9
:109F2000FF4E8491F901E55DFF4ED491F901EB51AB
:109F3000F04FC491CC2389F08111FBDAEC2FF0E0D3
:109F4000EE0FFF1FE553F04FA591B491EC91ED2377
:109F500081E090E021F480E002C080E090E0DF91B9
:109F6000CF9108951F93CF93DF93282F30E0F9010D
:109F7000EF58FF4E8491F901E55DFF4ED491F90150
:109F8000EB51F04FC491CC23C1F0162F8111D1DADF
:109F9000EC2FF0E0EE0FFF1FEF54F04FA591B491BE
:109FA0008FB7F894111105C09C91ED2FE095E9232E
:109FB00002C0EC91ED2BEC938FBFDF91CF911F91FD
:109FC0000895CF93DF9390E0FC01E55DFF4E24916F
:109FD000FC01EB51F04F8491882361F190E0880FF0
:109FE000991FFC01E956F04FC591D491FC01EF5443
:109FF000F04FA591B491611109C09FB7F894888181
:10A00000209582238883EC912E230BC0623061F46B
:10A010009FB7F8943881822F809583238883EC91B1
:10A020002E2B2C939FBF06C08FB7F894E8812E2B60
:10A0300028838FBFDF91CF9108951F93CF93DF9334
:10A04000182FEB0161E0BDDF209711F460E004C040
:10A05000CF3FD10531F461E0812FDF91CF911F9186
:10A0600081CFE12FF0E0EF58FF4EE4914E2F50E00A
:10A07000FA013197E231F10508F09DC08827EC5BC9
:10A08000FE4F8F4F0C9477A984B5806884BDC7BDFF
:10A0900097C084B5806284BDC8BD92C080918000A5
:10A0A000806880938000D0938900C093880088C026
:10A0B00080918000806280938000D0938B00C09359
:10A0C0008A007EC080918000886080938000D09359
:10A0D0008D00C0938C0074C08091B0008068809324
:10A0E000B000C093B3006CC08091B00080628093D8
:10A0F000B000C093B40064C08091900080688093E9
:10A100009000D0939900C09398005AC0809190001D
:10A11000806280939000D0939B00C0939A0050C0BF
:10A1200080919000886080939000D0939D00C093B0
:10A130009C0046C08091A00080688093A000809120
:10A14000A0008F7B8093A000D093A900C093A800AB
:10A1500037C08091A00080628093A000D093AB00B4
:10A16000C093AA002DC08091A00088608093A000B9
:10A17000D093AD00C093AC0023C0809120018068D3
:10A1800080932001D0932901C093280119C08091A8
:10A190002001806280932001D0932B01C0932A017B
:10A1A0000FC080912001886080932001D0932D0101
:10A1B000C0932C0105C0C038D1050CF04CCF46CF60
:10A1C000DF91CF911F910895863308F086539091C7
:10A1D0007B00282F2870977F922B90937B008770AD
:10A1E000806480937C0080917A00806480937A0000
:10A1F00080917A0086FDFCCF8091780020917900D3
:10A2000090E0922B08953FB7F89480913F0D909184
:10A21000400DA091410DB091420D26B5A89B05C0FF
:10A220002F3F19F00196A11DB11D3FBFBA2FA92FD5
:10A23000982F8827820F911DA11DB11DBC01CD0152
:10A2400042E0660F771F881F991F4A95D1F708953E
:10A250008F929F92AF92BF92CF92DF92EF92FF9236
:10A260006B017C01D0DF4B015C01C114D104E1041E
:10A27000F104E9F0C8DFDC01CB0188199909AA09CA
:10A28000BB09883E9340A105B10578F321E0C21ACD
:10A29000D108E108F10888EE880E83E0981EA11C21
:10A2A000B11CC114D104E104F10421F7DECFFF9009
:10A2B000EF90DF90CF90BF90AF909F908F900895D8
:10A2C0002FB7F89460913B0D70913C0D80913D0D3E
:10A2D00090913E0D2FBF0895089508950895089513
:10A2E0001092550A08950F931F93CF93DF93EC01BB
:10A2F0001F8A1E8A8C01075E1F4F40E060E0C80184
:10A300000E94148340E064E0C8010E941483D8DFF7
:10A310006C8F7D8F8E8F9F8FDF91CF911F910F91CB
:10A3200008950F931F93CF93DF93EC018091430D1A
:10A33000811112C00A8D1B8D6AEA70E0C8010E946B
:10A34000206AD801ED91FC910284F385E02DC801CB
:10A35000199581E08093430D4AE06EE0CE01499665
:10A360000E94148321E83FEF3B872A878FE790E024
:10A370009D878C871F861E86398B288B9B8B8A8BAB
:10A380001D8A1C8ADF91CF911F910F9108950F9321
:10A390001F93CF93DF93EC011F8A1E8A8C01075E07
:10A3A0001F4F40E060E0C8010E94D78240E064E0B7
:10A3B000C8010E94D78284DF6C8F7D8F8E8F9F8F24
:10A3C000DF91CF911F910F9108950F931F93CF931A
:10A3D000DF93EC01E8A1F9A180819181A281B38191
:10A3E0008E01075E1F4F81159649A105B10509F43D
:10A3F0004FC040E056E960E070E08FE497E00E94D3
:10A40000926C64E170E080E090E022DFE8A1F9A1C5
:10A4100080819181A281B38181152BE49207A105EE
:10A42000B105E9F068F4803629E09207A105B1058D
:10A43000A1F080389542A105B105C1F442E012C0F7
:10A44000811521EE9207A105B10559F08115924CB5
:10A45000A140B10559F445E005C041E003C043E027
:10A4600001C046E06FE0C8010E94D7828FE497E008
:10A4700016D8E8A1F9A140815181628173818FE4EE
:10A4800097E00E94926C64E170E080E090E0E0DE92
:10A490004AE06EE0C8010E94D78241E067E1C8014E
:10A4A0000E94D7824AA168E1C8010E94D78221E8B0
:10A4B0003FEF3B872A878FE790E09D878C871F8639
:10A4C0001E86398B288B9B8B8A8B1D8A1C8ADF9179
:10A4D000CF911F910F9108950C94276ACF93DF932A
:10A4E000C7EED9E081E090E09A8389831092550A03
:10A4F0008ADE6C837D838E839F83E49AEC9ADF915E
:10A50000CF910895EF92FF920F931F93CF93DF9314
:10A51000EC016623E1F0262F653608F024E60A896F
:10A520001B89E888F988D801AE19BF0930E00E947C
:10A5300085A928EC30E040E050E00E9406AFE20E32
:10A54000F31EFB86EA86021B130B1D870C87DF9127
:10A55000CF911F910F91FF90EF900895CF93DF93CC
:10A56000CDB7DEB7A2970FB6F894DEBF0FBECDBF52
:10A5700080310CF080E126E731E13A8329832EE631
:10A5800031E13C832B8326E631E13E832D832EE5AA
:10A5900031E138872F8326E531E13A8729872EE498
:10A5A00031E13C872B8726E431E13E872D872EE37E
:10A5B00031E1388B2F8720E331E13A8B298B2EE173
:10A5C00031E13C8B2B8B21E031E13E8B2D8B2CEE4E
:10A5D00030E1388F2F8B22EE30E13A8F298F28ED32
:10A5E00030E13C8F2B8F2BEC30E13E8F2D8F2FEB0A
:10A5F00030E138A32F8F27EB30E13AA329A3E82FCE
:10A60000EE0FFF0BEC0FFD1F81819281A2960FB61A
:10A61000F894DEBF0FBECDBFDF91CF9108958F922A
:10A620009F92AF92BF92CF92DF92EF92FF920F93E1
:10A630001F93DC0118968D919C9119971E96CD90D1
:10A64000DC901F976817790709F456C05896FC905C
:10A6500058974C01092E000CAA08BB088B01072E45
:10A66000000C220B330B861797073CF41696ED91DE
:10A67000FC911797FF2039F015C01496ED91FC91CD
:10A680001597FF2079F00D2C000CEE08FF08A901AA
:10A690009801281939094A095B091C966D917C912A
:10A6A0001D970EC00D2C000CEE08FF08A9019801A3
:10A6B000281939094A095B091A966D917C911B97F3
:10A6C000CB01770FAA0BBB0BBC01CD016C197D0927
:10A6D0008E099F090E9441A98F01FF0F220B330BA6
:10A6E000A9019801281939094A095B090E94DAAEC3
:10A6F000C20ED31EE41EF51EC6011F910F91FF90DE
:10A70000EF90DF90CF90BF90AF909F908F90089583
:10A71000CF93DF93EC017F8B6E8B81DF9C018A816D
:10A720009B8188309105C1F437FF06C061E0213874
:10A730008FEF38074CF001C060E0A90120383105E7
:10A740002CF04FE750E002C041E85FEF57FF1FC019
:10A750005195419551091BC00997E9F4922F832F18
:10A760002038310514F09FE780E0492F582F4138F9
:10A770008FEF580714F441E85FEF57FF03C051957E
:10A7800041955109632F661F6627661F6C5FCE01D6
:10A7900049960E94148394DD6C8F7D8F8E8F9F8FDE
:10A7A000DF91CF910895CF93DF93EC017F8B6E8B78
:10A7B00036DF9C018A819B8188309105C1F437FF87
:10A7C00006C061E021388FEF38074CF001C060E02F
:10A7D000A901203831052CF04FE750E002C041E8D4
:10A7E0005FEF57FF1FC05195419551091BC0099755
:10A7F000E9F4922F832F2038310514F09FE780E091
:10A80000492F582F41388FEF580714F441E85FEF74
:10A8100057FF03C0519541955109632F661F662765
:10A82000661F6C5FCE0149960E94D78249DD6C8F0E
:10A830007D8F8E8F9F8FDF91CF9108950F931F9300
:10A84000CF93DF93EC013CDD0C8D1D8D2E8D3F8D64
:10A85000DC01CB01801B910BA20BB30B853F914018
:10A86000A105B10540F06E897F89CE01DF91CF91BE
:10A870001F910F9198CFDF91CF911F910F91089564
:10A88000CF93DF93EC0161E089E09BDB60E089E03E
:10A8900069DB1092930987EF94E099838883DF91B5
:10A8A000CF910895CF92DF92EF92FF928091940919
:10A8B000833009F061C0809195098130D1F488EE30
:10A8C00093E0A0E0B0E08093260990932709A0933D
:10A8D0002809B093290980E797E1A0E0B0E08093D0
:10A8E0002A0990932B09A0932C09B0932D0932E0EB
:10A8F00001C030E0E0919509F0E0EA56F64F208182
:10A90000A0E1A30F48EE53E060E070E088EBC82EB2
:10A910008BE0D82EE12CF12C832F90E0FC01EE0F80
:10A92000FF1FEE0FFF1FEA5DF64F27FF10C0C0822A
:10A93000D182E282F382880F991F880F991FFC0150
:10A94000E65DF64F40835183628373830FC040837B
:10A95000518362837383880F991F880F991FFC01AD
:10A96000E65DF64FC082D182E282F3823E5F220F23
:10A970003A13D2CF30938F09FF90EF90DF90CF90B2
:10A980000895CF93DF9380919309811151C0109264
:10A99000910910928E09C1E0C0939309D091920958
:10A9A00061E089E00EDB60E089E0DCDA2D2F30E049
:10A9B00040E050E060E47FE180E090E00E94DAAEA9
:10A9C000C093B00089E08093B1002093B3008BEA7C
:10A9D000289F212D112426952093B40080916F008B
:10A9E0008B7F80936F008091B00080628093B00075
:10A9F0002091840030918500E0918E0981E08E0FD6
:10AA000080938E0984E0E89FF0011124EA5DF64FFF
:10AA100080819181A281B381820F931F90938B00DB
:10AA200080938A00B29A80916F00846080936F0057
:10AA3000DF91CF9108954F925F926F927F928F92A4
:10AA40009F92AF92BF92CF92DF92EF92FF928AE1F4
:10AA500080938F092093900988E28093920981E086
:10AA600080939509809396098EE08093940980ECF9
:10AA700092E1A0E0B0E08093260990932709A0938B
:10AA80002809B093290980EB94E0A0E0B0E080931E
:10AA90002A0990932B09A0932C09B0932D09A4E1C6
:10AAA000440F551F661F771FAA95D1F722E030E0AB
:10AAB000B0EBCB2EB4E0DB2EE12CF12C80E6482E5F
:10AAC00089E0582E612C712C90E4892E9CE9992EF6
:10AAD000A12CB12CC901880F991F880F991FFC0167
:10AAE000EA5DF64F77FF05C0408251826282738231
:10AAF00004C0C082D182E282F382C9010196880F2C
:10AB0000991F880F991FFC01EA5DF64F283129F043
:10AB1000C082D182E282F38204C080829182A282CA
:10AB2000B382440F551F661F771F2E5F3F4F2A3198
:10AB3000310581F6FF90EF90DF90CF90BF90AF90FE
:10AB40009F908F907F906F905F904F901ACF8F92D1
:10AB50009F92AF92BF92CF92DF92EF92FF9282E1EB
:10AB600080938F0986E08093900996E290939209F2
:10AB700091E090939509909396098093940988EDBC
:10AB800090E4A0E0B0E08093260990932709A09379
:10AB90002809B09329098CE19CE0A0E0B0E0809303
:10ABA0002A0990932B09A0932C09B0932D09742F97
:10ABB00066275527442722E030E0ACE1CA2EACE0FE
:10ABC000DA2EE12CF12CB8E38B2EB8E19B2EA12CD0
:10ABD000B12CC901880F991F880F991FFC01EA5DEC
:10ABE000F64F77FF05C080829182A282B38204C0B3
:10ABF000C082D182E282F382F901EE0FFF1FEE0FD5
:10AC0000FF1FE65DF64FC082D182E282F382440FDD
:10AC1000551F661F771F2E5F3F4F22313105C9F642
:10AC20008CE199E8A0E0B0E080936A0990936B0909
:10AC3000A0936C09B0936D09FF90EF90DF90CF90D7
:10AC4000BF90AF909F908F909CCE1F920F920FB6A7
:10AC50000F9211240BB60F922F933F934F935F9354
:10AC60006F937F938F939F93AF93BF93EF93FF93D4
:10AC700090918E0980918F09981316C010928E09B9
:10AC8000809195098F5F80939509909195098091A6
:10AC90009609891740F481E0809395098091910984
:10ACA0008F5F80939109FEDD9091910980919009C9
:10ACB00098130DC08091B0008F7D8093B00080917B
:10ACC0006F008B7F80936F001092930927C0809153
:10ACD000B00085FF04C08091B0008F7D03C08091DB
:10ACE000B00080628093B000209184003091850094
:10ACF000E0918E0981E08E0F80938E0984E0E89FB9
:10AD0000F0011124EA5DF64F80819181A281B38127
:10AD1000820F931F90938B0080938A00FF91EF9195
:10AD2000BF91AF919F918F917F916F915F914F9163
:10AD30003F912F910F900BBE0F900FBE0F901F9061
:10AD400018951F920F920FB60F9211240BB60F9207
:10AD50001F932F933F934F935F936F937F938F93A3
:10AD60009F93AF93BF93EF93FF93CF93DF9300D065
:10AD70001F92CDB7DEB78091E709CCD811E0892BBF
:10AD800009F010E040DA69837A838B839C838981A0
:10AD90009A81AB81BC814091EB095091EC096091A3
:10ADA000ED097091EE09841B950BA60BB70B209152
:10ADB000E8093091E9092430310509F44CC0253007
:10ADC000310521F021303105E9F414C02091EA0960
:10ADD000222339F02091550A20FF02C0289A01C091
:10ADE0002898112379F0813E2EE29207A105B10542
:10ADF00048F02BC0112379F125E030E03093E909C8
:10AE00002093E8092091E8093091E90925303105BE
:10AE100011F5E091550AF0E0EE0FFF1FE151F64FFA
:10AE20009183808389819A81AB81BC818093EB0976
:10AE30009093EC09A093ED09B093EE098091550A27
:10AE40008F5F8093550A833330F084E090E09093D5
:10AE5000E9098093E8090F900F900F900F90DF9110
:10AE6000CF91FF91EF91BF91AF919F918F917F9182
:10AE70006F915F914F913F912F911F910F900BBE5A
:10AE80000F900FBE0F901F901895CF93C091510D4A
:10AE90006C2F70E088E0D1D889E18093500D9091BB
:10AEA0000E02992311F0CD5F01C0C350C093510D24
:10AEB0008091510D873970F0992321F08FEF8093A5
:10AEC000510D08C08D3D30F086E98093510D88E723
:10AED0008093500D8091510D8F3F19F410920E0206
:10AEE00005C08A3118F481E080930E024091500D24
:10AEF00050E060E070E025E437E585E89AE00E94E4
:10AF000023409093E2118093E111CF910895CF9265
:10AF1000DF92EF92FF92CF93DF93EC019C01AFEFB2
:10AF2000B0E00E9428AFCC24CA9423E0D22EE12CBA
:10AF3000F12CA70196010E94DAAEB90188E07DD814
:10AF40009E01A4E6B0E00E9428AFA70196010E94EE
:10AF5000DAAE8091F20F82132093F20FDF91CF913E
:10AF6000FF90EF90DF90CF90089561E088E00E941D
:10AF7000B24F80915506882361F08091E3118111D1
:10AF800008C067E773E180915306909154060C94D2
:10AF9000AB4D0895CF9380914D0D81110FC081E08D
:10AFA00080934D0D80915506882341F065E473E14F
:10AFB00080915306909154060E94AB4DC0914C0D68
:10AFC0006C2F85E00E94B24F4091F70F50E060E097
:10AFD00070E02AEC37E585E89AE00E9423409093E0
:10AFE0004B0D80934A0D81E06C2F682760934C0DC8
:10AFF000CF9108958091070180FF12C060E08EE339
:10B000000E94B24F1092EC0580915506882341F0C2
:10B010006CEB72E180915306909154060C94AB4D09
:10B0200008958091070180FF13C061E08EE30E94C4
:10B03000B24F81E08093EC0580915506882341F062
:10B0400066EA72E180915306909154060C94AB4DE0
:10B0500008958091070181FF12C060E08FE30E9494
:10B06000B24F1092E50580915506882341F06FE8B4
:10B0700072E180915306909154060C94AB4D089563
:10B080008091070181FF13C061E08FE30E94B24FFE
:10B0900081E08093E50580915506882341F069E7BA
:10B0A00072E180915306909154060C94AB4D089533
:10B0B0008091B205882371F01092B20580915506F7
:10B0C000882341F061EF71E180915306909154061D
:10B0D0000C94AB4D08958091890F833099F0809145
:10B0E000B20581110FC081E08093B20580915506B1
:10B0F000882341F06CED71E18091530690915406E4
:10B100000C94AB4D08958091B205882319F080E02E
:10B1100090E0CECF80E090E0DECF8091B10583302B
:10B1200079F083E08093B10580915506882341F042
:10B130006BEC71E180915306909154060C94AB4DE9
:10B1400008958091B105823079F082E08093B10555
:10B1500080915506882341F06AEB71E18091530696
:10B16000909154060C94AB4D08958091B1058130B7
:10B1700079F081E08093B10580915506882341F0F4
:10B1800069EA71E180915306909154060C94AB4D9D
:10B190000895CF93DF93C091E111D091E211BE01E8
:10B1A00085E89AE00E94BC3F882329F0BE0185E82B
:10B1B0009AE00E94D43F60E088E00E94B24F809104
:10B1C00055068823D1F08091E311882319F06DEAA8
:10B1D00073E10DC08091E011882319F064E973E1F7
:10B1E00006C08091D40C811108C065E873E180919C
:10B1F0005306909154060E94AB4D1092E3111092A9
:10B20000E011DF91CF9108958091E311811110C079
:10B21000C0DF81E08093E31180915506882341F0DF
:10B2200066EC73E180915306909154060E94AB4DF9
:10B2300080914F0D882329F060E088E00E94B24F92
:10B2400001C093DE90914F0D81E0892780934F0DCF
:10B25000882329F04091EE0F5091EF0F04C04091E8
:10B26000F00F5091F10F60E070E024E039E585E8DF
:10B270009AE00E9423409093E2118093E111089597
:10B280000E94727F8091B305882361F180915A0AF0
:10B29000811128C080914B06811124C081E08093E8
:10B2A0004B060E94938D8091DE05882319F0109241
:10B2B000DE050CC080914F0690915006DC01ED91A7
:10B2C000FC910088F189E02D61E019958091550687
:10B2D000882341F06EE771E1809153069091540606
:10B2E0000C94AB4D089560E089E30C94B24F61E09B
:10B2F00089E30C94B24F10924E0D8091410681115A
:10B3000004C060E084E00E94B24F8091550688231B
:10B3100041F064E673E180915306909154060C94D9
:10B32000AB4D089581E080934E0D809141068111CF
:10B3300006C06091450D70E084E00E941D50809130
:10B340005506882341F062E573E1809153069091A0
:10B3500054060C94AB4D08951092410680914E0D09
:10B36000811104C060E084E00C94B24F6091450DFF
:10B3700070E084E00C941D50CF93DF9360E085E093
:10B380000E94B24FC0914A0DD0914B0DBE0185E88D
:10B390009AE00E94BC3F882329F0BE0185E89AE02C
:10B3A0000E94D43F80915506882379F020914D0D5D
:10B3B0008091530690915406222319F069E373E1BA
:10B3C00002C06DE273E10E94AB4D10924D0DDF9112
:10B3D000CF91089561E085E00E94B24F80915506BB
:10B3E000882341F062E273E1809153069091540604
:10B3F0000C94AB4D089560E085E30E94B24F8091BC
:10B400004F0690915006DC01ED91FC9104A8F5A93E
:10B41000E02D199580915506882341F066E173E18E
:10B4200080915306909154060C94AB4D089561E0C1
:10B4300085E30E94B24F80914F0690915006DC0147
:10B44000ED91FC9104A8F5A9E02D19958091550680
:10B45000882341F06BE073E180915306909154068C
:10B460000C94AB4D08958F929F92AF92BF92CF9262
:10B47000DF92EF92FF9285E40E94E450BC01990FA5
:10B48000880B990B0E9497AD20E030E040E85AE32A
:10B490000E94F6AD20E030E040EA50E40E94F6ADB4
:10B4A0006B017C0180910D02882351F0C092460D02
:10B4B000D092470DE092480DF092490D10920D0286
:10B4C00026E636E646E65FE36091460D7091470D4D
:10B4D0008091480D9091490D0E94F6AD4B015C01A1
:10B4E00020ED3CEC4CEC5DE3C701B6010E94F6ADEB
:10B4F0009B01AC01C501B4010E948CA96093460D6B
:10B500007093470D8093480D9093490D2DE33CE2D5
:10B5100048E450E40E94F6AD2AE939E949E95EE3DE
:10B520000E948CA9FF90EF90DF90CF90BF90AF90DA
:10B530009F908F900895CF93DF938091070180FDB6
:10B540002AC0C091E905D091EA058091EE058823D3
:10B5500071F08EE30E94E450813092402CF0109202
:10B56000EA051092E9050AC081E090E003C08EE38D
:10B570000E94E4509093EA058093E9058091E905E3
:10B580009091EA058C179D0719F41092EB0503C002
:10B5900081E08093EB05DF91CF910895CF93DF9306
:10B5A0008091070181FD2AC0C091E205D091E30599
:10B5B0008091E705882371F08FE30E94E450813089
:10B5C00092402CF01092E3051092E2050AC081E04F
:10B5D00090E003C08FE30E94E4509093E3058093D2
:10B5E000E2058091E2059091E3058C179D0719F41F
:10B5F0001092E40503C081E08093E405DF91CF91D0
:10B600000895909155068823D9F08091B10688233A
:10B61000B9F081E080939B0F8093440D992311F141
:10B6200068E472E180915306909154060E943A4C6E
:10B630000E94628080915306909154060C94984D1C
:10B6400010929B0F992341F060E672E180915306BE
:10B65000909154060E94AB4D8091990F811102C0C8
:10B660001092440D0895909155068823F9F0809129
:10B67000B1068823D9F080914F0F8D30B9F481E065
:10B680008093990F8093440D992311F167E072E143
:10B6900080915306909154060E943A4C0E948E80ED
:10B6A00080915306909154060C94984D1092990FE6
:10B6B000992341F067E272E180915306909154061C
:10B6C0000E94AB4D80919B0F811102C01092440DDE
:10B6D00008958091890F8230C1F01CF48130A9F067
:10B6E0002FC0833011F1843059F580914406909138
:10B6F0004506DC01ED91FC910480F581E02D199562
:10B70000809142069091430614C080914806909122
:10B710004906DC01ED91FC910480F581E02D19953D
:10B72000809146069091470604C08091440690910E
:10B730004506DC01ED91FC910480F581E02D199521
:10B7400080914F0690915006DC01ED91FC91E05CF8
:10B75000FF4F0190F081E02D199580914F06909157
:10B760005006DC01ED91FC910284F385E02D60E050
:10B7700070E01994AEDF80914F0690915006DC0185
:10B78000ED91FC910084F185E02D199580914F0693
:10B7900090915006DC01ED91FC910480F581E02D43
:10B7A00019950E9447740E94727F8091B3058111A0
:10B7B0000E94BF8A8091510690915206DC01ED9162
:10B7C000FC910480F581E02D199580914D069091B2
:10B7D0004E06DC01ED91FC910480F581E02D199578
:10B7E00080916A0F882359F08091DC059091DD05E6
:10B7F000DC01ED91FC910480F581E02D1994089510
:10B8000080910C02882351F02EDE20E030E040E0F1
:10B8100050E40E9491AD87FF39C0089524DE20E0F6
:10B8200030E04AE754E40E94F6AD0E945DAA209100
:10B83000E70F3091E80F409158066217730710F434
:10B84000442351F1442309F445C00DDE20E030E0EB
:10B850004AE754E40E94F6AD0E945DAA2091E70FEA
:10B860003091E80F62177307A8F11092580681E033
:10B870008093570680915506882361F163ED72E14C
:10B8800080915306909154060C94AB4D10920C028B
:10B8900081E080935706089581E0809358061092C6
:10B8A000570680915506882391F062EF72E18091EE
:10B8B0005306909154060E943A4C0E944B806FEEC2
:10B8C00072E180915306909154060E94AB4D52DF75
:10B8D0000C94663508950E94727F8091B305882389
:10B8E00041F180914B06811101C0089510924B06E1
:10B8F0000E94618D8091DE05882319F01092DE058B
:10B900000CC080914F0690915006DC01ED91FC91A6
:10B910000088F189E02D60E0199580915506882313
:10B9200041F062E971E180915306909154060C94C4
:10B93000AB4D089580915606809355060895209149
:10B940007A0D222369F0A091780DB091790DED91D7
:10B95000FC9111970190F081E02DBC01CD0119946B
:10B9600008952091770D222369F0A091750DB09173
:10B97000760DED91FC9111970190F081E02DBC01C5
:10B98000CD01199408952091740D222369F0A0919E
:10B99000720DB091730DED91FC9111970190F081B2
:10B9A000E02DBC01CD01199408952091710D222341
:10B9B00069F0A0916F0DB091700DED91FC91119710
:10B9C0000190F081E02DBC01CD01199408952091E2
:10B9D0006E0D222369F0A0916C0DB0916D0DED916B
:10B9E000FC9111970190F081E02DBC01CD011994DB
:10B9F000089520916B0D222369F0A091690DB091FB
:10BA00006A0DED91FC9111970190F081E02DBC0140
:10BA1000CD01199408952091680D222369F0A09119
:10BA2000660DB091670DED91FC9111970190F08139
:10BA3000E02DBC01CD01199408952091650D2223BC
:10BA400069F0A091630DB091640DED91FC91119797
:10BA50000190F081E02DBC01CD0119940895209151
:10BA6000620D222369F0A091600DB091610DED91FE
:10BA7000FC9111970190F081E02DBC01CD0119944A
:10BA8000089580914F0690915006DC01ED91FC9154
:10BA9000EC5AFF4F0190F081E02D199480914F06F0
:10BAA00090915006DC01ED91FC91EE5AFF4F019010
:10BAB000F081E02D199480914F0690915006DC01A1
:10BAC000ED91FC91E05BFF4F0190F081E02D199426
:10BAD00080916A0F81110DC08091DC059091DD0588
:10BAE000DC01ED91FC910190F081E02D60E070E0CF
:10BAF0001994089580916A0F81110DC08091DC0521
:10BB00009091DD05DC01ED91FC910190F081E02D3B
:10BB10006FEF70E0199408956DCA83CA80917C0D0F
:10BB2000882311F067DA01C07CDA90917C0D81E006
:10BB3000892780937C0D08958CCAA2CA80917B0DC1
:10BB4000882311F086DA01C09BDA90917B0D81E0A9
:10BB5000892780937B0D089580915606882361F094
:10BB60000E949B84029741F06BEE74E18091530632
:10BB7000909154060C94AB4D0895809155068823FE
:10BB800041F06DE074E180915306909154060C945D
:10BB9000AB4D089580915506882341F06DEF73E118
:10BBA00080915306909154060C94AB4D0895CF9319
:10BBB000DF9320917F0D3091800D28173907D1F048
:10BBC0009093800D80937F0D20915506222391F054
:10BBD000EC016CEB74E180915306909154060E9445
:10BBE0003A4CBE018091530690915406DF91CF915B
:10BBF0000C94EC74DF91CF910895CF93DF93209153
:10BC00007D0D30917E0D28173907D1F090937E0D70
:10BC100080937D0D20915506222391F0EC0162EA7C
:10BC200074E180915306909154060E943A4CBE01F3
:10BC30008091530690915406DF91CF910C94EC744F
:10BC4000DF91CF9108952091740D222339F0BC012A
:10BC500080915E0D90915F0D0C94276A089520915C
:10BC6000710D222339F0BC0180915C0D90915D0D26
:10BC70000C94276A089520916E0D222339F0BC019F
:10BC800080915A0D90915B0D0C94276A0895209134
:10BC90006B0D222339F0BC018091580D9091590D04
:10BCA0000C94276A08952091680D222339F0BC0175
:10BCB0008091560D9091570D0C94276A089520910C
:10BCC000650D222339F0BC018091540D9091550DE2
:10BCD0000C94276A08952091620D222339F0BC014B
:10BCE0008091520D9091530D0C94276A0895CF9234
:10BCF000DF92EF92FF9220910002213019F42091FF
:10BD0000760F04C02230C9F520917C0F2223A9F1BF
:10BD10009C01211584E0380710F02FEF33E0ADE0EF
:10BD2000B0E00E9428AF2FEF33E040E050E00E94E7
:10BD3000DAAE69017A018FEFC81AD80AE80AF80A60
:10BD4000809168128C15C9F0C092681280915506D6
:10BD5000882399F06BE574E1809153069091540625
:10BD60000E943A4C6C2D8091530690915406FF909E
:10BD7000EF90DF90CF900C945F77FF90EF90DF9083
:10BD8000CF900895CF92DF92EF92FF922091000220
:10BD9000213019F42091730F04C02230C9F520918D
:10BDA000790F2223A9F19C01211584E0380710F0B6
:10BDB0002FEF33E0ADE0B0E00E9428AF2FEF33E08B
:10BDC00040E050E00E94DAAE69017A018FEFC81AB4
:10BDD000D80AE80AF80A809166128C15C9F0C09258
:10BDE000661280915506882399F064E474E180918D
:10BDF0005306909154060E943A4C6C2D8091530644
:10BE000090915406FF90EF90DF90CF900C945F7765
:10BE1000FF90EF90DF90CF90089581E080934C06E3
:10BE20005ADD80915506882341F06AE274E18091E1
:10BE30005306909154060C94AB4D089583E0809383
:10BE40004C061EDA80915506882341F067E374E1C1
:10BE500080915306909154060C94AB4D089582E066
:10BE600080934C060DDA80915506882341F06DE1F0
:10BE700074E180915306909154060C94AB4D089553
:10BE80000C94058E8091010281110C94E98D0C9423
:10BE9000058E0C94E98D80910002813011F482E0CE
:10BEA00001C081E00C94698B82E00C94698B81E085
:10BEB0000C94698B0C94362190919B0F81E089271B
:10BEC000A0CB80E09ECB81E09CCB9091990F81E04C
:10BED0008927C9CB80E0C7CB81E0C5CB8091EE0537
:10BEE000882321F087D821E138E503C09AD82AEFCA
:10BEF00037E54CE251E060E070E085E89AE00C94B0
:10BF000023408091E705882321F0A3D820E438E579
:10BF100003C0B6D829E238E54CE251E060E070E0B9
:10BF200085E89AE00C94234080914F06909150064A
:10BF3000DC01ED91FC9104ACF5ADE02D66E01995C6
:10BF400080915506882351F00E94418D64EF73E182
:10BF500080915306909154060C94AB4D08958091B6
:10BF60004F0690915006DC01ED91FC9102ACF3ADCF
:10BF7000E02D66E0199580915506882351F00E94C6
:10BF8000418D60EE73E180915306909154060C94BC
:10BF9000AB4D0895682F80915306909154060E94EE
:10BFA000897869EE74E180915306909154060C945F
:10BFB0003A4CF0DF80915306909154060C94984DC2
:10BFC000CF92DF92EF92FF929C01A3E6B0E00E9435
:10BFD00028AF2FEF33E040E050E00E94DAAE690175
:10BFE0007A018FEFC81AD80AE80AF80A8091AF05DB
:10BFF0008C15A1F0C092AF0580915506882371F091
:10C000006BE874E180915306909154060E943A4C7B
:10C010008C2DFF90EF90DF90CF90CBCFFF90EF90E3
:10C02000DF90CF900895CF92DF92EF92FF929C0124
:10C03000A3E6B0E00E9428AF2FEF33E040E050E0ED
:10C040000E94DAAE69017A018FEFC81AD80AE80AAD
:10C05000F80A8091B0058C15A1F0C092B0058091CE
:10C060005506882371F062E774E180915306909140
:10C0700054060E943A4C8C2DFF90EF90DF90CF90A9
:10C0800098CFFF90EF90DF90CF90089520915306C6
:10C0900030915406882319F06DEB76E002C061EC14
:10C0A00076E0C9010C943A4CF1DF809153069091EF
:10C0B00054060C94984D20915306309154068823D1
:10C0C00019F06EED74E102C063EE74E1C9010E94E3
:10C0D0003A4C80915306909154060C94984D6CED17
:10C0E00074E180915306909154060C943A4C68ED9B
:10C0F00074E180915306909154060C943A4CCF937E
:10C10000CDE266ED74E180915306909154060E9451
:10C110003A4CC150B1F780915306909154060E9459
:10C12000984D8091530690915406DC01ED91FC915D
:10C130000284F385E02DCF9119942BC80C94B55748
:10C1400080918B0D882311F024D802C00E94B5572E
:10C1500090918B0D81E0892780938B0D08958091BC
:10C160004F0690915006DC01ED91FC9100ACF1ADD1
:10C17000E02D66E0199580915506882351F00E94C4
:10C18000418D67EC76E180915306909154060C94B2
:10C19000AB4D089580914F0690915006DC01ED91D2
:10C1A000FC9104ACF5ADE02D65E019958091550644
:10C1B000882351F00E94418D6EEB76E18091530609
:10C1C000909154060C94AB4D089580914F06909138
:10C1D0005006DC01ED91FC9102ACF3ADE02D65E081
:10C1E000199580915506882351F00E94418D6AEA85
:10C1F00076E180915306909154060C94AB4D0895CE
:10C2000080914F0690915006DC01ED91FC9100ACBD
:10C21000F1ADE02D65E0199580915506882351F028
:10C220000E94418D68EA76E1809153069091540610
:10C230000C94AB4D089580914F0690915006DC010F
:10C24000ED91FC9104ACF5ADE02D64E01995809181
:10C250005506882351F00E94418D6FE976E1809167
:10C260005306909154060C94AB4D089580914F065F
:10C2700090915006DC01ED91FC9102ACF3ADE02D04
:10C2800064E0199580915506882351F00E94418DF4
:10C290006BE876E180915306909154060C94AB4D77
:10C2A000089580914F0690915006DC01ED91FC912C
:10C2B00000ACF1ADE02D64E019958091550688231E
:10C2C00051F00E94418D69E876E18091530690918A
:10C2D00054060C94AB4D089580914F0690915006F2
:10C2E000DC01ED91FC9104ACF5ADE02D63E0199516
:10C2F00080915506882351F00E94418D60E876E1D7
:10C3000080915306909154060C94AB4D0895809102
:10C310004F0690915006DC01ED91FC9102ACF3AD1B
:10C32000E02D63E0199580915506882351F00E9415
:10C33000418D6CE676E180915306909154060C9401
:10C34000AB4D089580914F0690915006DC01ED9120
:10C35000FC9100ACF1ADE02D63E01995809155069C
:10C36000882351F00E94418D6AE676E18091530660
:10C37000909154060C94AB4D089580914F06909186
:10C380005006DC01ED91FC9104ACF5ADE02D62E0CE
:10C39000199580915506882351F00E94418D61E6E0
:10C3A00076E180915306909154060C94AB4D08951C
:10C3B00080914F0690915006DC01ED91FC9102AC0A
:10C3C000F3ADE02D62E0199580915506882351F078
:10C3D0000E94418D6DE476E1809153069091540660
:10C3E0000C94AB4D089580914F0690915006DC015E
:10C3F000ED91FC9100ACF1ADE02D62E019958091DA
:10C400005506882351F00E94418D6BE476E18091BE
:10C410005306909154060C94AB4D089580914F06AD
:10C4200090915006DC01ED91FC9104ACF5ADE02D4E
:10C4300061E0199580915506882351F00E94418D45
:10C4400062E476E180915306909154060C94AB4DD2
:10C45000089580914F0690915006DC01ED91FC917A
:10C4600002ACF3ADE02D61E019958091550688236B
:10C4700051F00E94418D6EE276E1809153069091D9
:10C4800054060C94AB4D089580914F069091500640
:10C49000DC01ED91FC9100ACF1ADE02D61E019956E
:10C4A00080915506882351F00E94418D6CE276E11F
:10C4B00080915306909154060C94AB4D08950C94C2
:10C4C000498D0C94558D0F931F93CF93DF9300915B
:10C4D000860D1091870DC091BB05D091BC05B801A8
:10C4E000CE010E94BC3F882379F0B801CE010E94A2
:10C4F000D43F8091BD059091BE05DC01ED91FC918A
:10C5000000A0F1A1E02D19950091840D1091850DE9
:10C51000C091BB05D091BC05B801CE010E94BC3FC3
:10C52000882321F0B801CE010E94D43F72988091F7
:10C530005506882361F06EEA75E18091530690916B
:10C540005406DF91CF911F910F910C94AB4DDF9169
:10C55000CF911F910F910895CF93DF938091E011B8
:10C56000882321F11092E01160E088E00E94B24F30
:10C57000C091E111D091E211BE0185E89AE00E94DC
:10C58000BC3F882329F0BE0185E89AE00E94D43F91
:10C5900080915506882371F063E176E1809153061E
:10C5A00090915406DF91CF910C94AB4DDF91CF91D8
:10C5B0000C942080DF91CF9108958091E01181113A
:10C5C00002C00C9420800895CF93DF938091E311F3
:10C5D000882311F10E94C9581092E311C091E11112
:10C5E000D091E211BE0185E89AE00E94BC3F882309
:10C5F00029F0BE0185E89AE00E94D43F809155065B
:10C60000882371F06AEF75E180915306909154068A
:10C61000DF91CF910C94AB4DDF91CF910C940459E5
:10C62000DF91CF9108950C9404590E94C95840910C
:10C63000EC0F5091ED0F60E070E025EB37E585E8F9
:10C640009AE00E9423409093E2118093E11180913F
:10C650005506882341F06FED75E180915306909166
:10C6600054060C94AB4D08950E94B5574091EC0FC1
:10C670005091ED0F60E070E029EC38E585E89AE034
:10C680000E9423409093E2118093E111809155061E
:10C69000882341F06CEC75E180915306909154062B
:10C6A0000C94AB4D08956091F20F70E088E00E9409
:10C6B0001D5080915506882341F066EB75E180910D
:10C6C0005306909154060C94AB4D08950C947B59ED
:10C6D0000C94925980918A0D882319F00E947B59FD
:10C6E00002C00E94925990918A0D81E0892780931F
:10C6F0008A0D08950C94BC590E94BC5980914F0634
:10C7000090915006DC01ED91FC9104A0F5A1E02D83
:10C7100019940C94EA598091890D882319F00E948C
:10C72000BC5902C00E94EA599091890D81E0892785
:10C730008093890D08950C94FB590C94175A80919D
:10C74000880D882319F00E94FB5902C00E94175AD5
:10C750009091880D81E089278093880D08950C942D
:10C760007A8C8091190E81110C94648C0C947A8CC3
:10C770000C94648C0E94CA5780914F069091500689
:10C78000DC01ED91FC9102A0F3A1E02D1994CF936F
:10C79000DF93C091BB05D091BC056091860D70916F
:10C7A000870DCE010E94BC3F811129C04091830DAD
:10C7B00050E060E070E022E93FE6CE010E942B40AD
:10C7C0009093870D8093860D8091BD059091BE0555
:10C7D000DC01ED91FC91068CF78DE02D199580918F
:10C7E000D405882361F06091840D7091850D80914E
:10C7F000BB059091BC050E94BC3F882371F08091DD
:10C8000055068823E9F065EA75E180915306909119
:10C810005406DF91CF910C94AB4D0E94867226E8AE
:10C8200032E744E650E060E070E08091BB05909113
:10C83000BC050E942B409093850D8093840DDFCF23
:10C84000DF91CF9108950E946D74809155068823E1
:10C8500041F06AE775E180915306909154060C947B
:10C86000AB4D0895E091810DF091820D82810E947F
:10C87000964180915506882341F06CE575E18091E1
:10C880005306909154060C94AB4D089580911A0E66
:10C89000882319F00E94D67402C00E94C07480914F
:10C8A0005506882379F020915C0F80915306909172
:10C8B0005406222319F060E275E102C069E375E1D4
:10C8C0000C94AB4D089507C8CF9380915C0A8823E0
:10C8D00009F455C00E94C36C90915A0A882339F01C
:10C8E00091114DC08091DF05882389F148C09111D5
:10C8F00046C080915506882341F061E075E1809142
:10C900005306909154060E94AB4D0E945A6D81E0EF
:10C910008093DA0580910602813089F58091960F27
:10C92000882369F140915E0F50915F0F1416150630
:10C930005CF4052E000C660B770B20E43AE885E8E2
:10C940009AE0CF910C942340CF910C94408A82E0DE
:10C950008093DF0580915506882341F06DE075E1F5
:10C9600080915306909154060E94AB4DC1E0C09354
:10C97000DE050E946B5C0E945A6DC093DA05CF9170
:10C9800008950C94405908950895FC018281938183
:10C990008830910529F410922B0110922A010895F4
:10C9A000099721F410922901109228010895FC01A1
:10C9B000178A168A6CED75E082810C948581CF937D
:10C9C000DF93EC011F8A1E8A8A810E9488418B8D29
:10C9D000882331F08A810E9475819A8F898F1B8EFE
:10C9E000DF91CF910895DF92EF92FF920F931F9303
:10C9F000CF93DF93EC018A81893010F40E946F415C
:10CA0000DD8C6B8D7C8D098D1A8DEA80FB8089E031
:10CA10008E1508F466C00F30110538F001369DE61A
:10CA2000190728F000E61DE602C00FE010E06F30A5
:10CA3000710538F061368DE6780728F060E67DE60E
:10CA400002C06FE070E080E090E00E9495AD20E0D1
:10CA500030E04AE754E40E94F0A920E030E04CE8DE
:10CA600052E40E94F6AD9B01AC0160E070E08AEFF9
:10CA700094E40E94F0A90E9458AAFF2425E12E9D6B
:10CA8000F0012F9DF00D1124E25EFE4EDD2071F0CD
:10CA900023813481AB0177FF04C044275527461B0F
:10CAA000570B88279927841B950B0AC0258136814F
:10CAB000AB0177FF04C044275527461B570BCA011B
:10CAC0004FB7F89455E15E9DF0015F9DF00D112484
:10CAD000E25EFE4E108B0787328B218B948B838B0B
:10CAE0004FBF9D8D6B8D7C8D8A819923F9F08A30A3
:10CAF00058F495E1899FF0011124E25EFE4E058114
:10CB000016811695079502C00EEE12E041E00E94D4
:10CB1000B64161E070E080E090E00E9428518A8197
:10CB20000E94758108171907A0F31EC08A3058F4B7
:10CB300095E1899FF0011124E25EFE4E038114818C
:10CB40001695079502C00AEC18E040E00E94B64135
:10CB500061E070E080E090E00E9428518A810E94AC
:10CB6000758180179107A0F38A810E948841B801DE
:10CB70008A81DF91CF911F910F91FF90EF90DF900D
:10CB80000C948581CF93DF93EC018A81893010F476
:10CB90000E946F4148EE53E05B874A8720ED37E003
:10CBA0003D872C878CED95E09F878E87598B488B2E
:10CBB0003B8B2A8B9D8B8C8BDF91CF910895CF93EC
:10CBC000DF93EC017F8B6E8B8885998568177907D9
:10CBD00069F48A810E9488418B8D882329F18A819A
:10CBE0000E9475819A8F898F1B8E1EC0CE010E9474
:10CBF0000F53EA81EA30B0F49C01C39714F022E3AA
:10CC000030E02E3C8FEF380714F42EEC3FEF8FB757
:10CC1000F89495E1E99FF0011124E25EFE4E318720
:10CC200020878FBF81E08B8FDF91CF910895CF93C5
:10CC3000DF93EC0189A19AA1892B11F01AA219A204
:10CC40009B0177FF03C0319521953109B901CE01D0
:10CC50000E940F5390932D0180932C019F8B8E8BFC
:10CC60000E9460516D8F7E8F8F8F98A3DF91CF913F
:10CC700008950F931F93CF93DF938C01FC01778B63
:10CC8000668B0E940F53EC01F801828193818830FA
:10CC90009105D1F4D7FF06C060E08AE00E94B24F50
:10CCA00061E005C061E08AE00E94B24F60E086E08A
:10CCB0000E94B24FD7FF03C0D195C195D109D0933F
:10CCC0002B01C0932A011BC00997C9F4D7FF06C0E6
:10CCD00060E08DE00E94B24F61E005C061E08DE050
:10CCE0000E94B24F60E08BE00E94B24FD7FF03C0BA
:10CCF000D195C195D109D0932901C0932801DF9125
:10CD0000CF911F910F910895CF93DF93EC018A810A
:10CD1000893010F40E946F412EEC3FEF3B872A8749
:10CD200082E390E09D878C871F861E86398B288B37
:10CD30009B8B8A8B1D8A1C8A6EEE72E08A810E9410
:10CD400070816AEC78E08A810E94F7418CED95E071
:10CD50009A8F898F1B8EDF91CF910895CF93DF93A8
:10CD6000EC0189A19AA1892B11F01AA219A2CE0176
:10CD7000CBD510922D0110922C011F8A1E8A0E9481
:10CD800060516D8F7E8F8F8F98A3DF91CF91089523
:10CD90000F931F93CF93DF93FC0121A132A1232B8B
:10CDA00091F1EC010E9460510D8D1E8D2F8D38A1E7
:10CDB000DC01CB01801B910BA20BB30B4097A105AB
:10CDC000B10508F189A19AA10197E9F46E897F89DB
:10CDD000615071097F8B6E8BCE01161617062CF0F1
:10CDE000DF91CF911F910F91B9CF0E940F53909374
:10CDF0002D0180932C019F8B8E8B0E9460516D8F33
:10CE00007E8F8F8F98A3DF91CF911F910F910895FF
:10CE1000CF93DF93EC011B861A868FEF90E09D87FE
:10CE20008C871F861E86198A188A9B8B8A8B1D8A7F
:10CE30001C8A61E08CE20E94E14F8A819B81089705
:10CE400021F410922D0110922C011AA219A2DF9147
:10CE5000CF910895CF93DF93EC0121E03FEF3B8723
:10CE60002A878FEF90E09D878C871F861E86398BDF
:10CE7000288B9B8B8A8B1D8A1C8A61E08AE00E942A
:10CE8000E14F61E086E00E94E14F61E08DE20E94A7
:10CE9000E14F61E08DE00E94E14F61E08BE00E9494
:10CEA000E14F61E08EE20E94E14F8A819B818830F0
:10CEB000910529F410922B0110922A0106C00997BE
:10CEC00021F41092290110922801DF91CF91089549
:10CED0000F931F93CF93DF93EC011F8A1E8A8C015F
:10CEE000075E1F4F40E068E0C8010E94B84440E080
:10CEF0006CE0C8010E94B8440E9460516C8F7D8F25
:10CF00008E8F9F8FDF91CF911F910F910895CF93B7
:10CF1000DF93EC017F8B6E8B0E940F53AC018A81F3
:10CF20009B818830910541F4CE01499657FF02C09C
:10CF30006AE009C068E00DC00997D1F4CE014996B6
:10CF400057FF06C06EE042382FEF520744F001C091
:10CF50006CE04F3751052CF04EE750E002C042E83C
:10CF60005FEF57FF03C05195419551090E94B844A6
:10CF70000E9460516C8F7D8F8E8F9F8FDF91CF913C
:10CF800008950F931F93CF93DF93EC010E9460519C
:10CF90000C8D1D8D2E8D3F8DDC01CB01801B910BE7
:10CFA000A20BB30B853F9140A105B10540F06E89FE
:10CFB0007F89CE01DF91CF911F910F91A8CFDF9193
:10CFC000CF911F910F910895CF93DF93EC01809142
:10CFD0008D0D811109C06A8D7B8DCE0149960E940D
:10CFE000E97781E080938D0D21E83FEF3B872A8729
:10CFF0008FE790E09D878C871F861E86398B288B54
:10D000009B8B8A8B1D8A1C8ADF91CF9108950F9389
:10D010001F93CF93DF93EC010E9460510C8D1D8D07
:10D020002E8D3F8DDC01CB01801B910BA20BB30B2E
:10D03000853F9140A105B10548F06E897F89CE01F9
:10D04000DF91CF911F910F910C948853DF91CF9175
:10D050001F910F9108956F927F928F929F92AF923E
:10D06000BF92CF92DF92EF92FF920F931F93CF93D5
:10D07000DF938091EB0C9091EC0CDC01ED91FC9135
:10D080000480F581E02D1995B12C181619060CF0C5
:10D09000D5C0AA24A3948091EB0C9091EC0CDC01F8
:10D0A000ED91FC910480F581E02D1995892B09F40F
:10D0B000C5C0C091E70D81E08C0F8093E70D809192
:10D0C000EB0C9091EC0CDC01ED91FC910680F7816A
:10D0D000E02D1995EC2FF0E0E955F24F80838A306E
:10D0E000D1F6E090E70DF12C1092D10C1092D00CFB
:10D0F0001092CC0C1092CD0C1092CE0C1092CF0C42
:10D100001092CB0C1092CA0C1092C90C87EAC82E50
:10D110008DE0D82E00E010E0D0E0C0E00E151F0535
:10D120000CF06FC0F60191916F019D3009F466C05B
:10D130009C37A1F19A3009F055C0CC2359F16C2EDF
:10D14000712CC30101970E940C867093D10C6093DF
:10D15000D00C0E9460516093EE0C7093EF0C8093A2
:10D16000F00C9093F10C80918C0D882309F462C02F
:10D170008090D00C9090D10CB8016619770987EA9D
:10D180009DE00E943A488816990609F453C010920F
:10D19000A60D52C01092A60DD0E030C08C2F90E0AA
:10D1A000FC01ED58FD4E1082D13099F068F0D2307C
:10D1B000B1F40E940C866093CC0C7093CD0C8093DC
:10D1C000CE0C9093CF0C0BC00E940C866093C90CC0
:10D1D00006C00E940C867093CB0C6093CA0CDF5F74
:10D1E000C0E00CC00F3311053CF4EC2FF0E0ED581B
:10D1F000FD4E9083CF5F02C01092A60D0F5F1F4FB0
:10D200008DCF8091A60D81110EC08091C60C90919A
:10D21000C70C01969093C70C8093C60C60E087E81A
:10D220000E94D84802C0BB24B3941092A70D10925C
:10D23000E70D31CFA092A60DD1E0E0CF8B2DDF918D
:10D24000CF911F910F91FF90EF90DF90CF90BF9003
:10D25000AF909F908F907F906F900895CF93109292
:10D26000C80C1092C50C1092C70C1092C60C61E04D
:10D2700089E30E94B24F0E94DF478091EB0C9091AE
:10D28000EC0CDC01ED91FC910480F581E02D199509
:10D29000892B61F08091EB0C9091EC0CDC01ED910D
:10D2A000FC910680F781E02D1995E7CF0E94878ECB
:10D2B0008091EB0C9091EC0CDC01ED91FC910284DF
:10D2C000F385E02D19951092ED0C0E94605160934A
:10D2D000EE0C7093EF0C8093F00C9093F10CC1E086
:10D2E000BADE81110E94212E0E941D480E9459849D
:10D2F0008091C60C9091C70C0A9724F48091ED0C94
:10D30000882331F060E08AE80E94D848C093C80CB6
:10D310008091C80C882321F38091C50C882341F0AB
:10D3200049EC51E060E070E084E39EE00E94AAAE28
:10D3300060E089E30E94B24F60E08AE3CF910C94F1
:10D34000B24FEF92FF920F931F93CF93DF9300D0D2
:10D3500000D0CDB7DEB766EA75E0CE0101960E9437
:10D36000FB4B0D811E81F02EEE24E3948091EB0C9B
:10D370009091EC0CDC01ED91FC910480F581E02DA5
:10D380001995892B21F18091EB0C9091EC0CDC012B
:10D39000ED91FC910680F781E02D19958F3439F4D9
:10D3A000E092A50D80939A0DE092990DDFCF9091B8
:10D3B000A50D9923D9F2E091990D91E09E0F9093DC
:10D3C000990DF0E0E656F24F80839F1578F2809138
:10D3D000990D8F1510F4F12C21C04BE050E06EE850
:10D3E0007DE0CE0101960E94AC7AAAE9BDE0E6EAB2
:10D3F000F5E0FF24F3941127CF01865A954080175A
:10D40000910734F49D9181919817B1F3F12CF4CFE9
:10D4100010929A0D1092A50D1092990DCE010196C1
:10D420000E94CB4B8F2D26960FB6F894DEBF0FBE11
:10D43000CDBFDF91CF911F910F91FF90EF90089595
:10D44000DC01ED91FC910190F081E02D1994CF93D6
:10D45000DF93EC017F8B6E8B0E940F53BC018A819E
:10D46000DF91CF910C9485810895089508950895D2
:10D470000895623039F0633041F0613041F44093F7
:10D48000F70D08954093F60D08954093F50D089516
:10D49000623069F06330A1F06130D1F45093FB0D3C
:10D4A0004093FA0D3093FD0D2093FC0D0895509399
:10D4B000020E4093010E3093040E2093030E089544
:10D4C00050930B0E40930A0E30930D0E20930C0ECA
:10D4D0000895089520910F0E211102C0FC0162836E
:10D4E000089520910F0E211102C0FC01648308955C
:10D4F00020910F0E211102C0FC016383089508954D
:10D5000080910F0E811101C037C20895089580E007
:10D5100008950895089508950895089508958091AF
:10D520000F0E811103C08FE090E01EC3089580911B
:10D530000F0E811120C0633091F028F4613049F062
:10D54000623051F00895653081F060F0663081F00E
:10D55000089589E090E00EC08AE090E00BC08BE077
:10D5600090E008C08CE090E005C08DE090E002C043
:10D570008EE090E0F9C2089520910F0E211107C0AE
:10D58000FC018481882319F082E090E0EDC20895C7
:10D5900020910F0E211107C0FC018381882319F00F
:10D5A00081E090E0E1C2089580910F0E811103C0E7
:10D5B0008BE090E0D9C2089580910F0E811104C0D4
:10D5C00060E080E190E00EC3089580910F0E81111C
:10D5D00004C060E08FE090E005C3089580910F0ED5
:10D5E000811126C06330A1F028F4613049F0623027
:10D5F00059F008956530A1F078F06630A9F00895EB
:10D6000060E089E090E013C060E08AE090E00FC045
:10D6100060E08BE090E00BC060E08CE090E007C041
:10D6200060E08DE090E003C060E08EE090E0DAC260
:10D63000089580910F0E811126C06330A1F028F467
:10D64000613049F0623059F008956530A1F078F00A
:10D650006630A9F0089561E089E090E013C061E0D0
:10D660008AE090E00FC061E08BE090E00BC061E0E9
:10D670008CE090E007C061E08DE090E003C061E0E5
:10D680008EE090E0AFC2089520910F0E211108C0E6
:10D69000FC018281882321F061E088E090E0A2C251
:10D6A000089520910F0E211108C0FC018481882368
:10D6B00021F061E082E090E095C2089520910F0E84
:10D6C000211108C0FC018381882321F061E081E001
:10D6D00090E088C2089580910F0E811104C061E02E
:10D6E00086E090E07FC2089580910F0E811104C002
:10D6F00060E08BE090E076C2089580910F0E81117A
:10D7000004C061E087E090E06DC2089580910F0E43
:10D71000811104C061E085E090E064C208958091C9
:10D720000F0E81112EC06091F80D7091F90D80914E
:10D73000080E9091090E0E94D43F1092FE0D809128
:10D740000F0E81110CC06091FF0D7091000E809141
:10D75000080E9091090E0E94D43F1092050E809100
:10D760000F0E81110CC06091060E7091070E809112
:10D77000080E9091090E0E94D43F10920E0E109246
:10D78000EC0D089580910F0E811117C08091EC0D62
:10D79000811113C02FE33FE648EB5BE060E070E0EF
:10D7A0008091080E9091090E0E9423409093F90DEC
:10D7B0008093F80D81E08093EC0D089580910F0E19
:10D7C000882329F06CED75E081E00C94444184E0FD
:10D7D00090E0CAC180910F0E882329F068EE73E0B3
:10D7E00081E00C94444160E084E090E0FBC18091D2
:10D7F0000F0E81111BC08091EF0D8823B9F068EEE8
:10D8000073E081E00E9444411092EF0D2CEB3CE666
:10D8100048E95AE360E070E08091080E9091090EAB
:10D820000E9423409093EE0D8093ED0D08956CEDD2
:10D8300075E080E00C94444124EF31E0DB010E946C
:10D8400085A92FEF30E040E050E00E94DAAECA0137
:10D85000B90164527A4F8F4F9F4F80E00C9444413E
:10D8600080910F0E882331F060ED77E081E00E9417
:10D87000444136C361E083E090E0B4C120910F0ED3
:10D88000211102C002963FC3089520910F0E22235A
:10D8900089F06FE676E080E00E9444412BE631E4B7
:10D8A00042E350E060E070E08091080E9091090E34
:10D8B0000C942340029627C380E00E946F4181E0D0
:10D8C0000E946F4180910F0E811103C082E00E947F
:10D8D0006F416CED75E080E00E9444416CED75E0B5
:10D8E00081E00E94444180910F0E81110CC084EFB1
:10D8F00092E7A1E0BB27ABBFFC016791769182E084
:10D900000E94444122C00895FC0180899189938737
:10D910008287828993899587848784899589978767
:10D920008687089526E00C94254F10925C0A40915A
:10D93000C9055091CA0560E070E020EA3FE6809199
:10D94000BB059091BC050C94234080910F0E811172
:10D9500012C084EF92E7A1E0BB27ABBFFC01679147
:10D96000769182E00E94444181E08093F00D109214
:10D97000F40D1092F10D089581E08093EF0D6CEDA0
:10D9800075E00C94444181E20E948A4F21E0892B8A
:10D9900009F420E0822F08958091CF05882309F4AF
:10D9A00046C081E08093580AEEDF882329F08091F9
:10D9B000D2058823D9F106C08091D005811105C018
:10D9C0008091CF050E94027531C09091CF059630AD
:10D9D00069F5823081F08330D1F0813039F5E09102
:10D9E000C709F091C80972978081918145E550E09F
:10D9F00060E070E017C0E091C709F091C809729724
:10DA0000808191814AE550E060E070E00BC0E091D8
:10DA1000C709F091C8097297808191814FE550E064
:10DA200060E070E08953964F0E94A755ACC20895FC
:10DA30008091BD059091BE05DC01ED91FC910688B9
:10DA4000F789E02D19958091150E811146D78091A7
:10DA5000140E882391F061E088E00E94B24F40915B
:10DA6000120E5091130E60E070E02BE532E78091CA
:10DA7000BB059091BC050E94234080911A0E88231B
:10DA800021F08091190E811101C086DF8091190E5D
:10DA9000882379F080911A0E882359F08091180E0E
:10DAA000882339F0E091160EF091170E82810E94C2
:10DAB00096413BCF80915A0A811155C064DF88237B
:10DAC000E9F081E080935A0A8091BD059091BE05EE
:10DAD000DC01ED91FC910288F389E02D19950ED3BC
:10DAE00022EA30E748E95AE360E070E08091BB0544
:10DAF0009091BC050E94234018DF09C08091190E47
:10DB0000882329F180911A0E882311F04FD744CF32
:10DB100037D78091180E882339F0E091160EF091D6
:10DB2000170E82810E9496414091100E5091110E65
:10DB300014161506BCF4052E000C660B770B28E1B5
:10DB40003DE68091BB059091BC050C9423408091EB
:10DB5000180E882339F0E091160EF091170E82818D
:10DB60000E94964165CF08950F931F9320910F0E49
:10DB7000211135C044EF52E761E077279C01220F65
:10DB8000331F820F931F092E000CAA0BBB0B0296AA
:10DB9000A11DB11D840F951FA61FB71FABBFFC01B0
:10DBA000879104EF12E721E033274091F40D93E0D1
:10DBB000499FA0011124052E000C660B770B4E5FC8
:10DBC0005F4F6F4F7F4F040F151F261F371F2BBF4F
:10DBD000F8010791801718F01F910F91B6CE1F9191
:10DBE0000F9108958F929F92AF92BF92CF92DF9242
:10DBF000EF92FF920F931F93CF93DF93EC01A62E2A
:10DC000080910F0E81116BC044EF52E761E07727DE
:10DC10006E01CC0CDD1CCC0EDD1E0D2C000CEE08B4
:10DC2000FF08D701C6010296A11DB11D480F591F5B
:10DC30006A1F7B1F6BBFFA01879144EF52E761E0D7
:10DC40007727B090F40D93E0B99E80011124012E46
:10DC5000000C220B330B0E5F1F4F2F4F3F4F400F17
:10DC6000511F621F731F6BBFFA014791481708F0DD
:10DC700036C08090F20D9090F30D0091080E109137
:10DC8000090EB401C8010E94BC3F882321F0B401F1
:10DC9000C8010E94D43F84EF92E7A1E0BB278C0D1E
:10DCA0009D1DAE1DBF1DABBFFC016791769182E04B
:10DCB0000E944441B092F10DC093F40DAA2079F076
:10DCC0001092F00D25EA3CE642E350E060E070E09F
:10DCD000C8010E9423409093F30D8093F20DDF91D1
:10DCE000CF911F910F91FF90EF90DF90CF90BF9059
:10DCF000AF909F908F900895CF92DF92EF92FF9216
:10DD000080910F0E811134C080910E0E882381F115
:10DD100061E08EE090E066DF60910C0E70910D0E78
:10DD2000CB01A0E0B0E0C0900A0ED0900B0EE12C29
:10DD3000F12CC816D906EA06FB0664F4BC01CD0135
:10DD40006C197D098E099F090E940F4CC60ED71EC3
:10DD5000E81EF91E2CE73EE6B701A6018091080EE9
:10DD60009091090E0E9423409093070E8093060E17
:10DD7000FF90EF90DF90CF900895CF92DF92EF92D7
:10DD8000FF9280910F0E811134C08091050E88237F
:10DD900081F161E08DE090E025DF6091030E7091EC
:10DDA000040ECB01A0E0B0E0C090010ED090020EB6
:10DDB000E12CF12CC816D906EA06FB0664F4BC0176
:10DDC000CD016C197D098E099F090E940F4CC60E6A
:10DDD000D71EE81EF91E2DEB3EE6B701A601809185
:10DDE000080E9091090E0E9423409093000E80939C
:10DDF000FF0DFF90EF90DF90CF900895CF92DF92CC
:10DE0000EF92FF9280910F0E811134C08091FE0D30
:10DE1000882381F161E08CE090E0E4DE6091FC0D0C
:10DE20007091FD0DCB01A0E0B0E0C090FA0DD09054
:10DE3000FB0DE12CF12CC816D906EA06FB0664F4AA
:10DE4000BC01CD016C197D098E099F090E940F4C00
:10DE5000C60ED71EE81EF91E2EEF3EE6B701A6013C
:10DE60008091080E9091090E0E9423409093F90D25
:10DE70008093F80DFF90EF90DF90CF900895809100
:10DE80000F0E81112CC08091F70D882341F08091F5
:10DE9000FE0D811104C081E08093FE0DAFDF809103
:10DEA000F60D882361F080910F0E811108C08091DA
:10DEB000050E811104C081E08093050E5EDF809124
:10DEC000F50D882361F080910F0E811108C08091BB
:10DED0000E0E811104C081E080930E0E0DCF0895C7
:10DEE0001092EF0D2CEB3CE644EF51E060E070E067
:10DEF0008091080E9091090E0E9423409093EE0DA0
:10DF00008093ED0D089580910F0E81110AC08091CC
:10DF1000EF0D882331F060ED77E081E00E9444410D
:10DF2000DFCF089580910F02882311F0729801C00D
:10DF3000729A90910F0281E0892780930F020895D1
:10DF400081E080935C0A08951092DB051092C7056A
:10DF50001092BA051092C3051092C4051092C5051F
:10DF60001092C60581E08093580A4091CB055091EC
:10DF7000CC0560E070E023EC3FE68091BB0590911A
:10DF8000BC050C9423408091930981111CC0109210
:10DF9000A4091092A5091092A6091092A70910923F
:10DFA000A8091092A9091092AC098091560A909183
:10DFB000570ADC01ED91FC910190F081E02D19955B
:10DFC0001092580A089523EC3FE645E050E060E0E7
:10DFD00070E08091BB059091BC050C94234060914A
:10DFE000250E7091260E8091BB059091BC050E9474
:10DFF000BC3F882319F081E08093240E089560E0EF
:10E0000087E00E94B24F1092590A089561E087E0BC
:10E010000E94B24F81E08093590A0895CF93DF9315
:10E020008091320E811110C084EF91E09093310EF7
:10E030008093300E8BE290E090932F0E80932E0E03
:10E0400081E08093320E20C080912E0E90912F0E91
:10E050008532910514F0049709C08331910514F0BD
:10E06000029704C0823091052CF0019790932F0EF7
:10E0700080932E0E80912E0E90912F0E97FF04C04C
:10E0800010922F0E10922E0EC0912D0ECC2311F057
:10E09000B6DF01C0BBDF81E08C2780932D0EC091DD
:10E0A000300ED091310E1C161D0654F01092320E17
:10E0B000A6DF2EE730E74AEF50E060E070E007C0EF
:10E0C0002EE030E7AE010D2E000C660B770B809131
:10E0D000BB059091BC050E94234090932C0E809329
:10E0E0002B0E80912E0E90912F0EC81BD90BD09322
:10E0F000310EC093300EDF91CF9108950F931F938F
:10E10000CF93DF9380915A0A882329F0DF91CF9132
:10E110001F910F9183CF00912B0E10912C0EC09167
:10E12000BB05D091BC05B801CE010E94BC3F88233D
:10E1300021F0B801CE010E94D43FDF91CF911F9111
:10E140000F915DCFCF92DF92EF92FF9210925A0A19
:10E150002091BF053091C0054091C1055091C20585
:10E160006091C3057091C4058091C5059091C60565
:10E170000E948BA96B017C0120E030E0A9010E9484
:10E1800091AD87FD09C0C092C305D092C405E0924D
:10E19000C505F092C60508C01092C3051092C405CB
:10E1A0001092C5051092C605FF90EF90DF90CF90BA
:10E1B000A5CF0F931F93CF93DF9380912A0E909159
:10E1C000DB0581112AC0992309F456C00091280E5D
:10E1D0001091290EC091BB05D091BC05B801CE01AC
:10E1E0000E94BC3F882321F0B801CE010E94D43F99
:10E1F0000DDF29ED30E742EC51E060E070E0809106
:10E20000BB059091BC050E942B409093290E8093F2
:10E21000280E81E080932A0E5AC08091590A9923D2
:10E2200061F0882329F0DF91CF911F910F91E7CE04
:10E23000DF91CF911F910F91E9CE8823C9F36091AF
:10E24000280E7091290E8091BB059091BC050E940B
:10E25000D43F29ED30E744E150E060E070E0809188
:10E26000BB059091BC050E942B409093290E809392
:10E27000280E10922A0E2BC0C0911002D0911102CC
:10E280002297D0931102C09310021C161D0674F43D
:10E29000BE01772787E00E941D50CC2321F081E04A
:10E2A0008093590A14C01092590A11C06091280E27
:10E2B0007091290E8091BB059091BC050E94D43FBE
:10E2C0009EDE8FEF90E09093110280931002DF9119
:10E2D000CF911F910F9108950F931F93CF93DF93C9
:10E2E0000091200E1091210EC091220ED091230E8C
:10E2F000C00FD11FD093230EC093220EBE017727EB
:10E3000087E00E941D50CC2321F081E08093590AC0
:10E3100002C01092590A10161106ECF580911E0EDB
:10E3200090911F0EC817D9070CF485C08091240E58
:10E33000882371F010921F0E10921E0E8CEF9FEF2B
:10E340009093210E8093200E81E080931D0E73C068
:10E3500068E770E080E090E00E940F4CDC01CB01A8
:10E360000A96A11DB11D90931F0E80931E0E68E2A8
:10E3700070E080E090E00E940F4CDC01CB010A9637
:10E38000A11DB11D66277727681B790B7093210E9D
:10E390006093200E50C0012B09F44DC080911E0ED9
:10E3A00090911F0E8C179D070CF445C080911D0E97
:10E3B000882311F10091250E1091260EC091BB0506
:10E3C000D091BC05B801CE010E94BC3F882399F1D1
:10E3D000B801CE010E94D43F12DE1092230E10929B
:10E3E000220E10921D0E8091DB05882321F1DF9112
:10E3F000CF911F910F91DDCE69E670E080E090E053
:10E400000E940F4CDC01CB018A569F4FAF4FBF4F8C
:10E4100090931F0E80931E0E68E270E080E090E003
:10E420000E940F4CDC01CB010A96A11DB11D9093F7
:10E43000210E8093200EDF91CF911F910F910895AF
:10E44000EF92FF921F93CF93DF9300D0CDB7DEB74B
:10E4500084E689838CE38A8388E28B831091270E7C
:10E460001330E8F4E12EF12C10FF02C0C8DD01C02A
:10E47000CDDDE1E0F0E0EC0FFD1FEE0DFF1D408172
:10E4800050E060E070E020E232E78091BB059091BF
:10E49000BC050E9423401F5F1093270E03C0AFDD11
:10E4A0001092270E0F900F900F90DF91CF911F9138
:10E4B000FF90EF90089560E088E00C94B24F61E027
:10E4C00089E20C94B24F0F931F93CF93DF9360E0D8
:10E4D0008BE20E94B24F00911B0E10911C0EC09156
:10E4E000BB05D091BC05B801CE010E94BC3F88237A
:10E4F00041F0B801CE01DF91CF911F910F910C94A3
:10E50000D43FDF91CF911F910F91089581E08093C7
:10E51000580A8091D30576D236CD1F920F920FB64E
:10E520000F9211242F933F938F939F93AF93BF9399
:10E5300080913B0D90913C0DA0913D0DB0913E0D11
:10E540003091330E23E0230F2D3720F40196A11DC7
:10E55000B11D05C026E8230F0296A11DB11D209311
:10E56000330E80933B0D90933C0DA0933D0DB093E3
:10E570003E0D80913F0D9091400DA091410DB091C5
:10E58000420D0196A11DB11D80933F0D9093400D4A
:10E59000A093410DB093420DBF91AF919F918F9188
:10E5A0003F912F910F900FBE0F901F9018950F93D2
:10E5B0001F93CF93DF9300912B0E10912C0EC091DF
:10E5C000BB05D091BC05B801CE010E94BC3F882399
:10E5D000A1F0B801CE010E94D43F2FEE3FE648EBF8
:10E5E0005BE060E070E08091BB059091BC050E940B
:10E5F000234090932C0E80932B0E6091250E7091EA
:10E60000260E8091BB059091BC050E94BC3F8111F4
:10E610004BC01092240E8FEF90E09093230E8093C6
:10E62000220EF4DC68E770E080E090E00E940F4C7E
:10E63000DC01CB010A96A11DB11D90931F0E8093A2
:10E640001E0E68E270E080E090E00E940F4CDC015A
:10E65000CB010A96A11DB11D66277727681B790B90
:10E660007093210E6093200E2CE631E744E150E0D8
:10E6700060E070E08091BB059091BC050E942B404A
:10E680009093260E8093250E2FEE3FE648EB5BE03D
:10E6900060E070E08091BB059091BC050E94234032
:10E6A00090932C0E80932B0EDF91CF911F910F91A1
:10E6B00008958F929F92AF92BF92CF92EF92FF9266
:10E6C0000F931F93CF93DF932091D605223008F04C
:10E6D00078C07B018C018090C3059090C405A09008
:10E6E000C505B090C60520E030E0A901C501B40120
:10E6F0000E9491AD181654F520E030E0A901C50143
:10E70000B4010E9489AA181654F420E030E048E4CD
:10E7100052E4C501B4010E9491AD1816D4F420E072
:10E7200030E048E452E4C501B4010E9489AA1816F9
:10E730009CF420E030E048EC52E4C501B4010E94B2
:10E7400091AD87FF09C0CBE4D0E008C0C0E0D0E0C5
:10E7500005C0C2E3D0E002C0C4E6D0E08FEF8C0D6C
:10E76000823068F4209739F06C2FC8010E948252E1
:10E770006C2FC7010CC0C801C7D8C70116C08DEFE8
:10E780008C0D8230F0F4209779F06C2FC801DF9166
:10E79000CF911F910F91FF90EF90CF90BF90AF90CE
:10E7A0009F908F900C948252C801DF91CF911F915E
:10E7B0000F91FF90EF90CF90BF90AF909F908F9070
:10E7C000A3C8DF91CF911F910F91FF90EF90CF9051
:10E7D000BF90AF909F908F9008958F929F92AF922D
:10E7E000BF92CF92DF92EF92FF92C090C305D0907C
:10E7F000C405E090C505F090C60520E030E0A90111
:10E80000C701B6010E9489AA20E030E040E05FE342
:10E8100087FD0BC0C701B6010E948CA94B015C01AA
:10E820000E9458AA97FD27C010C0C701B6010E94D8
:10E830008BA90E9458AA97FD1EC0653671058105F7
:10E840009105DCF424E6822F14C0C501B4010E94B6
:10E8500058AA65367105810591057CF420E030E009
:10E8600040E05FE3C701B6010E948CA90E9458AA4C
:10E8700084E6861B03C084E601C080E0FF90EF9031
:10E88000DF90CF90BF90AF909F908F9008950F939F
:10E890001F93CF93DF930091B4051091B505C091FC
:10E8A000BB05D091BC05B801CE010E94BC3F8823B6
:10E8B00021F0B801CE010E94D43F80915A0A8823EA
:10E8C00039F010925A0ADF91CF911F910F9116CC17
:10E8D000DF91CF911F910F91089560E089E20E942E
:10E8E000B24F2FE532E742E350E060E070E0809104
:10E8F000BB059091BC050C9423401F920F920FB65C
:10E900000F9211240BB60F922F933F934F935F9367
:10E910006F937F938F939F93AF93BF93EF93FF93E7
:10E9200080911A0E8823A9F0669917C0EE98CBDD66
:10E930008091190E882389F08091180E882339F070
:10E94000E091160EF091170E82810E94964170D8C8
:10E9500004C0669B02C0EE98B6DDFF91EF91BF91B7
:10E96000AF919F918F917F916F915F914F913F9167
:10E970002F910F900BBE0F900FBE0F901F90189508
:10E9800061E08BE20E94B24FEE9A23E632E748E85C
:10E9900053E160E070E08091BB059091BC050E945E
:10E9A000234090931C0E80931B0E089561E08BE230
:10E9B0000E94B24FEE9A23E632E748E853E160E066
:10E9C00070E08091BB059091BC050E94234090931C
:10E9D0001C0E80931B0E08950F931F93CF93DF930C
:10E9E000EC01AB0160E070E02AE00E94734C8C0106
:10E9F000CE010E94984D800F911FDF91CF911F9102
:10EA00000F9108958F929F92AF92BF92CF92DF9213
:10EA1000EF92FF920F931F93CF93DF931F921F925A
:10EA2000CDB7DEB7082E000C990BAA0BBB0BFC016F
:10EA30003197ED30F10508F033C28827EA5AFE4FCE
:10EA40008F4F0C9477A984E080938F098AE080939C
:10EA5000900986E28093920981E0809395098093E2
:10EA600096098093940941E157E120E030E08091DC
:10EA70008F0990E0281739070CF059C1FA018591E8
:10EA80009491A0E0B0E0880F991FAA1FBB1FF90165
:10EA9000EE0FFF1FEE0FFF1FEA5DF64F808391839D
:10EAA000A283B3832F5F3F4F4E5F5F4FE0CF84E081
:10EAB00080938F098AE08093900986E2809392097F
:10EAC00081E0809395098093960982E08093940970
:10EAD00049E057E120E030E080918F0990E028176D
:10EAE00039070CF024C1FA0185919491A0E0B0E0BF
:10EAF000880F991FAA1FBB1FF901EE0FFF1FEE0F12
:10EB0000FF1FEA5DF64F80839183A283B3832F5F5B
:10EB10003F4F4E5F5F4FE0CF84E08093900985E2E6
:10EB20008093920981E08093950988E0809396090B
:10EB300083E08093940980E090E0FC01EF5FF84E61
:10EB4000E491DC01A956B64FEC930196883091050B
:10EB5000A1F70E945254EBC088E080938F0986E0B1
:10EB60008093900986E28093920981E080939509D1
:10EB70008093960984E08093940941EF56E120E068
:10EB800030E080918F0990E0281739070CF0CFC052
:10EB9000FA0185919491A0E0B0E0880F991FAA1F17
:10EBA000BB1FF901EE0FFF1FEE0FFF1FEA5DF64FCF
:10EBB00080839183A283B3832F5F3F4F4E5F5F4F6C
:10EBC000E0CF88E080938F0986E08093900986E209
:10EBD0008093920981E0809395098093960985E05E
:10EBE0008093940941EE56E120E030E080918F0956
:10EBF00090E0281739070CF09AC0FA01859194919A
:10EC0000A0E0B0E0880F991FAA1FBB1FF901EE0F0B
:10EC1000FF1FEE0FFF1FEA5DF64F80839183A283F3
:10EC2000B3832F5F3F4F4E5F5F4FE0CFE091C70947
:10EC3000F091C80972978081918140E550E060E0D1
:10EC400070E08953964F0E94A7552AC182E18093B4
:10EC50008F0985E08093900982E28093920981E098
:10EC6000809395098093960987E08093940980E9C1
:10EC700093E3A0E0B0E08093260990932709A09346
:10EC80002809B0932909F2E08F2E912C01E010E0C1
:10EC900080E090E0A0E0BBE54CE454E060E070E090
:10ECA00024EEC22E2CE0D22EE12CF12C9801220F62
:10ECB000331F220F331F5401AA0CBB1CAA0CBB1C10
:10ECC0002A5D364FF901B7FF0DC0C082D182E282C2
:10ECD000F38295012A5D364FF901408351836283A7
:10ECE00073830CC0408351836283738395012A5DD3
:10ECF000364FF901C082D182E282F382880F991FD8
:10ED0000AA1FBB1F0E5F1F4FF2E08F0E911C22E166
:10ED10008216910459F688E79FEFA0E0B0E0809357
:10ED20006A0990936B09A0936C09B0936D090E94D6
:10ED3000C154B6C0CE0101960E94405423E040E188
:10ED400050E060E070E072C084E080938F0982E35D
:10ED50008093900986E28093920981E080939509DF
:10ED6000809396098AE08093940949ED56E120E06A
:10ED700030E080918F0990E028173907C4F6FA0136
:10ED800085919491A0E0B0E0880F991FAA1FBB1F46
:10ED9000F901EE0FFF1FEE0FFF1FEA5DF64F8083B4
:10EDA0009183A283B3832F5F3F4F4E5F5F4FE1CFCD
:10EDB00084E080938F0980E28093900986E28093BB
:10EDC000920981E080939509809396098BE0809366
:10EDD000940941ED56E120E030E080918F0990E008
:10EDE000281739070CF0A3CFFA0185919491A0E080
:10EDF000B0E0880F991FAA1FBB1FF901EE0FFF1F7C
:10EE0000EE0FFF1FEA5DF64F80839183A283B383E9
:10EE10002F5F3F4F4E5F5F4FE0CFCE0101960E94C4
:10EE2000405421E040E154E060E070E0CE01019602
:10EE30000E941B5535C084E080938F0983E0809346
:10EE4000900986E28093920981E0809395098093EE
:10EE500096098DE08093940949EC56E120E030E07A
:10EE600080918F0990E0281739070CF060CFFA01E4
:10EE700085919491A0E0B0E0880F991FAA1FBB1F55
:10EE8000F901EE0FFF1FEE0FFF1FEA5DF64F8083C3
:10EE90009183A283B3832F5F3F4F4E5F5F4FE0CFDD
:10EEA0000F900F90DF91CF911F910F91FF90EF90F6
:10EEB000DF90CF90BF90AF909F908F9008950F9369
:10EEC0001F93CF93DF93EC01462F50E060E070E09A
:10EED0002AE00E94734C8C01CE010E94984D800F55
:10EEE000911FDF91CF911F910F9108952FB7F89443
:10EEF000882381F0809160119091611190936F113E
:10EF000080936E11809170119091711118161906ED
:10EF1000ACF00FC0809162119091631190936F11CA
:10EF200080936E11809170119091711118161906CD
:10EF30002CF4809170119091711107C08091701123
:10EF40009091711191958195910990937111809390
:10EF500070112FBF0895AF92BF92CF92DF92EF92C0
:10EF6000FF920F931F93CF93DF931F921F92CDB702
:10EF7000DEB78C017A836983CE0101966C0158015A
:10EF800092E0A90EB11CE12CF12CC8010E94BAAE8E
:10EF9000F60161916F01861731F0C8010E94CCAE75
:10EFA000FFEFEF1AFF0A0F5F1F4F0A151B0569F7E6
:10EFB00081E0EF2809F480E00F900F90DF91CF916E
:10EFC0001F910F91FF90EF90DF90CF90BF90AF9087
:10EFD0000895EF92FF920F931F93CF93DF931F92A9
:10EFE0001F92CDB7DEB78C017B018AEA8A8341E0AC
:10EFF00050E0BE016E5F7F4FC8010E94C143D70140
:10F00000ED91FC910284F385E02DC701199582E80A
:10F01000898341E050E0BE016F5F7F4FC8010E94CD
:10F02000C1430F900F90DF91CF911F910F91FF90EF
:10F03000EF900895CF92DF92EF92FF920F931F937C
:10F040000E9460516B017C016093DC117093DD11B3
:10F050008093DE119093DF118091710A0E948A4F94
:10F060008093DB119091730A992329F091E081112B
:10F0700090E09093DB1180917B0A90917C0AA091A3
:10F080007D0AB0917E0A97018601081B190B2A0B95
:10F090003B0B40917F0A5091800A6091810A7091E8
:10F0A000820A9091740A041715072607370760F43F
:10F0B000C092770AD092780AE092790AF0927A0A9E
:10F0C0001092760A892F1EC09093750A8091DB11E9
:10F0D0008093740AC092770AD092780AE092790AF3
:10F0E000F0927A0A891761F0C0927B0AD0927C0A6A
:10F0F000E0927D0AF0927E0A91E09093760A02C037
:10F100001092760A1F910F91FF90EF90DF90CF90B1
:10F110000895462F50E060E070E02AE00C94734CB4
:10F120000F931F93CF93DF93EC012AE00E94734C5F
:10F130008C01CE010E94984D800F911FDF91CF91DD
:10F140001F910F910895CF92DF92EF92FF920F934C
:10F150001F93CF93DF936B01770FEE08FF08F7FE45
:10F160001BC0EC016DE20E94334C8C0144275527F3
:10F17000BA014C195D096E097F092AE0CE010E948F
:10F18000734C800F911FDF91CF911F910F91FF90D2
:10F19000EF90DF90CF9008952AE0B701A601DF91AC
:10F1A000CF911F910F91FF90EF90DF90CF900C9433
:10F1B000734CCF92DF92EF92FF920F931F93CF93F6
:10F1C000DF938C016B01770FEE08FF08F7FE12C08A
:10F1D0006DE20E94334CEC0144275527BA014C19CB
:10F1E0005D096E097F092AE0C8010E94734CC80FAF
:10F1F000D91F06C02AE0B701A6010E94734CEC019A
:10F20000C8010E94984D8C0F9D1FDF91CF911F91D7
:10F210000F91FF90EF90DF90CF9008950F931F9381
:10F22000CF93DF931F92CDB7DEB78C0169830E9425
:10F23000BAAE6981861729F0C8010E94CCAE81E080
:10F2400001C080E00F90DF91CF911F910F91089541
:10F25000CF930E94708484E090E090936E0A809334
:10F260006D0A85E39EE09093FF108093FE1010924C
:10F27000F91080916C0A9091350E891718F091E081
:10F280009093F6102EE33EE030930911209308117D
:10F290001092031190913E0E891718F091E090930F
:10F2A000001127E43EE030931311209312111092C5
:10F2B0000D119091470E891718F091E090930A1163
:10F2C00020E53EE030931D1120931C111092171180
:10F2D0009091500E891718F091E0909314111092AC
:10F2E0006B0A20E030E0F901EB52F14F408151818F
:10F2F000415051094432510520F491E090936B0A3A
:10F3000005C02D5F3F4F2837310569F790916B0A93
:10F31000992341F12091480E3091490E2D5D3F4FC8
:10F320003093490E2093480E20914A0E30914B0E97
:10F330002352310930934B0E20934A0E2091510EE7
:10F340003091520E2D5D3F4F3093520E2093510E4F
:10F350002091530E3091540E235231093093540EA4
:10F360002093530E90914E0F9F3049F490914F0F80
:10F370009F3029F41092F5101092F41008C02091DB
:10F380009D0F30919E0F3093F5102093F41022E1E1
:10F3900030E03093F2102093F11020916D0A3091FB
:10F3A0006E0AA9E5BEE0EDE9F0E141E0B683A58390
:10F3B0009C91992329F0891718F040832F5F3F4FC4
:10F3C0001A96379690E1E13FF90781F730936E0A7C
:10F3D00020936D0A2131310534F080E190E0909363
:10F3E0006E0A80936D0A0E945B848AEF90E190938D
:10F3F00000108093FF0F8091FE109091FF1090936A
:10F40000FE0F8093FD0F87EF90E1909302108093A1
:10F41000011088EF90E1909304108093031086EF21
:10F4200090E1909306108093051084E091E1909311
:10F430000A108093091080910811909109119093FE
:10F4400008108093071081E091E190930C10809355
:10F450000B1082E091E190930E1080930D1080E0EC
:10F4600091E19093101080930F108EE091E19093B2
:10F470001410809313108091121190911311909396
:10F480001210809311108BE091E1909316108093ED
:10F4900015108CE091E190931810809317108AE07A
:10F4A00091E190931A108093191088E191E1909363
:10F4B0001E1080931D1080911C1190911D1190932E
:10F4C0001C1080931B1085E191E190932010809394
:10F4D0001F1086E191E1909322108093211084E126
:10F4E00091E1909324108093231020916D0A309124
:10F4F0006E0A2450310960E07AE0C7E0462F50E000
:10F500004217530724F5CA010496789FF001799FAA
:10F51000F00D1124E350F04FC49FC001C59F900D22
:10F520001124AC0141565F4E53834283DC01A35644
:10F53000BF4E15964D915C9116975183408382562C
:10F540009F4E95838483B187A0876F5FD7CF81E07B
:10F5500080936F0ACF9108950F931F93CF93DF93FA
:10F56000FC01248135812115310519F4FB0110823C
:10F5700011C0EA0121972C173D0708F4E9018B011E
:10F58000FC0160817181AE01C8010E94C1ACC00F55
:10F59000D11F1882DF91CF911F910F910895FC0127
:10F5A000128213821482158216821782128608959F
:10F5B00080E008950F931F93CF938C0169E178E168
:10F5C00089E898E00E943A4CD8011896ED91FC9198
:10F5D00019976081718189E898E0FED9C1E0D8016E
:10F5E0001A968C91C81700F564E178E189E898E0F3
:10F5F0000E943A4C6C2F89E898E08BDD61E178E15C
:10F6000089E898E00E943A4CF80190858185E92FBD
:10F61000F82FEC0FF11DEC0FF11D6081718189E86D
:10F6200098E0DAD9CF5FDBCFCF911F910F9108958A
:10F63000CF93DF93CDB7DEB76E970FB6F894DEBFEA
:10F640000FBECDBF8F300CF080E029E038E13A8367
:10F65000298322E038E13C832B8324EF37E13E838A
:10F660002D8328EE37E138872F832EED37E13A8757
:10F67000298727ED37E13C872B8723ED37E13E874C
:10F680002D872CEC37E1388B2F8721EC37E13A8B33
:10F69000298B24EB37E13C8B2B8B29EA37E13E8B1E
:10F6A0002D8B2DE937E1388F2F8B2BE837E13A8FFF
:10F6B000298F2AE737E13C8F2B8F25E737E13E8FF3
:10F6C0002D8FE82FEE0FFF0BEC0FFD1F8181928134
:10F6D0006E960FB6F894DEBF0FBECDBFDF91CF910F
:10F6E0000895AF92BF92CF92DF92EF92FF920F9365
:10F6F0001F93CF93DF938DEE91E17EE1D72ED80E4D
:10F70000CC24C39402E010E0C3E0D0E0E2E0BE2EDF
:10F71000EE24E394F12C8091F60C9091F70CDC012F
:10F72000ED91FC910480F581E02D1995892B09F468
:10F73000ADC0A09030018091F60C9091F70CDC01E7
:10F74000ED91FC910680F781E02D199596B3B39A5F
:10F750002091840030918500285A344E30938D00DA
:10F7600020938C002A2D2C7119F01092F30C4BC0B1
:10F7700093FB992790F9E091F30CE11116C09923BE
:10F7800051F2803241F6C092F30C8093ED118091DA
:10F79000131290911412892B09F0BDCFF09214121C
:10F7A000E09213121092F50CB6CF9111DECFE1303A
:10F7B00041F4803409F0AFCFB092F30C8093EE1196
:10F7C000E6CF91E09E0F9093F30CF0E0E351FE4EF4
:10F7D0008083903209F09FCF1092F30CEDEEF1E1AF
:10F7E0002FEF3FEF8191281B3109DE12FBCF4091B3
:10F7F0000B1280910C1290E0982F8827840F911D96
:10F800002817390729F0D0931412C093131283CF0D
:10F810008091131290911412019739F48091F50C94
:10F820008F5F8093F50C843020F0109314120093B6
:10F8300013128091F40C8F5F8093F40C9091F20C72
:10F84000981708F5C092151220E030E0F901E35155
:10F85000FE4E4281838190E0982F8827840F911D6E
:10F86000AC014F5E52404B3D554028F4F901E85041
:10F87000F34F918380832E5F3F4F2C31310531F759
:10F880001092F40C48CF1092151245CFDF91CF9112
:10F890001F910F91FF90EF90DF90CF90BF90AF90AE
:10F8A0000895EF92FF920F931F93CF93DF931092DF
:10F8B000340E82E08093350E68EE73E07093370E5D
:10F8C0006093360E40ED57E05093390E4093380E5A
:10F8D0002CED35E030933B0E20933A0E8FE0809371
:10F8E0003C0E10923D0E94E090933E0E7093400EAD
:10F8F00060933F0E5093420E4093410E3093440E5E
:10F900002093430E8093450E1092460E93E0909301
:10F91000470E7093490E6093480E50934B0E4093E0
:10F920004A0E30934D0E20934C0E80934E0E109243
:10F930004F0E91E09093500E7093520E6093510EC3
:10F940005093540E4093530E3093560E2093550E01
:10F950008093570E1092580EE9E5FEE0A2E6BEE055
:10F9600080E008EE13E060ED77E04CED55E031E02B
:10F9700022E095E0980F9083128301837483638360
:10F9800056834583ED01229791E0388321962883A1
:10F990001C928F5F3A961A968C3059F71092D10EBE
:10F9A0009093D20E1092D30E9093D40E80E090E0FC
:10F9B0009C012C5C314FF901EF55FF4F11821082F1
:10F9C0003296108203968837910591F784E290E091
:10F9D0009093D60E8093D50E81E08093D70E2CE0C5
:10F9E00030E03093D90E2093D80E94E09093DA0E45
:10F9F00021E230E03093DC0E2093DB0E27E02093F1
:10FA0000DD0E29E030E03093DF0E2093DE0E20E1A2
:10FA10002093E00E7AE070934D0F2BE020934E0F71
:10FA200020934F0F48EE53E05093510F4093500FE7
:10FA300020ED37E03093530F2093520F1092540F64
:10FA400064E66093550F6093560F5093580F4093A0
:10FA5000570F30935A0F2093590F10925B0F10924B
:10FA60005C0F80935D0F10925F0F10925E0F80937A
:10FA7000600F8093610FE8ECF0E0F093630FE09388
:10FA8000620FE0E2F3E0F093650FE093640F5093B0
:10FA9000670F4093660F3093690F2093680F809330
:10FAA0006A0FE9E5F0E0F0936C0FE0936B0FE0E88C
:10FAB000F0E0F0936E0FE0936D0FEFEFF0E0F09356
:10FAC000700FE0936F0FF093720FE093710F8093BC
:10FAD000730F9093740F1092750F8093760F90931D
:10FAE000770F1092780F1092790F80937A0F1092FF
:10FAF0007B0F10927C0F80937D0F10927E0F98E207
:10FB000090937F0F5093810F4093800F5093830FFA
:10FB10004093820F3093850F2093840F8093860F3C
:10FB200092E39093870FE2E0E093880F8093890F30
:10FB300060938A0FE6E4E0938B0F90938C0F109202
:10FB40008D0F10928E0F10928F0F1092900F1092B7
:10FB5000910F1092920FEAEFF0E0F093940FE09380
:10FB6000930F1092950F1092960F6093970F61E488
:10FB70006093980F1092990F90939A0F10929B0F89
:10FB800090939C0FEEE5F1E0F0939E0FE0939D0FB4
:10FB900010929F0FACEDB5E0B093A10FA093A00F12
:10FBA00000EA1FE01093A30F0093A20F3093A50F5C
:10FBB0002093A40FC8E8D3E1D093A70FC093A60F5A
:10FBC00068EBE62E6BE0F62EF092A90FE092A80FFC
:10FBD000E0E4FFE1F093AB0FE093AA0F1092AC0FBB
:10FBE0001092AD0F1092AE0F69E16093AF0F80934A
:10FBF000B00F8093B10F8093B20F5093B40F409326
:10FC0000B30F3093B60F2093B50FF092B80FE09278
:10FC1000B70F1093BA0F0093B90FD093BC0FC093D6
:10FC2000BB0F20E737E13093BE0F2093BD0F10923A
:10FC3000BF0F1092C00F1092C10F9093C20F9093FC
:10FC4000C30F9093C40F8093C50F1092D50F1092DD
:10FC5000C60F99E09093C70F1092C80F1092C90F6A
:10FC60001092CA0F1092CB0FB093CD0FA093CC0F70
:10FC7000F093CF0FE093CE0F8093D00F7093D10FFE
:10FC80001092D20F21E030E03093D40F2093D30FA5
:10FC900040E052EC61E070E04093D60F5093D70FF4
:10FCA0006093D80F7093D90F4093DA0F5093DB0F06
:10FCB0006093DC0F7093DD0F40E056E960E070E088
:10FCC0004093DE0F5093DF0F6093E00F7093E10FCE
:10FCD0004093E20F5093E30F6093E40F7093E50FAE
:10FCE0001092E60F20E039E13093E80F2093E70F00
:10FCF0001092E90F9EE19093EA0F1092EB0F2EE124
:10FD000030E03093ED0F2093EC0F3093EF0F209302
:10FD1000EE0F3093F10F2093F00F9093F20F90932A
:10FD2000F30F8093F40F8093F50F1092F60F9093DA
:10FD3000F70F8093F80F8AE29FE4A0E0B0E0809391
:10FD4000F90F9093FA0FA093FB0FB093FC0F04E30D
:10FD50001EE0C0E0D0E0CE010E94BAAEF801619191
:10FD60008F01861719F0CE010E94CCAE2196C93CB6
:10FD7000F1E0DF0781F7DF91CF911F910F91FF90A5
:10FD8000EF9008954F925F926F927F928F929F9221
:10FD9000AF92BF92CF92DF92EF92FF92CF93DF9319
:10FDA000EB01A091EB11B091EC119D012F5F3F4F42
:10FDB00045E0429F2001439F500C1124052C000C6C
:10FDC00066087708812C912C54012A33E1E03E0724
:10FDD000ECF447E253E761E0772775016401C40C56
:10FDE000D51CE61CF71C4C0D5D1D6E1D7F1D6BBFE9
:10FDF000FA014791569165E0860E911CA11CB11C39
:10FE0000C417D50729F12F5F3F4FDFCF25E0822EA2
:10FE1000912CA12CB12C21E030E0A217B30708F4FB
:10FE20004CC047E253E761E07727480D591D6A1D32
:10FE30007B1D6BBFFA0147915691F5E08F0E911C27
:10FE4000A11CB11CC417D50719F02F5F3F4FE5CF98
:10FE500047E253E761E07727E5E0E29F6001E39F37
:10FE6000D00C11240D2C000CEE08FF084E5F5F4FE4
:10FE70006F4F7F4F4C0D5D1D6E1D7F1D6BBFFA01D7
:10FE800047915691FC015383428347E253E761E077
:10FE900077274C5F5F4F6F4F7F4FC40ED51EE61E16
:10FEA000F71EEBBEF601C790FC01C4823093EC1143
:10FEB0002093EB11C901019606C01092EC1110922B
:10FEC000EB1180E090E0DF91CF91FF90EF90DF9019
:10FED000CF90BF90AF909F908F907F906F905F90EA
:10FEE0004F9008950F931F938091E61181111EC0CA
:10FEF0000E9460510091E7111091E8112091E911E1
:10FF00003091EA11AB01BC01401B510B620B730B2A
:10FF10008091E4119091E511A0E0B0E0841795077D
:10FF2000A607B70718F481E08093E6111F910F919F
:10FF300008958091E4119091E511892B89F08091C9
:10FF4000E611882381F00E9460516093E71170935D
:10FF5000E8118093E9119093EA111092E611089547
:10FF600081E08093E61108951F920F920FB60F92D1
:10FF700011242F938F939F931092950010929400C9
:10FF80008091640A8F5F8093640A9091621289174E
:10FF900084F01092640A2091660A80916D1290910B
:10FFA0006E12820F911D27FD9A9590936E12809389
:10FFB0006D128091630A8F5F8093630A9091721231
:10FFC000891784F01092630A2091650A809170125B
:10FFD00090917112820F911D27FD9A959093711245
:10FFE000809370129F918F912F910F900FBE0F9061
:10FFF0001F9018958091620A811104C08091610A56
:020000021000EC
:10000000882321F080917100826003C0809171008B
:100010008D7F8093710008951F93CF93DF931F927C
:10002000CDB7DEB710E0181731F089830E946F60FA
:100030001F5F8981F8CF0F90DF91CF911F910895B5
:10004000CF93DF9360E088E00E94B24F1092E311FB
:10005000C091E111D091E211BE0185E89AE00E94C1
:10006000BC3F882329F0BE0185E89AE00E94D43F76
:1000700081E08093E01180915506882341F06BE583
:1000800077E180915306909154060E94AB4DDF9129
:10009000CF910C9445576091E70F7091E80F80E085
:1000A00090E00E9495AD20E030E04AE754E40E94E1
:1000B000F0A9AB01BC0121E0809153069091540658
:1000C0000C94BB4C6CE477E18091530690915406FC
:1000D0000E943A4C60919C0F809153069091540677
:1000E00018D890919C0F8091AF05981779F06CE328
:1000F00077E180915306909154060E943A4C6091AA
:10010000AF05809153069091540603D86AE377E1D6
:1001100080915306909154060C943A4C6BE277E12F
:1001200080915306909154060E943A4C60919A0F28
:1001300080915306909154060E94897890919A0F6D
:100140008091B005981781F06BE177E180915306BB
:10015000909154060E943A4C6091B00580915306EC
:10016000909154060E94897869E177E18091530665
:10017000909154060C943A4C482F50E095E1899F99
:10018000F0011124E25EFE4E21813281808591854D
:10019000280F391F838194818217930728F0858166
:1001A000968128173907E8F485E1849FF001859F3F
:1001B000F00D1124E25EFE4E8581968128173907E5
:1001C00028F52581368185E1849FF001859FF00D1A
:1001D0001124E25EFE4E8285823019F4118610866B
:1001E000128685E1849FF001859FF00D1124E25E67
:1001F000FE4E328321838091840090918500280FE8
:10020000391F309389002093880008958381948159
:1002100082179307C0F623813481D5CF80916A0A73
:10022000811157C0E091FE10F091FF1085819681F9
:100230009093FB108093FA101092FD101092FC1016
:10024000E0910811F0910911858196819093051133
:10025000809304111092071110920611E09112116F
:10026000F09113118581968190930F1180930E1157
:100270001092111110921011E0911C11F0911D11AA
:1002800085819681909319118093181110921B11FA
:1002900010921A1182E190E09093F2108093F11085
:1002A00081E08093F7108093011180930B1180936C
:1002B00015118093F31080E090E021E0FC01E356FB
:1002C000FF4E2183079684359105C1F781E0809325
:1002D0006A0A089510921711089510920D11089549
:1002E0008A3010F40C94294108958A3058F495E12D
:1002F000899FF0011124E25EFE4E818192819695E4
:100300008795089580E090E008958A3010F40C9469
:10031000444108951F920F920FB60F9211240BB60D
:100320000F920F931F932F933F934F935F936F936E
:100330007F938F939F93AF93BF93CF93EF93FF934D
:1003400080916112893048F0109261128091CD1134
:10035000882399F08091C6110DC0E0916112E1509F
:1003600025E1E29FF0011124E25EFE4E87818823A1
:1003700021F0808192B1892782B9E091611285E1F3
:10038000E89FF0011124E25EFE4E8781882321F070
:10039000808192B1892B82B9E0916112C5E1CE9F33
:1003A000F0011124E25EFE4E80859185892B09F0D3
:1003B0004DC0E0916112CE9FF0011124E25EFE4E2D
:1003C0008285813009F060C00E946051E091611225
:1003D000CE9FF0011124E25EFE4E03851485258533
:1003E0003685E0916112CE9FF0011124E25EFE4E4F
:1003F0000784F089E02DAB01BC01401B510B620B5F
:10040000730BCF01A0E0B0E084179507A607B707EC
:10041000D8F5E0916112A0916112CA9FD001112418
:10042000A25EBE4E53968D919C915497CE9FF00143
:100430001124E25EFE4E91878087E0916112CE9F8B
:10044000F0011124E25EFE4E82E08287809161120B
:1004500093DE809161128F5F80936112FF91EF9123
:10046000CF91BF91AF919F918F917F916F915F914C
:100470004F913F912F911F910F910F900BBE0F90B5
:100480000FBE0F901F901895E0916112809184002B
:100490009091850025E1E29FF0011124E25EFE4E7D
:1004A00021813281820F931F90938900809388006D
:1004B000D0CF1F93CF93DF9380916012811173C0CF
:1004C000109261129FB7F89485E128EB3BE04CED68
:1004D00055E064E971E1A1E0B0E0E0916112E9303A
:1004E00008F052C0E09161128E9FF0011124E25E8B
:1004F000FE4E32832183E09161128E9FF001112420
:10050000E25EFE4E56834583E09161128E9FF001BC
:100510001124E25EFE4E74836383E0916112F091D8
:100520006112ED0101C0CC0FFA95EAF78E9FF00140
:100530001124E25EFE4EC083E09161128E9FF001B5
:100540001124E25EFE4E1782E09161128E9FF0014F
:100550001124E25EFE4E11861086E09161128E9F9C
:10056000F0011124E25EFE4E1286E09161128E9F30
:10057000F0011124E25EFE4E148A138AE0916112AA
:10058000EF5FE0936112A9CF9FBF8FB7F89420EA85
:100590003FE03093C8112093C7111092C6118FBF4E
:1005A00081E080936012DF91CF911F9108950F93A6
:1005B0001F93CF93DF938C01C62FD42FDC011196AC
:1005C0008D919C911297DC01ED91FC910190F0814D
:1005D000E02DD8016C911995F80181819281DC019F
:1005E000ED91FC910190F081E02D6C2F1995F801AF
:1005F00081819281DC01ED91FC910190F081E02DEF
:100600006D2F1995F80180816C2F70E0680F711DB6
:100610006D0F711D6F77772781819281DF91CF9167
:100620001F910F910C94206A0F931F93CF93DF9328
:100630008C01C62FD42FDC0111968D919C911297BD
:10064000DC01ED91FC910190F081E02DD8016C91DD
:100650001995F80181819281DC01ED91FC91019065
:10066000F081E02D6C2F1995F80181819281DC01D8
:10067000ED91FC910190F081E02D6D2F1995F8011D
:1006800080816C2F70E0680F711D6D0F711D6F7789
:10069000772781819281DF91CF911F910F910C94E7
:1006A000206A4F925F926F927F92AF92BF92CF92E9
:1006B000DF92EF92FF921F93CF93DF93DD24D394C9
:1006C00045E0C42E52E0A52EB12CC3E0D0E0EE24CC
:1006D000E394F12C8091441290914512DC01ED914C
:1006E000FC910480F581E02D1995892B09F4BEC099
:1006F000109130018091441290914512DC01ED91EE
:10070000FC910680F781E02D199596B3B39A20915C
:100710008400309185002059384E30938D0020930D
:100720008C00212F2C7139F010925F12D09343125C
:10073000C0934212CFCF93FB992790F9E0915F12BB
:10074000E11116C0992331F28F3021F6D0925F1259
:10075000809346128091421290914312892B09F0A6
:10076000B9CFF0924312E092421210924112B2CFEE
:100770009111DACF91E09E0F90935F12F0E0EA5B67
:10078000FD4E8083993109F0A5CF81116CC0809115
:100790005D1282FF05C0D0934312C093421263C022
:1007A00083FDF9CF8091421290914312019739F461
:1007B000809141128F5F80934112843020F0B0927B
:1007C0004312A0924212809140128F5F8093401298
:1007D00090913F12981708F044C0D0923E12AEE1BB
:1007E000B2E1E7E4F2E140E050E0BA0110E0CF010D
:1007F000FC011B3098F401964080512C612C712C27
:10080000012E04C0440C551C661C771C0A94D2F7B8
:100810004429552966297729185FEACF9A0137704C
:10082000205E3340C29EC001C39E900D112497FDEF
:10083000079623E0959587952A95E1F784529A4F7C
:100840008D939D931B503BE0769567955795479503
:100850003A95D1F782E1AE33B80749F610924012CB
:1008600002C010923E1210925F1234CFDF91CF91EE
:100870001F91FF90EF90DF90CF90BF90AF907F904F
:100880006F905F904F9008958091700A833031F49B
:1008900080911C1290911D120C94717B089580918F
:1008A000700A823029F480911A1290911B12F9CEAD
:1008B0000895F5DFE9CF1092F71010920111109210
:1008C0000B11109215111092F31080E090E0FC01D2
:1008D000E356FF4E1182079684359105C1F70895BE
:1008E0008091700A823039F0833049F0813049F4C8
:1008F0008091171201C080E180936C0A04C08EE0E1
:10090000FBCF10926C0A80916C0A08958091700A56
:10091000823039F0833049F0813059F480911612D9
:100920000895BDDF80913E120895AEDF80911512CB
:10093000089580E008958091700A823049F08330F4
:1009400069F0813089F4809111129091121208950A
:10095000A6DF8091421290914312089595DF809115
:10096000131290911412089581E090E008958F92EF
:100970009F92AF92BF92CF92DF92EF92FF921F931E
:10098000CF93DF93EC0111E08E819F81892B09F4D5
:1009900010E02C813D81E885F985C580D68087816E
:1009A00090E0A601480F591F2417350764F1808590
:1009B0000D2C000CEE08FF08A901330F660B770B16
:1009C0000380F481E02D9A01AB012C193D094E09F9
:1009D0005F09882329F0A1E0BFEF0E9402AF04C0A5
:1009E000AFEFB0E00E94F6AE4F01FF0FAA08BB08C0
:1009F000A50194012C193D094E095F090E94DAAE48
:100A00003F832E834BC0A601481B590B4217530747
:100A10000CF43FC080850D2C000CEE08FF08A901E6
:100A2000330F660B770B81809280092C000CAA088B
:100A3000BB089A01AB01281939094A095B098823C7
:100A400099F0A1E0BFEF0E9402AFA701960128191B
:100A500039094A095B090E94DAAEDA01C9018150FD
:100A60009F4FAF4FBF4F12C0AFEFB0E00E94F6AE46
:100A7000A7019601281939094A095B090E94DAAED3
:100A8000DA01C9018F5F9109A109B1099F838E83A2
:100A900005C01F821E82111101C019828E819F81A3
:100AA000009789F08F3F910519F014F08FEF90E0D7
:100AB00081305FEF950714F481E09FEF9F838E8371
:100AC00081E018271A83DF91CF911F91FF90EF905B
:100AD000DF90CF90BF90AF909F908F900895CF936D
:100AE000DF93C0910D12D0910E1260910F12709190
:100AF0001012CE010E94BC3F81110DC02EE031E8E2
:100B00004CE251E060E070E0CE010E9423409093FF
:100B1000101280930F12DF91CF9108954115510566
:100B200029F06115710511F00C94AC7A0895EF92DB
:100B3000FF920F931F93CF93DF931F921F92CDB716
:100B4000DEB78C018CE789831A82F801E480F58096
:100B5000FFEFEF1AFF0AB701C8010E942A4B882352
:100B600081F0F8012081318184819581BE016F5F20
:100B70007F4F820F931F0E94BAACF801F582E48286
:100B800081E00F900F90DF91CF911F910F91FF9017
:100B9000EF900895AF92BF92CF92DF92EF92FF92C3
:100BA0000F931F93CF93DF9300D01F92CDB7DEB783
:100BB0008C0149835A836B837C83CE0101966C013F
:100BC000580194E0A90EB11CE12CF12CC8010E943F
:100BD000BAAEF60161916F01861731F0C8010E942B
:100BE000CCAEFFEFEF1AFF0A0F5F1F4F0A151B0570
:100BF00069F781E0EF2809F480E00F900F900F90E3
:100C00000F90DF91CF911F910F91FF90EF90DF90A8
:100C1000CF90BF90AF900895CF92DF92EF92FF9266
:100C20000F931F93CF93DF93EC0100917312E0E0D9
:100C3000F0E020E030E0A90110E0CE17DF071CF162
:100C4000309711F40D32E1F0DF01AD58BD4EFC904C
:100C500080ED8F0D8A30A8F4AAE0B0E00E94F6AED5
:100C60002F2DFF0C330B205331096901330FEE0890
:100C7000FF089B01AC012C0D3D1D4E1D5F1D01C0E9
:100C800011E03196DACFCA01B901112339F09095FC
:100C90008095709561957F4F8F4F9F4FDF91CF91DA
:100CA0001F910F91FF90EF90DF90CF90089580916A
:100CB000740A811105C081E09091760A911101C0FA
:100CC00080E00895CF93DF932091A0093091A1098E
:100CD000E9012697A881B981A056B64F12961C92B9
:100CE000082E000C990BAA0BBB0BFC013197EE30C0
:100CF000F10508F057C18827ED59FE4F8F4F0C942E
:100D000077A9F9013A97808191818056964F0E9488
:100D100056A7882309F44BC1E091A009F091A109DD
:100D200036970190F081E02DE056F64F81E0A0C0AB
:100D3000F9013C97808191818056964F0E9493A63D
:100D4000882309F434C1E091A009F091A1093697F4
:100D50000190F081E02DE056F64F82E089C0F90164
:100D60003E97808191818056964F0E94D6A5882318
:100D700009F41DC1E091A009F091A10936970190F5
:100D8000F081E02DE056F64F83E072C0F9017097D4
:100D9000808191818056964F0E9459A5882309F43D
:100DA00006C1E091A009F091A10936970190F08168
:100DB000E02DE056F64F84E05BC0F9017297808128
:100DC00091818056964F0E9414A5882309F4EFC0A4
:100DD000E091A009F091A10936970190F081E02DF2
:100DE000E056F64F85E044C0F90174978081918107
:100DF0008056964F0E949BA4882309F4D8C0E091A6
:100E0000A009F091A10936970190F081E02DE056FC
:100E1000F64F86E02DC0F90176978081918180564A
:100E2000964F0E9415A4882309F4C1C0E091A0093F
:100E3000F091A10936970190F081E02DE056F64F30
:100E400087E016C0F9017897808191818056964F8E
:100E50000E9407A4882309F4AAC0E091A009F09198
:100E6000A10936970190F081E02DE056F64F88E019
:100E700082839DC0F901B097808191818056964F01
:100E80000E9429A1882309F492C0E091A009F09161
:100E9000A10936970190F081E02DE056F64F83814D
:100EA0009481A581B6814097A105B10509F07FC065
:100EB0008EC0F9017A97808191818056964F0E9469
:100EC0003CA3882309F473C0E091A009F091A10923
:100ED00036970190F081E02DE056F64F8AE0C8CFBA
:100EE000F9017C97808191818056964F0E9471A272
:100EF000882309F45CC0E091A009F091A10936971C
:100F00000190F081E02DE056F64F8BE0B1CFF90172
:100F1000B097808191818056964F0E9429A18823A5
:100F200009F445C0E091A009F091A109369701901C
:100F3000F081E02DE056F64F83819481A581B68142
:100F400080319440A105B10591F543C0F9017E9728
:100F5000808191818056964F0E94A2A1882339F109
:100F6000E091A009F091A10936970190F081E02D60
:100F7000E056F64F8DE07CCFF901B09780819181EA
:100F80008056964F0E9429A1882389F0E091A009FC
:100F9000F091A10936970190F081E02DE056F64FCF
:100FA0008EE066CFE881F981E056F64F1282E0913B
:100FB000A009F091A10936970190F081E02DE0564B
:100FC000F64F81E09281911106C080E004C089E073
:100FD0004FCF8CE04DCFDF91CF910895EF92FF92EC
:100FE0000F931F93CF93DF931F921F92CDB7DEB75E
:100FF00041110AC07C0197FF03C0F194E194F1080C
:10100000E616F70664F402C0E12CF12C81E080932F
:10101000610A8FEF633371059CF425E012C06E15F1
:101020007F0534F01092610A81E091E021E00AC06E
:101030006D337105BCF381E08093610A23E001C048
:1010400024E092E03091610A332379F03FB7F894BD
:10105000899F902D11249093650A2093721200911C
:101060007012109171123FBF0AC09FB7F89410928E
:10107000650AF0927112E09270129FBF87014A8355
:1010800089830E94FA7F4A818981442319F017FFDE
:1010900019C014C0813031F417FD10C0E016F106FC
:1010A0008CF40FC08F3F71F40E151F0554F00F3FE5
:1010B000110541F03CF00FEF10E004C000E010E03B
:1010C00001C08701C8010F900F90DF91CF911F9150
:1010D0000F91FF90EF900895CF92DF92EF92FF92E1
:1010E0000F931F93CF93DF93042FE22E433049F0E9
:1010F000453039F0443041F4F92EFF1CFF24FF1C29
:1011000004C0FF24F39401C0F12CFC0197FF03C03D
:10111000F195E195F109EF011092620A013009F4AD
:1011200032C1053009F06EC080918212811118C061
:10113000C0916F12D0E0D0938112C093801281E0F1
:101140008093620A21E030E030937F1220937E1278
:1011500030936E1220936D128093821211E0B9C009
:1011600080916D1290916E1281159640E8F581E0A4
:101170008093620A80916D1290916E1220917E127E
:1011800030917F12821B930BC0918012D0918112FB
:10119000089720F1BE0180E090E00E9495AD20917B
:1011A000691230916A1240916B1250916C120E9438
:1011B000F6AD20E030E040E05FE30E948CA90E94A1
:1011C00058AAEB01709381126093801280916D1286
:1011D00090916E1290937F1280937E12CF31D10541
:1011E0000CF075C0E1E001C0E0E01092620A1092DC
:1011F000811210928012109282128E2F11E0C0E0A4
:10120000D0E061C0EE20E1F0023029F480915D0A67
:1012100090915E0A04C080915F0A9091600AE8177D
:10122000F9070CF0B3C081E08093620A80916812E4
:1012300094E0F595E7959A95E1F7EE5F1FEF43C0CF
:10124000DB0177FF03C0B195A195B109AE17BF07C8
:10125000C4F480916712882309F49CC081E08093D4
:10126000620A80916612909165129130A1F5EA1B95
:10127000FB0BFD970CF0845011E054976CF5E4E003
:101280002CC0EA17FB070CF085C0809164128823FC
:1012900009F480C0043009F47DC081E08093620AC3
:1012A0008091681290916312913009F07CC0E23312
:1012B000F10514F48E5F77C0AE1BBF0BD3970CF40F
:1012C00072C0825070C01E1644F0E1E006C011E00A
:1012D00081E0E1E006C011E0E2E0181614F06E01D2
:1012E00060C06E019091620A9923D9F02FB7F894EB
:1012F0001E9F902D11249093660A809362121C16F3
:101300001D063CF480916D1290916E12892B09F4A8
:101310004CC0053021F0C0916D12D0916E122FBFDC
:1013200009C08FB7F8941092660AD0936E12C093DA
:101330006D128FBF0E94FA7FEE2019F0D7FF1DC0FB
:1013400018C0113031F4D7FD14C0CC16DD06ACF452
:1013500013C01F3F91F4023011F0033071F4CC152B
:10136000DD0554F0CF3FD10541F03CF0CFEFD0E0A8
:1013700004C0C0E0D0E001C0E601FF2001F1D1953A
:10138000C195D1091CC090E080E006C090E080E0EB
:101390001FEF03C09E2F8F2F11E06F01C92FD82F91
:1013A000E1E081E09FCF1FEF97CF8091660A082E82
:1013B000000C990B90936E1280936D12AACFCE0100
:1013C000DF91CF911F910F91FF90EF90DF90CF9021
:1013D0000895CF92DF92EF92FF9297FF26C0CC2420
:1013E000DD24C61AD70A0D2C000CEE08FF08092EC2
:1013F000000CAA0BBB0B9C01AD0121503F4F4F4F7E
:101400005F4FC701B60160957095809590950E94D9
:1014100041A92EEF30E040E050E00E94DAAEC20E6B
:10142000D31EE41EF51EC60126C0009711F1092E39
:10143000000CAA0BBB0B9C01AD01215031094109E5
:101440005109CB01770FAA0BBB0BBC01CD01615039
:101450007109810991090E9441A92EEF30E040E015
:1014600050E00E94DAAEDA01C9010196A11DB11D5A
:1014700002C080E090E0FF90EF90DF90CF90089561
:1014800080910602813019F485E080930602089568
:1014900010924A060895CF93DF93C0919212D09193
:1014A0009312BE0185E89AE00E94BC3F882329F090
:1014B000BE0185E89AE00E94D43F109293121092E8
:1014C0009212DF91CF9108950F931F93CF93DF93E3
:1014D00080918E0F90918F0FA091900FB091910FEE
:1014E000181619061A061B060CF044C00E94727FDB
:1014F0008091B3058823C9F1009192121091931243
:10150000B80185E89AE00E94BC3F8823D9F0E3E85F
:10151000FCE0C0E0D0E0819191918017910769F4DF
:101520000E946051CC0FDD1FCC0FDD1FCB57D54F74
:10153000688379838A839B831DC02196CE31D10530
:1015400051F718C040918E0F50918F0F6091900FFE
:101550007091910F2BEF3AE885E89AE00E942340C2
:10156000909393128093921205C0DF91CF911F91B7
:101570000F9191CFDF91CF911F910F91089580919D
:101580005A0A811137C00E94727F8091E611882328
:10159000B1F08091B305882391F01092B3051092B9
:1015A000E6110E94997F80918512882341F066E1BF
:1015B00079E180918312909184120E94AB4D8091C9
:1015C0004B06882311F081E001C080E0DED281E08B
:1015D0008093DE050E946B5C80914F0690915006CF
:1015E000DC01ED91FC910480F581E02D19950E94BC
:1015F000695B6ACF08950E94727F8091B30588234A
:1016000069F0BDDF80915506882341F066E279E1FB
:1016100080915306909154060C94AB4D089580919F
:101620005A0A811155C080914C06823068F0809131
:101630005506882309F44CC064ED78E18091530687
:10164000909154060C94AB4D0E94727F8091E611EC
:10165000882309F43DC08091B305811139C081E030
:101660008093B3051092E6110E94997F80918512B4
:10167000882341F065EC78E1809183129091841287
:101680000E94AB4D80914F0690915006DC01ED9188
:10169000FC910280F381E02D199580914C06811117
:1016A00016C04091840F5091850F81E08093DE0534
:1016B0004115510551F060E070E020E439E585E81E
:1016C0009AE00E942340FDD102C00E944059FCCE06
:1016D0000895CF93823069F490917D0F20917A0F15
:1016E00030917E0F40917B0F50917C0F6091790F6C
:1016F0000CC09091770F2091740F3091780F40912A
:10170000750F5091760F6091730F6093671250932D
:101710006412409365123093631220936612909383
:101720006812909100028917B9F08093000290919D
:101730005506992389F0C82F6CEA78E18091530609
:10174000909154060E943A4C6C2F809153069091D0
:101750005406CF910C945F77CF910895833079F040
:1017600030F4813051F0823091F48BE30BC084303F
:1017700041F0853061F482E405C08CE303C080E46D
:1017800001C081E40E948A4F21E0892B09F420E006
:10179000822F0895E3DF91E0892708950F931F9327
:1017A00080918A1281110DC00E946051609386124F
:1017B00070938712809388129093891281E08093AE
:1017C0008A12809112028A3AF1F485E0C7DF8823F9
:1017D00071F08CEE97E09093EC0C8093EB0C90936F
:1017E0005406809353068FEF809312020CC089E851
:1017F00098E09093EC0C8093EB0C909354068093BC
:101800005306109212020E946051009186121091AC
:1018100087122091881230918912DC01CB01801B44
:10182000910BA20BB30BC397A105B10508F449C0F6
:101830000E94605160938612709387128093881281
:101840009093891285E08ADF882321F0809112022B
:10185000882349F085E082DF811133C08091120234
:101860008F3F79F518C08CEE97E09093EC0C809345
:10187000EB0C909354068093530680915506882371
:1018800031F062E978E18CEE97E00E94AB4D8FEF8A
:101890008093120216C089E898E09093EC0C809334
:1018A000EB0C909354068093530680915506882341
:1018B00031F06DE778E189E898E00E94AB4D109235
:1018C00012021F910F9108951092190E80915506E2
:1018D000882379F020915C0F8091530690915406F3
:1018E000222319F06DE478E102C060E678E10C94FF
:1018F000AB4D089581E08093190E809155068823A1
:1019000079F020915C0F8091530690915406222328
:1019100019F06FE178E102C061E378E10C94AB4D1E
:1019200008950F931F93CF93DF9320916A0F211196
:101930001BC0C091DC05D091DD05088119819C0197
:10194000AFEFB0E00E9428AF2FEF33E040E050E06F
:101950000E94DAAED801ED91FC91B901CE01DF9180
:10196000CF911F910F911994DF91CF911F910F91FA
:10197000089580914B0681110C946B5C0C94405936
:10198000FECD4DCE0E94727F8091B3058111F7CDBF
:1019900046CECF939C01A4E6B0E00E9428AF2FEF83
:1019A00033E040E050E00E94DAAEC22F30E0809198
:1019B0009412281B310937FF03C031952195310955
:1019C000233031053CF1C33020F0C23618F0C4E6B4
:1019D00001C0C0E080914F0690915006DC01ED916E
:1019E000FC91E25BFF4F0190F081E02D6C2F199587
:1019F000C093941280915506882361F06AE579E1DD
:101A000080915306909154060E943A4C8C2FCF91AE
:101A10000C94D95FCF9108959C010197849710F49D
:101A2000822F0895C901845691098438934040F467
:101A3000C90164E670E00E9450A9822F94E61BC0A1
:101A4000283E43E03407D8F0C90168EE73E00E94F5
:101A500050A948E15CEF649FC001659F900D749FA1
:101A6000900D1124280F391FC9016AE070E00E940F
:101A700064A9822F9AE0699F80191124089580E05B
:101A8000089567E679E180915306909154060C948D
:101A90003A4C80914F0690915006DC01ED91FC91FB
:101AA0000484F585E02D60E0199480914F069091B3
:101AB0005006DC01ED91FC910484F585E02D61E098
:101AC0001994CF93DF9380916A0F882349F1809115
:101AD0000102882329F1C091DC05D091DD0589A19F
:101AE0009AA1892B11F01AA219A28B8D9C8D9B872C
:101AF0008A872FEF30E03D872C879F878E87E8818C
:101B0000F9810190F081E02D60E070E0CE0119953F
:101B10001F8A1E8A0E9460516D8F7E8F8F8F98A3BF
:101B2000DF91CF910895CF93DF9380916A0F88233F
:101B300049F180910102882329F1C091DC05D091FF
:101B4000DD0589A19AA1892B11F01AA219A2898D0C
:101B50009A8D9B878A872FEF30E03D872C879F8760
:101B60008E87E881F9810190F081E02D60E070E0DE
:101B7000CE0119951F8A1E8A0E9460516D8F7E8F3B
:101B80008F8F98A3DF91CF9108951F93CF93DF9309
:101B900090916A0F9923C9F0182FC091DC05D0915C
:101BA000DD05CE010E94846C8E899F89892B49F4C2
:101BB000112319F0898D9A8D02C08B8D9C8D9F8B7E
:101BC0008E8B81E090E09AA389A3DF91CF911F9142
:101BD0000895809101028823B9F01092010280914A
:101BE0005506882341F06AE479E18091530690918B
:101BF00054060E94AB4D0E94727F8091B3058823EA
:101C000019F080914B06C1CF089580910102811196
